:020000040800F2
:1000000000200010911C0308B52502083960000883
:10001000B3250208B1250208AF2502080000000040
:10002000000000000000000000000000AD250208F4
:10003000AB25020800000000A92502085155000860
:10004000F91C0308F91C0308F91C0308F91C030830
:10005000F91C0308F91C0308F91C0308F91C030820
:10006000F91C0308F91C0308F91C03082D2E0008CD
:100070001D2E00080D2E0008FD2D0008ED2D000896
:10008000D92D0008C52D0008F91C0308F91C030828
:100090007D270208F91C0308F91C0308F91C030852
:1000A000494C0008A94C0008394C0008D14C000804
:1000B000994C0008894C0008794C0008F91C030889
:1000C000F91C0308F91C0308F91C0308F91C0308B0
:1000D000F91C03080156000885550008F91C03089F
:1000E000F91C0308F91C030899250208F91C0308E8
:1000F000594C0008F91C0308694C0008F91C030856
:10010000000000000000000000000000F91C0308CF
:10011000F91C0308F91C03082D38010811380108DF
:10012000B12D00089D2D0008892D0008752D0008AF
:10013000612D0008F91C0308000000000000000009
:10014000F91C0308F91C0308F91C0308000000004F
:10015000000000000000000000000000000000009F
:100160000000000000000000F91C0308F91C03084F
:10017000F91C03080000000000000000000000005F
:0801800000000000F91C030857
:10018800002870B51EDB0928044620DD012303EB97
:1001980083035B00B0FBF3F2092AF8D87BB10E4E5B
:1001A800B4FBF3F00928CCBF57223022A6FB03E5A5
:1001B800024403FB1044EB0801F8012BF0D10023A3
:1001C8000B7070BD2D230B7040420131DBE73030DE
:1001D80001F8010BF3E700BFCDCCCCCC884230B49A
:1001E8004FF001042ED301FB04F4B0FBF4F58D426B
:1001F800F9D284B1AAB901E0B0FBF4F5092DCCBF5E
:10020800572230222A4404FB150003F8012BB4FBC3
:10021800F1F4002CF0D100221A7030BC7047B0FB0A
:10022800F4F5092DCCBF372230222A4404FB1500EF
:1002380003F8012BB4FBF1F4002CF0D100221A7062
:1002480030BC70470546002AEBD1D7E703685A1C33
:1002580002601970704700BF2DE9F047089C2578A7
:10026800002B804689460CBF4FF0200A4FF0300A19
:10027800661C35B3002A29DD334601E0024698B1F1
:1002880013F8011B501E0029F8D1971E60B13D4696
:10029800013D51464046C8476B1C002BF8DC2578C9
:1002A80027EAE770013055B1041B29464046C84784
:1002B800301916F8015B002DF7D1BDE8F087BDE8CD
:1002C800F087002A04DC2846BDE8F0870020EBE729
:1002D800571EDCE783684268D0ED037A00EB8301A0
:1002E8000133934281ED040A836004BF00238360D5
:1002F80000EB830393ED047A036870EE277A9A4241
:10030800C0ED037A77EEC77AC0ED037A0CDA0133D1
:1003180007EE103AF8EEC76AB7EE007A87EEA60A3B
:10032800036030EE070A704707EE102AB8EEC77A66
:1003380087EE870A704700BF90ED057A90ED004A76
:10034800D0ED066AD0ED014AD0ED047A90ED035A5B
:10035800D0ED025AA4EE007AB0EE406AB0EE470A39
:10036800B0EE667AA6EE247A67EEC07AA0EE457AF9
:10037800E6EE257A80ED057AC0ED067A704700BF73
:10038800D0ED057A90ED013AD0ED003AD0ED064A6D
:1003980090ED024A90ED077A90ED035A90ED086AC5
:1003A800D0ED045AC0ED067AF0EE406A27EE830AD3
:1003B800C0ED056AA3EEA60A80ED087AA4EE240A29
:1003C800A5EE470AA5EEC60A80ED070A704700BFEA
:1003D800D0ED007A90ED017A30EE670AE7EE007A08
:1003E800B0EE670AC0ED007A704700BF704700BFE3
:1003F8000A44914214D030B40139551E41F2210209
:1004080011F8014F082380EA042004044CBF82EA53
:1004180040004000013B80B2F7D18D42F0D130BCA2
:1004280070474378007840EA032010FB01F04FF44E
:10043800807190FBF1F000F30F0000B270472DE9D6
:10044800F04F654B654EB3F80AC03468B3F80480C2
:1004580087B04FEA0C2A05901889B4EB0A0A4FF0C6
:1004680000024FF0000565EB020BA0FB0A4500FBFC
:100478000B55E00940EA45604FEA084407198E46E3
:10048800D8884FEAE51141EB0208A0FB0A45CDE9FF
:100498000278B3F8028000FB0B55200A40EA056099
:1004A8004FEAC83410EB04084FEA252141EB020952
:1004B8009A89A2FB0A0102FB0B11C20D42EA4122F2
:1004C80012F5FA604FEAE15343F10001B0F5FA6F13
:1004D800CDE9000171F10001B4465EDA0524A2FB02
:1004E800040104FB031100FB03F402FB0144DDE9F2
:1004F8000267A0FB020121444D104FEA3004361B6D
:100508004FEA900444EA817467EB05078D10B8EB55
:10051800040869EB0509DDE9004531484FF0FF3172
:10052800844275EB0101CDE9026723DA40F6AC504D
:1005380012184FF000014B4102FB03F1A2FB02230A
:1005480003EB4103D900D000101A41EA527163EB62
:100558000101341847EB0105CDE902450B24A2FB44
:10056800040104FB031149104FEA3000B8EB0008FE
:1005780069EB01090AFB0BF3DDE90001AAFB0AABF1
:100588000BEB430B4FEADA7242EA4B02801A4FEA4E
:10059800EB7361EB0301CDE90001DCF80410A1FB6A
:1005A800082301FB0933540D5D1544EAC324DDE932
:1005B8000223A21A65EB03031D46D30B059A43EAEF
:1005C800454302B11360BEF1000F02D0009BCEF884
:1005D800003007B0BDE8F08F68590020481D0020A2
:1005E80024FAFFFF90F8203033B1012B03D14FF4E8
:1005F80000638382704770474FF48063838270473B
:1006080070B40468037B2268022101FA03F31A42DA
:1006180013D042690A495C2000FB02124FF6FE76AD
:1006280050685289C5680068296831402960C168E6
:10063800D24392B20A40C260636070BC704700BF88
:10064800404E002030B40A4B1D7875B1094B00208C
:1006580003EBC5051A6899885062D4682143D160B4
:10066800083323F8040CAB42F4D130BC704700BF08
:100678002051002024510020F0B4334C00EB8000BE
:1006880004EB80046468002C5BD0304E49004FF4C2
:100698002040CDB2B060A169090444D460682C4FF1
:1006A80045F08071384041F4903101434FF42040C7
:1006B8006160B06003E0411E002838D00846A16997
:1006C8008F07F8D54FF42040A262B06002E0421EC6
:1006D80068B31046A2691106F9D562681C4945F04D
:1006E800007545F480350A4015434FF42040656095
:1006F800B06002E0421ED0B11046A2699207F9D557
:10070800A362A3694FF420409B06B06005D4431E42
:1007180068B11846A3699B06F9D52023B060E36148
:100728000120F0BC7047411E08B10846B3E7094AEA
:10073800138801339BB24FF0FF31B1601380F0BCD6
:1007480070472046F0BC704774560020481D0020B2
:10075800009800FC265200202DE9F04F83B080233A
:100768000190242219210020FFF786FFBE4CBF4DBF
:10077800DFF80093BE4EDFF800C34FF0640A4FF075
:1007880010084FF47A77D9F80430C3F30803002B24
:1007980040F03281EFF31183002B40F02D81216866
:1007A800B26800BF23689942F9D1286807FB00F3B3
:1007B8009B1AB3FBF0F307FB013101200091D9F834
:1007C8000430C3F30803002B40F0F980EFF31183E2
:1007D800002B40F0F4802368B16800BF2268934280
:1007E800F9D1D5F800B007FB0BF2521AB2FBFBF2B5
:1007F80007FB0323009A9B1AB3F57A7FDFD3BAF17C
:10080800010AC0D15046972320221921FFF734FF4F
:10081800DFF86092964EDFF860C24FF00A0A4FF098
:1008280010084FF47A77D9F80430C3F30803002B83
:1008380040F02481EFF31183002B40F01F812168E1
:10084800B26800BF23689942F9D1286807FB00F312
:100858009B1AB3FBF0F307FB013101200091D9F893
:100868000430C3F30803002B40F08C80EFF31183AE
:10087800002B40F087802368B16800BF226893424C
:10088800F9D1D5F800B007FB0BF2521AB2FBFBF214
:1008980007FB0323009A9B1AB3F57A7FDFD3BAF1DB
:1008A800010AC0D15046102323221921FFF7E4FE84
:1008B800DFF8C0916E48DFF8C0E14FF0640A4FF0EE
:1008C800100C4FF47A76D9F80430C3F30803002BE0
:1008D80040F0AE80EFF31183002B40F0A98021682F
:1008E800826800BF23689942F9D12F6806FB07F395
:1008F8009B1AB3FBF7F306FB013101270091D9F8E6
:100908000430C3F3080303BBEFF31183EBB9236887
:10091800816800BF22689342F9D1D5F800B006FB80
:100928000BF2521AB2FBFBF206FB0323009A9B1A46
:10093800B3F57A7FE3D3BAF1010AC4D1019A4FF42F
:100948008053938203B0BDE8F08FEFF311888CF3E6
:10095800128881680368DB0344BFCEF800708168A1
:100968002368DEF800205FFA88F888F31188D5F844
:1009780000801A4406FB08F35B1AB3FBF8F306FB86
:100988000233D3E7EFF3118E88F31288B168336826
:10099800DB0344BFCCF80000B1682368DCF8002012
:1009A8005FFA8EFE8EF31188D5F800E01A4407FB33
:1009B8000EF35B1AB3FBFEF307FB02336AE7EFF3B0
:1009C800118E88F31288B1683368DB0344BFCCF812
:1009D8000000B1682368DCF800205FFA8EFE8EF311
:1009E8001188D5F800E01A4407FB0EF35B1AB3FB35
:1009F800FEF307FB0233FDE6EFF3118288F312885A
:100A0800B0683368D90303D50123CCF80030B06847
:100A18002368DCF80010D2B282F311882A681944DE
:100A280007FB02F31B1AB3FBF2F307FB0131C4E621
:100A3800EFF311828CF3128887680368D90303D512
:100A48000123CEF8003087682368DEF80010D2B2A0
:100A580082F311882A68194406FB02F3DB1BB3FBF7
:100A6800F2F306FB013148E7D4560020D85600209F
:100A780010E000E000ED00E0D0560020EFF3118216
:100A880088F31288B0683368D90303D50123CCF8FA
:100A98000030B0682368DCF80010D2B282F3118805
:100AA8002A68194407FB02F31B1AB3FBF2F307FB8E
:100AB8000131D2E6002326220360027027228270C9
:100AC800012243600271837170472DE9F341056982
:100AD80006460F467DBBD0F80080C8F30A0323B34F
:100AE8000023D6F8008001932FF072FC042819D156
:100AF800214C236943F001032361BBB2A8F80030FD
:100B08002FF066FC04282ED108F102030193019B03
:100B18003F0C1F802FF05CFC2369042823F001039D
:100B2800236125D06FF0010505E02FF051FC042862
:100B380005D04FF0FF35284602B0BDE8F0810E4CD5
:100B4800236943F002032361C4F81480236943F046
:100B5800400323612FF03CFC2369042823F002039F
:100B68002361BDD0E5E7236923F001032361D9E7B9
:100B7800336804333360DEE700200240F8B50446EA
:100B88000D468E180027B54201D12069F8BDE368EB
:100B9800591CE160234415F8012B1A720429F2D17B
:100BA800A1682046FFF791FFE7602061EBE700BFEF
:100BB800014B186804F0BEBD901D002010B490E8E9
:100BC8000600047B40690223A3404B6013685DF86C
:100BD800044B4FF6FE710B40136004F04BBD08B593
:100BE80004F000F840B12D2282710022C271202148
:100BF800BDE8084005F006B808BD00BF0B4B984299
:100C080006D0A3F5784398420DD04FF0FF307047D7
:100C18000022074B03EB02135A89013292B25A8120
:100C2800588980B270470122F3E700BF00300140C5
:100C3800345900202DE9F041384EF36882B08046DF
:100C480013B11A689B88138540F2E933344901E0EF
:100C5800002B5ED00A89013B12F0020F9BB2F7D03D
:100C6800304B2F49E8221A7040F2E93301E0002B9B
:100C78004FD00A89013B12F0010F9BB2F7D0294BE4
:100C88001B782749274C6D460DF1060740F2E933DA
:100C980001E0002B38D00A89013B12F0020F9BB209
:100CA800F7D00023237040F2E93300E063B30A89E8
:100CB800013B12F0010F9BB2F8D02078C0B205F8C2
:100CC800010BBD42E2D1F36813B11A689B889361A6
:100CD8009DF804009DF800509DF801109DF8024011
:100CE8009DF803209DF8053041EA052143EA0023D9
:100CF80042EA04220120A8F83810A8F83A20A8F8F7
:100D08003C3002B0BDE8F0810846FFF777FFC0B27B
:100D1800D5E70348FFF772FFB3E700BF481D00207F
:100D2800003001400C3001402DE9F04F8B4D8C4ACA
:100D380028688C4CA5F5EC711C2381F8DE3100F194
:100D480038439B0A0026D25C81F8DF6102F01F0657
:100D580052090123022A85B0E56003FA06F300F080
:100D6800BE81032A00F0C081012A00F0B381B1F8E6
:100D7800DC31029302A940F2013303931FF0F0FC27
:100D8800E368002B00F0B58119689888764A886175
:100D9800138823F040031B041B0C138013889BB299
:100DA80023F0380343F00803138013889BB243F001
:100DB8004003138008856C4940F2E93302E0002BB8
:100DC80000F084810A89013B12F0020F9BB2F6D031
:100DD800664B654924221A7040F2E93302E0002B81
:100DE80000F074810A89013B12F0010F9BB2F6D022
:100DF8005E4B1B785C4940F2E93302E0002B00F0BF
:100E080061810A89013B12F0020F9BB2F6D0574B61
:100E1800554980221A7040F2E93302E0002B00F0B5
:100E280051810A89013B12F0010F9BB2F6D04F4B5A
:100E38001B78E36813B11A689B88936104F040FA41
:100E4800054604F03DFA401B6328FAD9E36813B15C
:100E58001A689B881385444940F2E93302E0002B65
:100E680000F02C810A89013B12F0020F9BB2F6D0E8
:100E78003E4B3D4920221A7040F2E93302E0002B34
:100E880000F01C810A89013B12F0010F9BB2F6D0D9
:100E9800364B1B78344940F2E93302E0002B00F06E
:100EA80009810A89013B12F0020F9BB2F6D02F4B41
:100EB8002D49AF221A7040F2E93302E0002B00F00E
:100EC800F9800A89013B12F0010F9BB2F6D0274B3B
:100ED8001B78E36813B11A689B88936104F0F0F9F2
:100EE800054604F0EDF98542FBD0E36813B11A68B2
:100EF8009B8813851C4940F2E93302E0002B00F07F
:100F0800D5800A89013B12F0020F9BB2F6D0174B2D
:100F1800154923221A7040F2E93302E0002B00F051
:100F2800C5800A89013B12F0010F9BB2F6D00F4B26
:100F38001B780D4940F2E93302E0002B00F0B28043
:100F48000A89013B12F0020F9BB2F6D0074B064903
:100F580060221A7040F2E9330DE000BFEC7C0020FB
:100F6800B85B0308481D0020003001400C300140E8
:100F7800002B00F097800A89013B12F0010F9BB209
:100F8800F6D0664B1B78E36813B11A689B889361A7
:100F98006349644DDFF8A0C1634A644C4FF06408AC
:100FA80010264FF47A70DCF80430C3F30803002BE2
:100FB80058D1EFF31183002B54D10F68D2F808E011
:100FC80000BF0B689F42F8D1D5F8009000FB09F3E9
:100FD800A3EB0E03B3FBF9F300FB073301934FF0C8
:100FE800010EDCF80430C3F30803F3B9EFF31183FF
:100FF800DBB90B68D2F808A000BF0F68BB42F8D174
:10100800D5F800B000FB0BF9A9EB0A09B9FBFBF90D
:1010180000FB0393019FDB1BB3F57A7FE1D3B8F1A3
:101028000108C0D105B0BDE8F08FEFF3118A86F34F
:10103800128897681368DB0344BFC4F800E0976818
:101048000B68D4F800905FFA8AFA8AF31188D5F809
:1010580000A0994400FB0AF3DB1BB3FBFAF300FB87
:101068000933D7E7EFF3118E86F31288D2F8089088
:101078001368DF0303D501232360D2F808900B68B7
:1010880027685FFA8EFE8EF31188D5F800E01F44BA
:1010980000FB0EF3A3EB0903B3FBFEF300FB0733DE
:1010A80001939CE72248FFF7A9FD6CE72048FFF76A
:1010B800A5FD3EE71E48FFF7A1FD0AE71C48FFF71C
:1010C8009DFDE7E61A48FFF799FDB2E61848FFF7D5
:1010D80095FD8FE6174A55692B43536147E6154A34
:1010E80095692B43936142E6124AD5692B43D36134
:1010F8003DE60F4A138823F040031B041B0C1380A2
:1011080013889BB223F0380343F008031380138835
:101118009BB243F0400313804DE600BF0C30014002
:10112800D4560020D856002010E000E0D056002009
:10113800003001400010024000ED00E0F8B584895D
:101148004FF6FF764FF47A742BB311B30F78013151
:1011580001E0B44217D00589013CAD07A4B2F8D527
:1011680007734FF47A7402E0BCB2B4420BD005891D
:10117800ED0704F1FF37F7D5057BEDB20AB115701D
:101188000132013BE0E7FFF739FD003018BF0120CD
:10119800F8BDFF27DFE70120F8BD00BF08B540F222
:1011A800E93300E09BB10289013B12F0020F9BB2C8
:1011B800F8D0017340F2E93300E043B10289013B02
:1011C80012F0010F9BB2F8D0007BC0B208BDFFF748
:1011D80015FDC0B208BD00BF427A02B9704710B50C
:1011E80004460368406804F10A01984700236372C3
:1011F80010BD00BF437A5A1C0344D2B2427299729E
:10120800037A934200D802B9704710B504460368C0
:10121800406804F10A0198470023637210BD00BFBB
:1012280098B10B4B012210B402FA01F103F17504D5
:1012380002E00333A34209D01A788242F9D15A78DE
:101248000A42F6D001205DF8044B70470020FAE707
:10125800A031030810B40023094C01E0272B0AD061
:1012680003EB43020133A15C8142F7D122445DF8CC
:10127800044B9078704700205DF8044B704700BF1E
:10128800A031030870B5448806460D46C4F30B0424
:1012980022460021284631F00FFF3369094A93425C
:1012A80009D3094A934206D2224628461946BDE880
:1012B800704031F0DCBE23B121462846BDE87040BD
:1012C800184770BDEC900308D891030838B5054C51
:1012D800054DAC4200D338BD61682046FFF7D2FF08
:1012E8001434F6E7A08C0308EC900308064B074972
:1012F8008B4202D30023184670471A88C2F30B02A8
:101308009042F8D01433F3E7A08C0308EC9003085C
:10131800024A136823EA000010607047E455002071
:10132800F8B5174D2B78A52B28D16B78BE2B25D176
:10133800022229464FF6FF70FFF75AF8114FAC1CEE
:1013480022884AB1A618BE4218D2052A16D92146C3
:10135800FFF74EF83446F3E721460222FFF748F834
:101368000222A118FFF744F80634074B641B1C80BF
:1013780041F60F53C31A58425841F8BD0020F8BD32
:1013880000F0030800000408285200202DE9F04F5F
:10139800DFF848914C4F8BB00326A7EB09071822BA
:1013A800002104A831F088FE484BCDF8109005972D
:1013B8001A69120604D5464A5A6002F188325A6000
:1013C80001228DF824203422DA60424B424C1B88DB
:1013D800ADF800300222694604A8FFF7CFFB0222CD
:1013E80069464FF6FF70FFF703F8DFF8F4A0804670
:1013F8004FF0000B544536D30AAC002524F8245D81
:101408000222214604A8FFF7B9FB022221464046E2
:10141800FEF7EEFF40BAC043ADF80800022202A969
:1014280004A8FFF7ABFB079860B106ABC0F1040254
:101438002946184431F040FE069904A8FFF745FBF9
:10144800079508909DF82430089A23B11F490B6925
:1014580043F080030B61013E2DD0002A9FD1FFF796
:101468005FFF50B32CE065888DF80DB0C5F30B0510
:10147800AB1DADF808302388C3F30B02ADF80A2082
:101488001B0B062202A904A88DF80C30FFF776FB87
:10149800062202A94046FEF7ABFF616880462A464D
:1014A80004A8FFF76BFB616840462A46FEF7A0FFD9
:1014B800143480469EE7002AD1D0052002F048FB6C
:1014C8000BB0BDE8F08F00BF000004080020024008
:1014D8002301674515320308A08C030800F00308B0
:1014E800EC9003080378202B024600F10100F9D0A4
:1014F800092BF7D02D2B2CD02B2B03BF5378B7EE0D
:10150800000A0246B7EE000AA3F13001C8B2092862
:101518009FED467A10D8F2EE046A07EE901AF8EEBC
:10152800E77A12F8013FE7EE267AA3F13001C8B254
:101538000928B0EE677AF0D92E2B4CD003F0DF03E0
:10154800452B0BD0F7EE007A67EE276A20EE260AC5
:1015580070475378BFEE000A0246D5E710B45178B9
:101568002D2959D02B290ABF9178501C901C002492
:10157800A1F13003092B53D8002303EB830301EBBC
:10158800430310F8011FA1F13002092AA3F1300327
:10159800F3D9B3F59A7F28BF4FF49A73072B42D932
:1015A800DFED236A1A46F7EE007A083A072A67EE53
:1015B800A67AFAD803F007032BB1F2EE046A013BCE
:1015C80067EEA67AFBD124B3C7EE276A5DF8044B11
:1015D80020EE260A70475378A3F13001C8B20928D3
:1015E80002F10102AAD8F2EE046AF0EE665A07EE9A
:1015F800901AF8EEE77A12F8013F87EEA66AA3F18F
:101608003001C8B2092866EEA56A37EE067AEED927
:1016180094E767EE276AD9E7901C91780124A7E739
:10162800F7EE007ACFE7F7EE007AC5E70000000092
:1016380020BCBE4CB5EEC00ADFED317AF1EE10FAEF
:10164800CCBF30EE270A30EE670ADFED2E7A20EEA7
:10165800270A30B5FDEEC07A87B017EE904A0546E6
:1016680084EAE470002303A9A0EBE47001930093DB
:1016780002932DF0C9F9002CACBF20232D2303A819
:101688008DF800302FF082FC012803A924D002280D
:101698002DD0032805BF3023684668468DF80130F1
:1016A80031F012FD68462FF071FC0338C4B22246AF
:1016B8006946284631F03FFD00232B5528462FF078
:1016C80065FC2E22431C2A540DEB0401E81831F066
:1016D80018FD284607B030BD302368468DF8013024
:1016E8008DF802308DF8033031F0EEFCDAE7302364
:1016F80068468DF801308DF8023031F0E5FCD1E70D
:101708006F12033A00007A442DE9F0410646154667
:101718000846B6FBF2F43CB905FB1464124B1B5D9A
:1017280000F8013BBDE8F081B4FBF2F767B90E4B56
:1017380005FB174705FB1464DA5D00F8012B1B5DF8
:1017480000F8013BBDE8F081B7FBF2F8B8F1000FF3
:1017580002D04046FFF7D8FF05FB1878024B13F874
:10176800082000F8012BE3E7C05B03082DE9F047E8
:1017780014461D46064600234FF47A722046294631
:1017880030F0AEF8DFF848814B4A4C4F88FB003107
:101798000144C31782FB002EC3EB611188FB0128AB
:1017A80087FB00278644464AC3EBEE2EC1EB011C9B
:1017B80082FB0E29A0EB8C0C0744424A86F806C02F
:1017C800C3EB27474FEAEE7C08EB010ACCEBA90CE8
:1017D80082FB07824FEAE1780CEB4C0CC8EB6A18E5
:1017E800AEEBCC0EC8EB0818DFF8E8C086F804E0CA
:1017F800A1EB880171718CFB0010F917C1EBE212A3
:1018080040F2B55101FB1272C3EBE050B2F5896F9B
:101818004FEA800740DA40F2DA239A4244DCB2F514
:10182800B77FB4BF4FF0000C4FF0010C4FEA4C08E3
:10183800254B08EB0C0103EBC1031FFA8CFEB3F830
:101848008E00224908EB0C0301EBC30116310B2370
:1018580001E031F8020D82421BDA013BF9D11A4B43
:10186800C44403EBCC0C0123BCF87800B37007F236
:10187800B2770132121ABE44F270A6F800E0204690
:1018880029464FF47A72002330F02AF83281BDE8F5
:10189800F0870133DBB2E9E74FF0030EF44640F27C
:1018A80096504FF00608CCE74FF0020EF44640F28F
:1018B80029404FF00408C4E7C5B3A29107452EC2DA
:1018C800ABAAAA2A73B06D16A03103081832030810
:1018D80089888888792D0311104B2DE93048D3E980
:1018E800004554EA05020BD1034601220020187175
:1018F800587198719A70DA7018801881BDE830882C
:10190800074B1A6814EB020B45F1000C5A46634664
:10191800FFF72CFF0120BDE8308800BFC823002056
:10192800D4560020F0B402888578164FC37804791D
:101938004179A2F2B27202F0030606EB4606013DB7
:1019480005EB860507EB4505013BB5F87860857919
:10195800008940F2B557920807FB0232931903EB4E
:10196800430304EBC303C3EB031301EB8303C3EB90
:10197800031305EB830300214FF47A72C2FB0301C2
:10198800F0BC7047A0310308FAB170B48E18044651
:1019980003E0101A14D1B14214D014F8012BA2F1AB
:1019A8004103192B11F8013BA3F1410598BF2032DF
:1019B800192D03F12000ECD9D01A01D1002BEAD15E
:1019C80070BC7047002070BC70471046704700BF5D
:1019D8004FF0FF32FFF7D8BFA0F16103192B98BF72
:1019E80020387047A0F14103192B98BF2030704769
:1019F800202805D0093804288CBF00200120704712
:101A080001207047613819288CBF002001207047D9
:101A1800413819288CBF0020012070473038092828
:101A28008CBF002001207047A0F13003092B07D993
:101A380020F02000413819288CBF00200120704771
:101A48000120704730B402681146531C036011F836
:101A5800024B0160D31C517803609378151D056013
:101A68001B0443EA0123D078234343EA006030BCD7
:101A7800704700BF0368591C1A46016012F8021B20
:101A88000260587841EA0020704700BF03685A1C7A
:101A980002601878704700BF38B5044600681546DC
:101AA80031F0E5FA22682A44226038BD036810B490
:101AB8000A0A5C1C04601A7003685A1C02601970D8
:101AC8005DF8044B704700BF03685A1C026010B4ED
:101AD800197003680A0A5C1C04601A7003680A0C0F
:101AE8005C1C04601A700368090E5A1C02601970A5
:101AF8005DF8044B704700BF03685A1C02601970F8
:101B08000368090A5A1C0260197070472DE9F047EA
:101B1800002488B080460F461E46A14605AD531CDA
:101B28000393117839B3252933D1931CCDF810903C
:101B38000393507830284ED04FF0000AA0F13003BC
:101B4800DBB2092B42D96C2819D0642800F09380A5
:101B580024D825281CD063D9582876D063281BD1CF
:101B680031784046B847039A531C039311780436DA
:101B780001340029D7D1204608B0BDE8F087039B7F
:101B88005A1C03921B78642B7CD02AD8252B54D15D
:101B9800252140460134B847039AC0E7732833D05B
:101BA80044D975284FD106F1040E30682B4600221F
:101BB8000A217646FEF712FB049A009553463946E9
:101BC8004046FEF749FB039A0444A8E704AA03A980
:101BD8002CF062FEB7E7D31C039390784FF0010A0C
:101BE800ACE7732B10D05BD9752B3AD0782B96D1F4
:101BF800A3F15802B2FA82F2306852092B4610213A
:101C08000436FEF7EBFAD7E73368049A00933946AF
:101C180000234046FEF720FB04360444039A7EE77F
:101C28000028B9D1204608B0BDE8F0876E28B3D1A6
:101C3800039A336804361C6071E72AD9582BD7D029
:101C4800632B8DD06BE77828A6D1A0F15802B2FAA1
:101C580082F2306852092B461021FEF7BFFA04368B
:101C6800AAE706F1040E30682B4600220A217646C0
:101C7800FEF7B4FAA0E7331D306829461E46FEF782
:101C88007FFA99E7331D306829461E46FEF778FA31
:101C980092E7002B7FF443AF204608B0BDE8F087F9
:101CA8006E2BC6D03BE700BF0EB400B584B005ABC1
:101CB800019053F8042B0649039301A8FFF726FF68
:101CC800019B00221A7004B05DF804EB03B0704762
:101CD800550200080FB430B583B006AB0A490B486B
:101CE80053F8042B096800680193FFF70FFF084CAD
:101CF8000546206803F012FD0028FAD0284603B0F4
:101D0800BDE8304004B07047B8290020BC29002045
:101D1800901D0020DFED2B7AB4EEE70AF1EE10FA01
:101D28004ADDDFED296A9FED297A01E0B0EE670A06
:101D3800B4EEC70AF1EE10FA70EE667AF6DC9FEDA3
:101D4800247AF4EEC77AF1EE10FA38D5DFED1E6A80
:101D58009FED207A01E0F0EE407AF4EEC77AF1EEDA
:101D680010FA37EEA60AF6D4DFED1B7AB4EEE70ACE
:101D7800F1EE10FA14DDDFED137A37EEC00A60EEEB
:101D8800006A9FED166A9FED167ADFED167AA6EEC9
:101D9800867A20EE266AE6EE877AA6EE270A70474C
:101DA800DFED117AB4EEE70AF1EE10FA44BFDFED89
:101DB800087A37EEC00AE2E7F0EE407ABFE7B0EE05
:101DC800670AD1E7DB0F4940DB0FC940E4CB164176
:101DD800DB0F49C0E4CB16C1DB0FC93F92E741B91D
:101DE8009730083C15A82ABEDB0FC9BF09B909E01E
:101DF800194690FBF1F301FB13030846002BF7D1BA
:101E0800084670470146FBE707EE901AF8EE677A36
:101E18009FED837A27EE800A20EE070AFDEEC07A4E
:101E280017EE903A2033402B00F28C80DFED7D7A5C
:101E3800B4EEE70AF1EE10FA40F3E880B0EE407A2B
:101E48009FED796ADFED796A01E0B0EE677AB4EE6A
:101E5800E67AF1EE10FA77EE467AF6DC9FED747AC0
:101E6800F4EEC77AF1EE10FA40F1CD809FED6E6A7C
:101E7800DFED706A01E0F0EE477AF4EEE67AF1EE13
:101E880010FA37EE867AF6D4DFED6B7AB4EEE77A9D
:101E9800F1EE10FA51DCDFED697AB4EEE77AF1EE93
:101EA80010FA44BFDFED627A37EEC77A27EE076A89
:101EB800DFED635ADFED637ADFED636A9FED635A06
:101EC800E6EE257A67EE065AE6EE276AF7EE007A1E
:101ED800A5EEA67AF0EE675AE7EE055AE7EE457AE0
:101EE80087EEA55ADFED547A30EE277AFDEEC76A01
:101EF80016EE903A2033402B29D99FED557AF6EE0D
:101F0800006AB7EE006AF7EE004AC4EEA57A00232D
:101F1800836143610362C36180ED045A67EEA66A78
:101F280027EE866A27EE877AC0ED006AC0ED026A5E
:101F380080ED016A80ED037A7047DFED3A7A37EE7B
:101F4800C77AB3E7B7EE005AF0EE455ACAE7B4EEDF
:101F5800E70AF1EE10FA5FDD9FED336ADFED336AD1
:101F680001E0B0EE677AB4EEE67AF1EE10FA77EEB9
:101F7800467AF6DC9FED2E7AF4EEC77AF1EE10FA87
:101F880047D59FED296ADFED2B6A01E0F0EE477A2D
:101F9800F4EEE67AF1EE10FA37EE867AF6D4DFED53
:101FA800267AB4EEE77AF1EE10FA27DCDFED237A31
:101FB800B4EEE77AF1EE10FA44BFDFED1D7A37EEA2
:101FC800C77A27EE076ADFED1E4ADFED1E6ADFEDEE
:101FD8001E7AE6EE246A67EE064AE6EE267AB7EE41
:101FE800006AA4EEA77AF6EE006A36EE476AF8EEC3
:101FF800007A27EE277A66EE266A84E7DFED097A0B
:1020080037EEC77ADDE7B0EE677A3DE7F0EE407A63
:1020180024E7B0EE677AC2E7F0EE477AAAE700BF96
:1020280027D4D236DB0F4940DB0FC940E4CB164139
:10203800DB0F49C0E4CB16C1DB0FC93FDB0FC9BFBB
:1020480092E741B99730083C15A82ABEF304353FFA
:102058000000008070B406688E4217D90139751ED9
:10206800002311F8014F0822634013F0800F4FEA54
:10207800430318BF83F0D503013ADBB2F5D18D4293
:10208800EFD1721C0260337070BC70470023F8E710
:1020980010B44C09012250F8243001F01F0102FA53
:1020A80001F10B4340F824305DF8044B704700BF42
:1020B8004B0901F01F0150F82320012303FA01F115
:1020C800114214BF18460020704700BFB0F1FF3F0F
:1020D8000AD0022810B403DC5DF8044BFEF7CCBA32
:1020E80000205DF8044B7047002070470378012BEF
:1020F80043D0022B3FD170B5836801F07F0113B143
:102108001C689B88238505461646406840F2E934DA
:1021180001E0002C37D00389013C13F0020FA4B270
:10212800F7D0017340F2E93100E061B30389013966
:1021380013F0010F89B2F8D0037B686840F2E931E7
:1021480000E019B30489013914F0020F89B2F8D0FC
:10215800067340F2E93300E0C3B10289013B12F093
:10216800010F9BB2F8D0037BAB6893B11A689B88C8
:102178009361012070BD0020704713460A464179DB
:1021880090F90400A2E7FEF739FDD6E7FEF736FD21
:10219800EAE7012070BD01224821A7E70122582162
:1021A800A4E700BF2DE9F04F037C012B83B08146E3
:1021B80000F09683022B44D1836913B11A689B8877
:1021C8001385D9F8140040F2E93302E0002B00F03F
:1021D800C1830289013B12F0020F9BB2F6D06B2338
:1021E800037340F2E93302E0002B00F0B383028965
:1021F800013B12F0010F9BB2F6D0037BD9F8140013
:1022080040F2E93302E0002B00F0A1830289013B90
:1022180012F0020F9BB2F6D08023037340F2E93329
:1022280002E0002B00F093830289013B12F0010FBA
:102238009BB2F6D0037BD9F8183013B11A689B8883
:1022480093616423B74CB84DDFF8E4A2B748DFF8D0
:10225800E4C2CDF804904FF010084FF47A7799460D
:10226800DAF80430C3F30803002B40F00E82EFF3D2
:102278001183002B40F009822668826800BF23681A
:102288009E42F9D1296807FB01F39B1AB3FBF1F3CE
:1022980007FB06364FF0010E0096DAF80430C3F358
:1022A8000803002B40F0D681EFF31183002B40F098
:1022B800D1812368816800BF22689342F9D1D5F89B
:1022C80000B007FB0BF2521AB2FBFBF207FB032329
:1022D800009A9B1AB3F57A7FDFD3B9F10109BFD110
:1022E800DDF8049099F81030012B53D0022B5BD104
:1022F800D9F8183013B11A689B881385D9F81400D7
:1023080040F2E93302E0002B00F039830289013BF7
:1023180012F0020F9BB2F6D06B23037340F2E9333D
:1023280002E0002B00F02B830289013B12F0010F21
:102338009BB2F6D0037BD9F8140040F2E93302E0EF
:10234800002B00F00A830289013B12F0020F9BB2B6
:10235800F6D00323037340F2E93302E0002B00F0C8
:10236800FC820289013B12F0010F9BB2F6D0D9F82A
:102378001820037B002A00F0F782136892889A617C
:1023880099F8100099F85010012800F09A81022855
:1023980056D115E003236B2299F8151099F914000A
:1023A800FFF794FE99F8103099F85010012B00F0BF
:1023B8008881022B44D1D9F8182012B11368928869
:1023C8001A85D9F8140040F2E93202E0002A00F038
:1023D8008F820389013A13F0020F92B2F6D01923C3
:1023E800037340F2E93202E0002A00F08182038997
:1023F800013A13F0010F92B2F6D0037BD9F814001A
:1024080040F2E93202E0002A00F0CE820389013A64
:1024180013F0020F92B2F6D0017340F2E93302E0F2
:10242800002B00F0C1820289013B12F0010F9BB220
:10243800F6D0037BD9F8183013B11A689B889361DA
:102448000F23DFF8ECA03948DFF8E8C0CDF8049096
:102458004FF010084FF47A779946DAF80430C3F34E
:102468000803002B40F01582EFF31183002B40F096
:1024780010822668826800BF23689E42F9D12968C5
:1024880007FB01F39B1AB3FBF1F307FB06364FF08A
:10249800010E0096DAF80430C3F30803002B40F06D
:1024A800DD81EFF31183002B40F0D8812368816828
:1024B80000BF22689342F9D1D5F800B007FB0BF2B0
:1024C800521AB2FBFBF207FB0323009A9B1AB3F5DF
:1024D8007A7FDFD3B9F10109BFD1DDF8049099F80B
:1024E800102099F84E10012A00F04E81022A40F07F
:1024F8005581D9F8183013B11A689B881385D9F813
:10250800140040F2E93202E0002A00F04A8203890E
:10251800013A13F0020F92B2F6D01A23037340F275
:10252800E9320CE0D4560020D856002010E000E034
:1025380000ED00E0D0560020002A00F03282038926
:10254800013A13F0010F92B2F6D0037BD9F81400C8
:1025580040F2E93202E0002A00F014820389013ACD
:1025680013F0020F92B2F6D0017340F2E93302E0A1
:10257800002B00F007820289013B12F0010F9BB289
:10258800F6D0D9F81820037B002A00F002821368DD
:102598009188996199F81020012A00F09681022A01
:1025A80000F00781012A00F09580022A40F09C8003
:1025B800D9F8182012B1136891881985D9F8140030
:1025C80040F2E93302E0002B00F0BE810289013BB2
:1025D80012F0020F9BB2F6D01C23037340F2E933CA
:1025E80002E0002B00F0B0810289013B12F0010FDC
:1025F8009BB2F6D0037BD9F8140040F2E93302E02D
:10260800002B00F090810289013B12F0020F9BB26F
:10261800F6D01823037340F2E93302E0002B00F0F0
:1026280082810289013B12F0010F9BB2F6D0D9F8E2
:102638001820037B002A00F07D81136892889A6134
:1026480099F81010012900F0FF80022956D003B034
:10265800BDE8F08FEFF3118188F31288866803686C
:10266800DB0344BFCCF800E086682368DCF8002070
:10267800C9B281F3118829681A4407FB01F39B1B2F
:10268800B3FBF1F307FB023322E6EFF3118288F381
:10269800128881680368DE0303D50123CCF8003073
:1026A80081682368DCF80060D2B282F311882A6856
:1026B8001E4407FB02F35B1AB3FBF2F307FB063673
:1026C800E8E50B46192299F8151099F91400FFF757
:1026D800FDFCB5E61C22182399F8151099F9140089
:1026E800FFF7F4FC99F81020012A00F0AD80022AC7
:1026F800ADD1D9F8182012B1136892881A85D9F883
:10270800140040F2E93302E0002B00F0098102894D
:10271800013B12F0020F9BB2F6D03723037340F24D
:10272800E93302E0002B00F0FB800289013B12F044
:10273800010F9BB2F6D0037BD9F8140040F2E933BD
:1027480002E0002B00F0E9800289013B12F0020F41
:102758009BB2F6D00223037340F2E93302E0002B68
:1027680000F0DB800289013B12F0010F9BB2F6D02A
:10277800037BD9F81830002B3FF469AF1A689B889F
:10278800936103B0BDE8F08F0B461A2299F8151033
:1027980099F91400FFF79AFC99F81020012A00F023
:1027A8009480022A7FF4FEAED9F8182012B113687B
:1027B80091881985D9F8140040F2E93302E0002B1A
:1027C80000F0A8800289013B12F0020F9BB2F6D0FC
:1027D8001B23037340F2E93302E0002B00F09A80D8
:1027E8000289013B12F0010F9BB2F6D0037BD9F8A6
:1027F800140040F2E93301E0002B7CD00289013B50
:1028080012F0020F9BB2F7D01823037340F2E9339A
:1028180001E0002B6FD00289013B12F0010F9BB23F
:10282800F7D0D9F81820037B002A6AD0136891885A
:10283800996199F81020012A3FF44CAF022A3FF41D
:10284800BCAE012A7FF453AF99F8151099F914001A
:102858000223372203B0BDE8F04F37E4EFF31181CC
:1028680088F3128886680368DB0344BFCCF800E06D
:1028780086682368DCF80020C9B281F311882968CA
:102888001A4407FB01F39B1BB3FBF1F307FB02336D
:102898001BE6EFF3118288F3128881680368DE0370
:1028A80003D50123CCF8003081682368DCF8006088
:1028B800D2B282F311882A681E4407FB02F35B1A1E
:1028C800B3FBF2F307FB0636E1E51B22182399F860
:1028D800151099F91400FFF7F9FB99F8102061E633
:1028E800417D90F9140080236B22FFF7EFFBA8E4E9
:1028F800FEF784F982E5FEF781F9D9F81820002A55
:1029080094D199F81020012A3FF4E4AE022A3FF44A
:1029180055AEE9E6FEF772F969E7FEF76FF928E7C1
:10292800FEF76CF908E7FEF769F9D9F81820002ACC
:102938007FF483AE99F81030012B85D0022B3FF439
:10294800DEAE03B0BDE8F08FFEF758F953E6FEF7A8
:1029580055F970E4FEF752F950E4FEF74FF9D9F84B
:102968001820002A7FF409AD99F8103099F8501012
:10297800012B3FF4A6AE022B3FF423AD60E5FEF732
:102988003DF9D8E4FEF73AF9D9F81820002A7FF47F
:10299800FEAD99F81020012A97D0022A3FF40AAF19
:1029A80000E6FEF72BF9D1E5FEF728F942E500BF6E
:1029B800F0B55B4B5B4A97B01968914200AF00F0E5
:1029C800A3805949594A00234FF47000C1F8880080
:1029D8003B607B60136843F48033136003E03B681B
:1029E800B3F5A04F09D0136803F400337B603B684C
:1029F80001333B607B68002BF1D04C4B1B6813F410
:102A0800003318BF01237B607B68012B52D0464CF2
:102A1800464B474AE260474A596A11605A6A42F08F
:102A280080725A625A6942F4FC025A6100250322F4
:102A380007F10801012341F6FF764FF09040FD6051
:102A4800BE603A73BB731DF08BFE4FF6FF7307F140
:102A580008013948BB601DF083FE07F108013748BB
:102A6800374E1DF07DFE07F1080136481DF078FE4F
:102A780007F1080134481DF073FE07F108013348D7
:102A88001DF06EFE07F108001DF0C4FEBB6830495A
:102A9800304AA1FB031330499B0CF0204FF0070E7E
:102AA8005C370B60566084F823009560C2F800E03C
:102AB800BD46F0BD294A1D4B122111605A685A6063
:102AC8005A685A605A6842F480625A605A6822F416
:102AD8007C125A605A6842F4E8125A601A6842F046
:102AE80080721A601A689201FCD559680F4A21F061
:102AF80003015960596841F002015960536803F0B5
:102B08000C03082BFAD182E700221A6062B6144B34
:102B18001B6883F30888134B1B689847FEE700BFC0
:102B2800FC9F0020EFBEADDE00ED00E0001002408B
:102B38000005FA057C5900200004004800080048F8
:102B48003F190100000C004800100048001400481C
:102B580083DE1B4310E000E0D8560020002002402E
:102B680000D8FF1F04D8FF1F064A0023516881427E
:102B780002F11C0204D001330C2BF7D1002070475E
:102B8800D8B27047141A0020074BC0EBC00030B40D
:102B980003EB8000054C056963692B43636101768B
:102BA800427630BC704700BF141A00200010024063
:102BB8002DE9F04F634C54F8204083B0002C7CD0B2
:102BC800A56D1F466B682365A1604FF4807304F1FF
:102BD8005E019046064604F5AF725B48206061616D
:102BE800A261E3602361287E29F008FFE86858B1F4
:102BF800FFF7BAFF721CD2B20C21FFF7C5FF236D95
:102C0800EA6862632433E364A86870B3FFF7ACFF33
:102C1800721CD2B20B218146FFF7B6FF4B48DFF892
:102C280030E1EB7EDEF81410C9EBC90900EB89002E
:102C38009B0902690A43CEF81420DFF818E1417BAA
:102C4800446100228DF80530C0F808E0012301A88E
:102C58008DF806208DF807308DF804101DF04AFD18
:102C6800236DAA68A2632833A36494F85D0001F079
:102C7800B9FF814694F85C0001F0B4FF3A07824638
:102C880095F819B01DD5B9F1000F1AD017F0110F2A
:102C98004FF00B0306F1010614BF4E213E2189F8BF
:102CA800063089F807605A46484601F0FBFBFB07E7
:102CB80043D5636B6BB3A36B5BB3204603B0BDE82E
:102CC800F08F17F0010F0CBF2E274E2718F0020FB8
:102CD8000DD0B9F1000F0AD00B22731C89F8062019
:102CE80089F8073048465A46394601F0DBFB18F0A8
:102CF800010FDED0BAF1000FDBD001360C238AF8C1
:102D080007605A4639468AF80630504601F0CAFB31
:102D1800CFE7AB7E8DF804302B7F00219B09012281
:102D280001A88DF805308DF806108DF807201DF0E4
:102D3800E1FC204603B0BDE8F08F484603F01EF9D9
:102D4800B7E700BFC429002078320308141A00200E
:102D580000100240C50B00080348D0F83C3113B1FD
:102D680000F59A7018477047141A00200348D0F8E5
:102D7800203113B100F58C7018477047141A0020E1
:102D88000348D0F804310BB1FC301847704700BF36
:102D9800141A00200348D0F8E8300BB1E030184787
:102DA800704700BF141A00200348D0F8CC300BB18C
:102DB800C4301847704700BF141A00200348D0F8E1
:102DC800B0300BB1A8301847704700BF141A002064
:102DD8000348D0F894300BB18C301847704700BFC7
:102DE800141A00200248836F0BB1703018477047DF
:102DF800141A00200248C36D0BB1543018477047AD
:102E0800141A00200248036C0BB138301847704779
:102E1800141A00200248436A0BB11C301847704747
:102E2800141A00200248836803B11847704700BF8E
:102E3800141A0020F8B505015A4C5B4B6259611908
:102E48009A4204EB050704BF01230B730646387A40
:102E580029F0D4FD3B7A03F01F015B090122022B04
:102E680002FA01F278D0032B71D0012B67D06319D5
:102E78000136187901F0B6FEF6B2074610B11223F2
:102E8800C67183716319587901F0ACFE10B1132330
:102E9800C67183716319987901F0A4FE10B11423E7
:102EA800C671837166190E21F279384601F0FAFA73
:102EB800707901F097FEF2790E2101F0F3FAB079FA
:102EC80001F090FEF2790E2101F0ECFA6359374ACD
:102ED800934251D0344A934259D0354A934240D014
:102EE8002C44227B002A2FD1012002249A8822F424
:102EF80080521204120C9A80998889B241F4805148
:102F080099801A8802F4415242F4457202432243DE
:102F18001A809A8822F470621204120C42F4E06259
:102F28009A809A8B22F400621204120C07219A8369
:102F380019821A8892B242F040021A80F8BD1D4BDD
:102F4800996A0A439A6292E700200446CEE7194B31
:102F580019690A431A618AE7164BD9680A43DA6085
:102F680085E702F5EA32116941F4004111611169FE
:102F780021F400411161B3E702F56042D16841F4E0
:102F88008051D160D16821F48051D160A8E702F561
:102F9800EC32116941F480411161116921F48041D9
:102FA80011619DE73459002000380040003001408D
:102FB800003C004000100240F0B53E4C059D00EB7F
:102FC800800004EB80046468002C71D03A4E4900FC
:102FD8004FF42040CFB2B060A169090454D46068AE
:102FE800DFF8E0E047F4903100EA0E0001434FF4C7
:102FF80020406160B06003E0411E002848D00846C8
:10300800A1698907F8D54FF42040A262B06003E0B7
:10301800421E00283CD01046A2695206F8D5274A1D
:103028006168DFF8A0E0B06042EA0342174301EAB2
:103038000E0217436760C3B1013BDBB201332B4477
:10304800A0694FF4204210F0040002F1FF3207D1CA
:10305800511C26D0A06910F0040002F1FF32F7D00D
:10306800626A05F8012B9D42EAD14FF42040B06016
:1030780002E0431E60B11846A3699B06F9D52023D8
:10308800B060E3610120F0BD411E08B10846A3E726
:103098000B4A138801339BB24FF0FF311380B160A4
:1030A800F0BD0749B2600B8801339BB20B80F0BDBD
:1030B8002046F0BD74560020481D00200024000260
:1030C80026520020009800FCF0B50E460178012930
:1030D80085B004464BD002294FD11D46836846F07F
:1030E800800113B118689B880385606840F2E93352
:1030F80001E0002B55D00689013B16F0020F9BB268
:10310800F7D0017340F2E93301E0002B49D001897F
:10311800013B11F0010F9BB2F7D0037B60684FF0C1
:10312800000C83894FF6FF764FF47A734FF0FF0E49
:10313800654502D126E0B34222D00189013B8F07C1
:103148009BB2F8D580F80CE04FF47A7302E0BBB27A
:10315800B34215D00189C90703F1FF37F7D5017BC1
:10316800C9B20AB1117001320CF1010CE0E790F913
:103178000400411C01D002280CDD002005B0F0BD80
:10318800FDF73CFDA3688BB11A689B889361012009
:1031980005B0F0BD617900923246FFF70DFF05B02A
:1031A800F0BD0392FDF72AFD039AB7E70120E5E792
:1031B800F0B500F10C0585B004460F4601230DF16A
:1031C800070202212846FFF77FFF18B9002630467C
:1031D80005B0F0BD9DF80730DB07F7D502AA03213B
:1031E80028462CF027F901230DF10702092128466A
:1031F800FFF76AFF06460028E8D011220A21284670
:10320800FEF774FF9DF8073013F00C0FDED1B4F908
:103218001A1002A8FDF705F940423880B4F91C10CD
:103228000DF10A00FDF7FDF840427880B4F91E1050
:1032380003A8FDF7F6F84042B880C8E737B500F1B3
:103248000C04054600220A212046FEF74FFF1420F1
:1032580002F0DCF80F220A212046FEF747FF0A2079
:1032680002F0D4F801AA032310212046FFF72CFF0F
:103278000A2002F0CBF89DF8043080336B839DF868
:1032880005308033AB839DF806308033EB83002212
:103298000A212046FEF72AFF0A2002F0B7F80DF1AE
:1032A8000302012302212046FFF70EFF01230DF13F
:1032B800030209212046FFF707FF11220A212046B1
:1032C800FEF714FF012003B030BD07B5032301AAA0
:1032D8000021FFF7F9FE9DF805309DF804001B0258
:1032E80043EA00439DF80600184303B05DF804FB69
:1032F80008B5FFF7EAFF014B586008BD481D0020DC
:1033080008B5FFF7E2FF014B186008BD481D002013
:10331800F0B5037C012B85B0044663D0022B67D13E
:10332800836913B11A689B881385606940F2E93391
:1033380001E0002B6CD00289013B12F0020F9BB216
:10334800F7D0C323037340F2E93301E0002B5FD0C9
:103358000289013B12F0010F9BB2F7D0037B606931
:103368004FF0060E838902AE4FF47A734FF6FF7161
:10337800FF2703E0013B9BB28B423CD002899507B3
:10338800F8D507734FF47A7302E0ABB28B4232D0B0
:103398000289D20703F1FF35F7D5027BD2B20EB10D
:1033A80032700136BEF1010EE8D1A36913B11A6873
:1033B8009B8893619DF80C009DF808609DF80910A2
:1033C8009DF80A509DF80B209DF80D3041EA062122
:1033D80043EA002342EA0522012021876287A38766
:1033E80005B0F0BD90F91400431C01D0022805DD9A
:1033F800002005B0F0BDFDF701FCD6E702AB617D0A
:10340800009343220623FFF7D7FD0028D2D1EFE728
:10341800FDF7F4FBA3E700BFF0B5037A012B85B0F5
:10342800044663D0022B67D1036913B11A689B88DD
:103438001385E06840F2E93301E0002B6CD0028983
:10344800013B12F0020F9BB2F7D0BB23037340F28B
:10345800E93301E0002B5FD00289013B12F0010F34
:103468009BB2F7D0037BE0684FF0060E838902AE6B
:103478004FF47A734FF6FF71FF2703E0013B9BB2CD
:103488008B423CD002899507F8D507734FF47A73BD
:1034980002E0ABB28B4232D00289D20703F1FF358A
:1034A800F7D5027BD2B20EB132700136BEF1010EF1
:1034B800E8D1236913B11A689B8893619DF80C00C1
:1034C8009DF808609DF809109DF80A509DF80B209A
:1034D8009DF80D3041EA062143EA002342EA05221D
:1034E8000120E1822283638305B0F0BD90F90C00CE
:1034F800431C01D0022805DD002005B0F0BDFDF712
:103508007DFBD6E702AB617B00933B220623FFF7E6
:1035180053FD0028D2D1EFE7FDF770FBA3E700BF0A
:10352800F0B585B002AB04460093A8220623192102
:103538000020FFF741FD00B39DF809709DF80810C1
:103548009DF80B609DF80A209DF80D509DF80C30F1
:1035580041EA072142EA062243EA052309B212B2E8
:103568001BB201EBD17102EBD27203EBD37349109A
:1035780052105B10E1822283638305B0F0BD00BF67
:103588001749184B184A194810B4D1F8884044F420
:103598007004C1F888401C6844F001041C605C6831
:1035A80022405A601A6822F0847222F480321A602B
:1035B8001A6822F480221A605A6822F4FE025A60BD
:1035C800DA6A22F00F02DA621A6B002410404FF018
:1035D800006218639C608A605DF8044B704700BF06
:1035E80000ED00E0001002400CC07FF8CCFC00FFAA
:1035F80038B50B4C23688BB15A68821A002A0546E5
:1036080004DA0CE05A68AA1A002A07DB9A682260D2
:1036180018461A6890472368002BF3D138BD38BD87
:10362800FC3800200B4B002210B4027203F5AA7478
:10363800042102E0072A09DC9979890702D519795A
:10364800815401329C4203F11403F3D15DF8044B19
:10365800704700BF3C5A030810B40D4C04232146A0
:10366800002200E08B7913F0010301F1140106D167
:103678000132122AF6D103705DF8044B704702EB51
:10368800820204EB82025DF8044B137903707047E1
:103698003C5A030830B40123302533243121322227
:1036A8004570C4714171C2700372037083710371F4
:1036B800837030BC704700BF436A8269D154436A43
:1036C8000169826B01338B4228BF00234362002AC1
:1036D8002FD0EFF31181502383F31288836B1A687C
:1036E800D2072CD470B45E686EB9456A826A954276
:1036F80017D084691444DC600ED9AA1A5A6085620E
:10370800002280F854201A6842F00102C9B21A60F7
:1037180081F3118870BC70470469A21A5A608662E6
:10372800EEE7012380F85430C9B281F3118870BCE8
:103738007047026D136843F0800313607047C9B285
:1037480081F31188704700BF426B10B462B1436CBB
:10375800C2684469D11A013B615C5DF8044B08BF3B
:1037680013464364C8B27047016A4369C4685B5C26
:103778000131A14228BF114601625DF8044BD8B25D
:10378800704700BF836B13B190F854007047836A89
:10379800406A181AB0FA80F040097047416A836A93
:1037A80099420AD3CB1A816B026961B14968501EEC
:1037B8000B4483420AD2C01A704702691144CB1ADB
:1037C800816B0029F2D1501EC01A70470020704743
:1037D800436B43B1426C5B6893422FBF981AC06831
:1037E8009B1AC0187047C269036A9A422FBFD01A41
:1037F800C0688018C01A70470A4B30B503F110042E
:1038080093F900205D78072AC8BF143A8118043359
:103818000D7313F8025C855413F8012C0A76A34241
:10382800EED130BDA032030803682DE9F041DF690D
:103838001FB13B46BDE8F0411847002A164611DD86
:1038480004460D460E4400E023689B6820469847CE
:103858000028F9D0236815F8011B1B6820469847F3
:10386800AE42F1D1BDE8F08110B45A2158240022AB
:103878000323047041708270C3705DF8044B704775
:10388800152303701623C370172383712D234370E8
:103898002E2303712F23C371704700BF2DE9F04712
:1038A8000569C3681D4028D00F4606464FF00048FA
:1038B8004FF00009B5FA85F328FA03F2D2431B3B0F
:1038C80032611540042B16D8DFE803F0312921199D
:1038D80003007B6A002B32D003F1FF3A1FFA8AFA01
:1038E800C7F824903C6A34B123682046514698476B
:1038F8006468002CF8D1002DDCD1BDE8F087386869
:10390800716B036889B29847002DD3D1F5E77868C1
:10391800B16B036889B29847002DCBD1EDE7B86841
:10392800F16B036889B29847002DC3D1E5E7F868C1
:10393800316C036889B29847002DBBD1DDE7F36A83
:103948001FFA83FACEE700BF30B50446006D6171F7
:103958000368A26823F00103036087B0A37900928B
:1039680013F004023DD04FF4805213F00203019289
:1039780044D102934FF480630022039311F00103B2
:10398800059237D1049308238D07694648BF0493ED
:103998001DF030F96079236DA17900F00202002A48
:1039A80015BF4FF440324FF480324FF400340024F6
:1039B80010F0010F586808BF2246CC074CBF0243DD
:1039C80020EA02025A609A6809074CBF42F00802CE
:1039D80022F008029A601A6842F001021A6007B0E1
:1039E80030BD13F0020301920BD04FF4005513467B
:1039F8000295C1E7042304930C23C5E74FF4005351
:103A0800B7E70293B8E700BF10B50446006DA160A0
:103A1800036823F001030360A37986B013F004025E
:103A2800009141D04FF4805213F00203019244D127
:103A380002934FF4806362790393D1074FF0000338
:103A48000493059345BF0423049308230C23694674
:103A5800920748BF04931DF0CDF86079236DA179D2
:103A680000F00202002A15BF4FF440324FF48032B2
:103A78004FF40034002410F0010F586808BF2246A4
:103A8800CC074CBF024320EA02025A609A68090731
:103A98004CBF42F0080222F008029A601A6842F00D
:103AA80001021A6006B010BD13F00203019207D09C
:103AB8004FF4005113460291BDE74FF40053B7E7A6
:103AC8000293B8E7022828BF022010B4084C094B1B
:103AD800207000EB8002C0EBC20207495DF8044B7E
:103AE800013003EB4203C0B20B6022F013BF00BFEA
:103AF800283E0020862D00206034002010B5FDF7F8
:103B0800E5FB094A094B0A490A4C0B481460002294
:103B18001A705A7008601BF021FAFDF737FCBDE8EF
:103B280010401BF003BA00BF60340020283E00207C
:103B380064340020862D0020343E002008B51BF098
:103B48000DFAFDF723FCBDE808401BF0EFB900BFF4
:103B58002DE9F04F013085B0C3B203938E4D8F4FDE
:103B68008F4C904E0A2302933220DFF8409229F0BE
:103B7800E7FA4FF4FA7A4FF0100C4FF47A70D9F84C
:103B88000430C3F30803002B40F0C880EFF311831F
:103B9800002B40F0C3802968A26800BF2B689942B7
:103BA800F9D1D7F800E000FB0EF39B1AB3FBFEF344
:103BB80000FB01314FF0010E0191D9F80430C3F335
:103BC8000803002B40F08E80EFF31183002B40F0A8
:103BD80089802B68A16800BF2A689342F9D1D7F879
:103BE80000B000FB0BF2521AB2FBFBF200FB0323FE
:103BF800019A9B1AB3F57A7FDFD3BAF1010ABED1D5
:103C0800039B002B40F0C4804FF47A7ADFF89C9134
:103C180050464FF0100CD9F80430C3F30803002BBA
:103C280040F09980EFF31183002B40F094802968CD
:103C3800A26800BF2B689942F9D1D7F800E000FBD1
:103C48000EF39B1AB3FBFEF300FB01314FF0010E9C
:103C58000191D9F80430C3F308033BBBEFF3118398
:103C680023BB2B68A16800BF2A689342F9D1D7F813
:103C780000B000FB0BF2521AB2FBFBF200FB03236D
:103C8800019A9B1AB3F57A7FE3D3BAF1010AC2D13C
:103C9800029B013B02937FF467AF4349434B44487F
:103CA800444A0860DA6005B0BDE8F08FEFF3118888
:103CB8008CF31288A1682368DB0344BFC6F800E0D0
:103CC800A1682B6832685FFA88F888F31188D7F8FA
:103CD80000801A4400FB08F35B1AB3FBF8F300FBFF
:103CE8000233CDE7EFF311888CF31288A1682368BB
:103CF800DB0344BFC6F800E0A1682B6832685FFAAE
:103D080088F888F31188D7F800801A4400FB08F374
:103D18005B1AB3FBF8F300FB023369E7EFF3118298
:103D28008CF31288D4F808E02368D90303D501235B
:103D38003360D4F808E02B683168D2B282F3118876
:103D48003A68194400FB02F3A3EB0E03B3FBF2F34A
:103D580000FB01312EE7EFF311828CF31288D4F8BF
:103D680008E02368D90303D501233360D4F808E0B9
:103D78002B683168D2B282F311883A68194400FB83
:103D880002F3A3EB0E03B3FBF2F300FB01315DE793
:103D9800184629F045F837E7D4560020D8560020B1
:103DA80010E000E0D0560020FC9F002000ED00E06D
:103DB800EFBEADDE0400FA0538B5434B5A89998940
:103DC800914224BF00225A81198ADA89914224BF7C
:103DD8000022DA81DA788AB3072A2FD03B493C4D92
:103DE80091F85300012400210A282C709C70D97185
:103DF8003DD00C2865D0DFED377A8ABB364C9FED75
:103E0800370AA278002918BFF0EE407A062A04D8AB
:103E1800334901EB820191ED040A217959B3013A42
:103E2800032A4DD8F7EE007A87EE800A2EF07EF945
:103E38002388984228BF1846208038BDD97921B1F7
:103E480098780428B8BF04209870204890F8530048
:103E58000A280CD00C28CED1DFED227A002ACDD04A
:103E6800072ACBD00A282CD1DFED1F7AC6E70A2013
:103E7800DFED1E7AC1E79B78154A07EE103A1178F4
:103E8800B8EEC77A27EE277A07EE901AF8EEE77AA7
:103E980067EE877AB4EEE70AF1EE10FA10DDC0EEAD
:103EA800077AFDEEE77A17EE903A102BA8BF102399
:103EB800012BB8BF0123DBB28B4238BF0B4613700E
:103EC80038BDDFED0B7A99E77C4900209049002046
:103ED800B45500206F120339184E00206F120338B2
:103EE800A03203080AD7A3390F506E3A5304E938B1
:103EF8006F12833A2DE9F047AC4FAD4E1BF02EF808
:103F0800BE421ED2DFF82483DFF824934446258876
:103F180062197DB14A450DD2052D0BD933886188C8
:103F2800C3F30B03994200F0E68014462588621912
:103F3800002DEFD1716830461436FDF7A3F9BE4263
:103F4800E4D39C4A1378A3F1170102290FD99A499F
:103F580011F83300002840F0FA80D800014449786D
:103F680029B1964911F83330002B00F01881944B91
:103F78005A78022A40F2E580002292495A701A784B
:103F88009148022A016000F2D88002EB82018F4B2F
:103F9800C2EBC10203EB4203998C5A8C8C4C9142C0
:103FA800236001D300225A848A4B9A78042A00F0AD
:103FB800ED8032B91A88B2F5F07F84BF4FF4F07201
:103FC8001A80854DFFF7F8FE2B68844A1A40002AAC
:103FD80000F0E880D80700F1D480590400F1CC80C3
:103FE8001A0700F1C4809B0400F1BA802BF0C4FFCB
:103FF80010B97B4821F02AFE8020FDF789F94FF49B
:104008000070FDF785F94FF48030FDF781F94FF422
:104018008020FDF77DF94FF40010FDF779F94FF096
:104028000070FDF775F94FF08060FDF771F94FF0FA
:104038000060FDF76DF919F0C5FD002130226948CF
:104048002FF03AF8206818F0CDFC674B276803F189
:10405800500102E0043399426DD01A78002AF9D150
:104068009C78D8788442F5D26049614B0D796149D2
:1040780061480A70614E624C0460C822642111FBD9
:104088000521002259609A60DA601A615A619A61C2
:10409800DA6183F8202083F82120376021F0FAFBC9
:1040A800584B9FED595A1B88584A9FED596A5079C9
:1040B800584906EE903AF8EEE66A1388C5EE265A95
:1040C80007EE103A53881279C1ED005A07EE903A7C
:1040D800B8EEC77A504BF8EEE77A18725A7227EEA4
:1040E800067A67EE867ABDE8F04783ED017AC3ED7C
:1040F800007A1AF01BBF63799B077FF416AF7168CB
:1041080094F804A03046FDF7BDF83388BAEB133FA6
:1041180004D01436BE42FFF4F9AE12E77388706813
:10412800AA1FC3F30B039A4204F10601A8BF1A465B
:104138002EF09DFFEDE7012296E700221A70234B2F
:104148002AE7204902EB420201EB820117E7D80077
:104158000C186468002C7FF401AF17241470FDE676
:104168002E48FDF7D5F84020FDF7D2F83EE72C4859
:10417800FDF7CEF82B6836E72A48FDF7C9F82B6813
:104188002EE72948FDF7C4F82B6826E79A8AB2F586
:104198007A7FBFF416AF4FF47A729A8211E7182328
:1041A8001370E4E643F400532B6013E7EC90030824
:1041B800A08C0308105900202C570308B4350308B5
:1041C800283E0020343E002064340020862D002044
:1041D80060340020184E0020E455002009600002D9
:1041E800147A00207C1E002060390020F43600205C
:1041F800783E0020681B0020C01E0020B01E002052
:10420800C655002090200020C0C9FB48C0230020CC
:1042180017B7D13894200020F43400200940000258
:1042280001600002092000020860000202F0030891
:104238000000040808B51AF091FEFDF7A7F81AF077
:1042480075FEFFF757FE0120BDE8084022F062BB6B
:104258002DE9F84F4FF4A07200218248824C834D1B
:10426800834E844FDFF82882DFF828922EF024FF4F
:1042780081488249DFF820E2DFF820C20022135982
:10428800834200F0C380B3F1804F00F0D580AB4289
:1042980000F0D980B34200F0D880BB4200F0D7804C
:1042A800734500F0D680634500F0A680434500F0D2
:1042B800D2804B4500F0D280DFF8E4A1534508BF17
:1042C8004FF4802300F09A801432B2F5B47FD6D12F
:1042D800654D6B4F6B4E05F5B4784FF0030A4FF000
:1042E800020903E01435A84500F08E80AB79002B55
:1042F800F8D02B791C09013C052C03F00F03F1D8E9
:1043080037F8140040FA03F2D207EBD54FF0010B4F
:104318000BFA03F3013B18402DF032FB5A4B1B5D9F
:10432800184416EBC004DDD056F830305748297AC7
:1043380003F13842920A825C02F01F005209022AF5
:104348000BFA00FB71D0032A68D0012A05D14B4A29
:104358004A4852694BEA02024261B4F804E0BEFAE4
:104368008EF2C2F11F0292B2D00803EB800002F075
:104378000702046A92004FF00F0C0CFA02FC24EAC0
:104388000C040462046A01FA02F222430024026265
:104398004FF0010C224603E0102A04F10204A1D0D8
:1043A8000CFA02F030EA0E0102F10102F4D1D3F85E
:1043B80008B00AFA04F1C9430BEA010BC3F808B0C4
:1043C800D3F808B0C3F808B0B3F804B01FFA8BFBF1
:1043D8002BEA00009880988880B298801868084076
:1043E8001860D3F800B009FA04F040EA0B0018602E
:1043F800D8680140D960CFE74FF40053D1F818A02E
:1044080043EA0A038B615FE7BDE8F88FD1F818A08B
:104418004FF4006343EA0A038B6155E7174A1748CC
:10442800D2694BEA0202C26197E7144A13489269BB
:104438004BEA0202826190E70123D1F81CA043EA0B
:104448000A03CB6140E70223F7E70423F5E71023CB
:10445800F3E72023F1E74FF48033CFE74FF400333D
:10446800CCE700BFA87800203C5A030800040040AD
:104478000008004000100040002C014000100240DD
:10448800A45B0308147B0020B05B0308B85B030837
:104498000040014000440140001400400034014045
:1044A80000480140002867D003682DE9F04F03F168
:1044B80038445C4EA40A0125345D04F01F066409E3
:1044C800022C05FA06F558D0032C00F0A580012C23
:1044D80058D08088B0FA80F4C4F11F04A4B2E5086B
:1044E80003EB850504F007042E6AA4000F27A740F4
:1044F80026EA07062E622E6A01F00307A2407C1EF8
:104508003243012CC1F3810CC1F300182A62C1F3B4
:1045180041113CD9C60700F18980850700F19580D3
:10452800440700F1A380020700F1B180C60600F13C
:10453800BF80850600F1CD80440600F1DB800206CD
:1045480000F1E980C60500F1F780850500F10581D5
:10455800440500F11381020500F12181C60400F130
:104568002F81850400F13D81440400F14B81020450
:1045780000F15981BDE8F08F70472B4CA66935438F
:10458800A561A6E7284C666935436561A1E7002463
:1045980022464FF0010E4FF0030904E00132102AC1
:1045A80004F10204E6D00EFA02F636EA0005F5D167
:1045B800D3F808A009FA04F5ED430AEA050AC3F896
:1045C80008A0D3F808B00CFA04FA4AEA0B0AC3F8B0
:1045D80008A0B3F804A01FFA8AFA2AEA06069E8001
:1045E800B3F804A008FA02F646EA0A06B6B29E80B4
:1045F8001E682E401E60D3F800A007FA04F646EAAB
:104608000A061E60D3F80CA001FA04F605EA0A0AA5
:1046180046EA0A05DD60C1E7034CE6693543E56112
:1046280057E700BFB85B0308001002401A6822F081
:1046380003021A601A683A431A60DA6822F0030221
:104648000A438507DA607FF56BAF1A6822F00C021F
:104658001A601A6842EA87021A60DA6822F00C02C5
:1046680042EA81024407DA607FF55DAF1A6822F0FA
:1046780030021A601A6842EA07121A60DA6822F0F1
:10468800300242EA0112DA6002077FF54FAF1A687A
:1046980022F0C0021A601A6842EA87121A60DA68C1
:1046A80022F0C00242EA8112C606DA607FF541AF05
:1046B8001A6822F440721A601A6842EA07221A60DD
:1046C800DA6822F4407242EA01228506DA607FF550
:1046D80033AF1A6822F440621A601A6842EA8722E5
:1046E8001A60DA6822F4406242EA81224406DA60FB
:1046F8007FF525AF1A6822F440521A601A6842EA18
:1047080007321A60DA6822F4405242EA0132DA606B
:1047180002067FF517AF1A6822F440421A601A6839
:1047280042EA87321A60DA6822F4404242EA813269
:10473800C605DA607FF509AF1A6822F440321A60BC
:104748001A6842EA07421A60DA6822F4403242EAFA
:1047580001428505DA607FF5FBAE1A6822F4402233
:104768001A601A6842EA87421A60DA6822F440221C
:1047780042EA81424405DA607FF5EDAE1A6822F418
:1047880040121A601A6842EA07521A60DA6822F47C
:10479800401242EA0152DA6002057FF5DFAE1A687C
:1047A80022F440021A601A6842EA87521A60DA68EC
:1047B80022F4400242EA8152C604DA607FF5D1AEA3
:1047C8001A6822F040721A601A6842EA07621A6090
:1047D800DA6822F0407242EA01628504DA607FF505
:1047E800C3AE1A6822F040621A601A6842EA876209
:1047F8001A60DA6822F0406242EA81624404DA60B0
:104808007FF5B5AE1A6822F040521A601A6842EA7B
:1048180007721A60DA6822F0405242EA0172DA60DE
:1048280002047FF5A7AE1A6822F040421A601A689F
:1048380042EA87771F60DA6822F0404242EA8171D3
:10484800D960BDE8F08F00BF03682DE9F04F03F190
:104858003845644EAD0A0124755D05F01F066D09E3
:10486800022D04FA06F400F0A280032D00F0A480C3
:10487800012D52D08088B0FA80F4C4F11F04A4B28C
:10488800E50803EB850504F007042E6AA4000F274A
:10489800A74026EA07062E622E6A01F0030702FAED
:1048A80004F47A1E3443012AC1F3810CC1F30018C1
:1048B8002C62C1F3411135D9C60700F197808507ED
:1048C80000F1A380440700F1B180020700F1BF8026
:1048D800C60600F1CD80850600F1DB80440600F1B4
:1048E800E980020600F1F780C60500F1058185051B
:1048F80000F11381440500F12181020500F12F81A7
:10490800C60400F13D81850400F14B81440400F1A7
:104918005981020455D4BDE8F08F334D6E69344394
:104928006C61A7E7002422464FF0010E4FF00309FF
:1049380004E00132102A04F10204ECD00EFA02F667
:1049480036EA0005F5D1D3F808A009FA04F5ED43D5
:104958000AEA050AC3F808A0D3F808B00CFA04FA62
:104968004AEA0B0AC3F808A0B3F804A01FFA8AFAA7
:104978002AEA06069E80B3F804A008FA02F646EA78
:104988000A06B6B29E801E682E401E60D3F800A0AC
:1049980007FA04F646EA0A061E60D3F80CA001FAE4
:1049A80004F605EA0A0A46EA0A05DD60C1E70E4D83
:1049B800AE693443AC615DE70B4DEE693443EC619D
:1049C80058E71A6822F040421A601A6842EA877764
:1049D8001F60DA6822F0404242EA8171D960BDE87E
:1049E800F08F00BFB85B0308001002401A6822F07D
:1049F80003021A601A683A431A60DA6822F003025E
:104A08000A438507DA607FF55DAF1A6822F00C0269
:104A18001A601A6842EA87021A60DA6822F00C0201
:104A280042EA81024407DA607FF54FAF1A6822F044
:104A380030021A601A6842EA07121A60DA6822F02D
:104A4800300242EA0112DA6002077FF541AF1A68C4
:104A580022F0C0021A601A6842EA87121A60DA68FD
:104A680022F0C00242EA8112C606DA607FF533AF4F
:104A78001A6822F440721A601A6842EA07221A6019
:104A8800DA6822F4407242EA01228506DA607FF58C
:104A980025AF1A6822F440621A601A6842EA87222F
:104AA8001A60DA6822F4406242EA81224406DA6037
:104AB8007FF517AF1A6822F440521A601A6842EA62
:104AC80007321A60DA6822F4405242EA0132DA60A8
:104AD80002067FF509AF1A6822F440421A601A6884
:104AE80042EA87321A60DA6822F4404242EA8132A6
:104AF800C605DA607FF5FBAE1A6822F440321A6008
:104B08001A6842EA07421A60DA6822F4403242EA36
:104B180001428505DA607FF5EDAE1A6822F440227D
:104B28001A601A6842EA87421A60DA6822F4402258
:104B380042EA81424405DA607FF5DFAE1A6822F462
:104B480040121A601A6842EA07521A60DA6822F4B8
:104B5800401242EA0152DA6002057FF5D1AE1A68C6
:104B680022F440021A601A6842EA87521A60DA6828
:104B780022F4400242EA8152C604DA607FF5C3AEED
:104B88001A6822F040721A601A6842EA07621A60CC
:104B9800DA6822F0407242EA01628504DA607FF541
:104BA800B5AE1A6822F040621A601A6842EA876253
:104BB8001A60DA6822F0406242EA81624404DA60EC
:104BC8007FF5A7AE1A6822F040521A601A6842EAC6
:104BD80007721A60DA6822F0405242EA0172DA601B
:104BE80097E600BF10B50409013C052C17D80D4BFA
:104BF80033F8142000F00F0042FA00F313F0010319
:104C08000DD0012303FA00F0013810402CF0B8FE53
:104C1800054A064B125D104403EBC00010BD00208E
:104C280010BD00BFA45B0308B05B0308147B002021
:104C380001490248FEF732BEC07900200048014011
:104C480001490248FEF72ABE707900200040014061
:104C580001490248FEF722BE48790020003401408D
:104C680001490248FEF71ABE487900200034014085
:104C780001490248FEF712BE2079002000080040D2
:104C880001490248FEF70ABEF878002000040040F7
:104C980002494FF08040FEF701BE00BFD0780020E7
:104CA80010B5064C06482146FEF7F8FD04F1F00160
:104CB8000448BDE81040FEF7F1BD00BFA878002009
:104CC800002C01400044014001490248FEF7E6BDBE
:104CD800A8780020002C01402DE9F0410468574DC8
:104CE800A30AAB4200F085805CD9554DAB426CD02D
:104CF80078D9544DAB4264D00135AB4240F09A802C
:104D08004FF49C7E072647794FEA970C00297CD000
:104D1800B000634685190227D4F80C809F400CEB3D
:104D28004503BFB2484D03F1040C47EA080745F8AC
:104D3800231045F82C20E760EFF31181502282F30D
:104D48001288821905EBC2021369002B41D0136245
:104D58000433821905EBC202576917B11F60536902
:104D68000433821905EBC202976917B11F60936972
:104D78000433821905EBC202D76917B11F60D369E2
:104D880004330027CAB21F6082F31188304405EB50
:104D9800C000036A03BBE3684FF6FE721340E3608A
:104DA800BDE8F0814A3DAB422BD00135AB4204D07F
:104DB800B3F5801F21D0BDE8F0814FF0980E03268F
:104DC800A1E74FF4887E06269DE74FF0E80E0526FA
:104DD80099E705EB0E03BCE7E36843F00103E360E2
:104DE800BDE8F081033DAB4226D14FF0C00E04264A
:104DF80089E74FF0200E002685E74FF0480E012680
:104E080081E74FF0700E02267DE7BF08022306FAFD
:104E180003F0BB40DB43E7680B4D9BB23B4087196F
:104E28000CEB470CE3600CF1040345F82C1045F833
:104E3800232081E7BDE8F081BDE8F0814B00100038
:104E48005000100051001000A878002030B5036809
:104E58005C4D18885C4CB4FBF2F20139013AAB4264
:104E680094B283B089B282B266D05848834263D084
:104E7800B3F1804F60D0A0F5983083425CD000F544
:104E88008060834258D0524883425BD000F58060EE
:104E980083427DD022F4407200F58C3092B2834276
:104EA8001A80D9621C850ED0484A93420BD002F56D
:104EB8004062934207D002F58062934203D002F524
:104EC8008062934201D100221A8601225A611A880F
:104ED8003C4992B242F001028B421A8062D0B3F18F
:104EE800804F61D03B4A934260D002F58062934282
:104EF8005ED002F5006293425CD002F58062934274
:104F08005AD002F59032934258D002F5406293424B
:104F180056D002F5806293421ED002F58062934219
:104F280008BF092219D002A84FF0012340F8043D18
:104F38001BF0E0FB03B030BD254822F0700283422D
:104F480092B2A3D101201A80D9621C8558611A88AF
:104F580092B202431A80C5E708221F4B03EBC20333
:104F680001A893F831408DF80440012300228DF800
:104F780005308DF807308DF806201BF0BBFB1B2C85
:104F8800D8D1164B019301A81BF0B4FB03B030BD78
:104F980001201A80D9621C8558611A8892B202438E
:104FA8001A809CE70022D8E70122D6E70222D4E73C
:104FB8000322D2E70422D0E70522CEE70622CCE777
:104FC8000722CAE7002C014000A24A04003401402D
:104FD8000010004000040040A0320308190100013D
:104FE800204B98422DD0B0F1804F2CD0A3F59433AC
:104FF80098422AD003F58063984228D003F50063CD
:10500800984226D003F58063984224D003F5903364
:10501800984222D003F54063984220D003F580637C
:10502800984207D003F58063984208BF092202D04E
:105038000020704708220C4B03EBC20393F83000A2
:1050480070470022F7E70122F5E70222F3E703227F
:10505800F1E70422EFE70522EDE70622EBE7072256
:10506800E9E700BF002C0140A03203082DE9F04F0A
:10507800013085B0C3B203930B4602918B4C8C4E22
:10508800002B00F09A8032208A4D8B4FDFF82C924B
:1050980028F056F84FF4FA7A4FF0100C4FF47A7063
:1050A800D9F80430C3F30803002B40F0DE80EFF397
:1050B8001183002B40F0D9802968A26800BF2B68B3
:1050C8009942F9D1D7F800E000FB0EF39B1AB3FB25
:1050D800FEF300FB01314FF0010E0191D9F80430C5
:1050E800C3F30803002B40F08780EFF31183002BF4
:1050F80040F082802B68A16800BF2A689342F9D1EA
:10510800D7F800B000FB0BF2521AB2FBFBF200FB1F
:105118000323019A9B1AB3F57A7FDFD3BAF1010A08
:10512800BED1039B002B40F0BD804FF47A7ADFF8A4
:105138008C9150464FF0100CD9F80430C3F3080393
:10514800002B75D1EFF31183002B71D12968A26868
:1051580000BF2B689942F9D1D7F800E000FB0EF3A5
:105168009B1AB3FBFEF300FB01314FF0010E0191D6
:10517800D9F80430C3F3080313BBEFF31183FBB969
:105188002B68A16800BF2A689342F9D1D7F800B00C
:1051980000FB0BF2521AB2FBFBF200FB0323019A4D
:1051A8009B1AB3F57A7FE3D3BAF1010AC4D1029B03
:1051B800013B0293002B7FF466AF05B0BDE8F08F8A
:1051C800EFF311888CF31288A1682368DB0344BFCE
:1051D800C6F800E0A1682B6832685FFA88F888F39F
:1051E8001188D7F800801A4400FB08F35B1AB3FB58
:1051F800F8F300FB0233D2E7EFF311888CF312883F
:10520800A1682368DB0344BFC6F800E0A1682B68E7
:1052180032685FFA88F888F31188D7F800801A4452
:1052280000FB08F35B1AB3FBF8F300FB023370E7EB
:10523800EFF311828CF31288D4F808E02368D903BD
:1052480003D501233360D4F808E02B683168D2B263
:1052580082F311883A68194400FB02F3A3EB0E03AA
:10526800B3FBF2F300FB01317FE7EFF311828CF31C
:105278001288D4F808E02368D90303D501233360E2
:10528800D4F808E02B683168D2B282F311883A6802
:10529800194400FB02F3A3EB0E03B3FBF2F300FB8C
:1052A800013118E7184627F0BBFD3EE710E000E0A3
:1052B800D0560020D4560020D856002000ED00E03B
:1052C800204B5B68C3F3080330B4BBB9EFF3118319
:1052D800A3B91D4B1D4C1868A16800BF1A689042FD
:1052E800F9D11B4B1C684FF47A7202FB04F3591A6C
:1052F800B1FBF4F130BC02FB00107047EFF31182F0
:10530800102383F3128811498C680B6813F4803FCB
:10531800104B02D0012018608C680B49D2B20D687E
:10532800186882F311880A4B19684FF47A72284476
:1053380002FB01F31B1B30BCB3FBF1F302FB003093
:10534800704700BF00ED00E0D456002010E000E0F8
:10535800D8560020D05600202DE9F84F8046FFF798
:10536800AFFF254E2549DFF8A0E0254A254D8446A4
:1053780010274FF47A740120DEF80430C3F30803D1
:10538800D3B9EFF31183BBB90B68D2F808A000BFFB
:10539800D1F800904B45F7D1D6F800B004FB0BF9D3
:1053A800A9EB0A09B9FBFBF904FB0393A3EB0C0374
:1053B8004345E1D3BDE8F88FEFF3118A87F31288EC
:1053C800D2F808B01368DB0344BF2860D2F808B0ED
:1053D8000B68D5F800905FFA8AFA8AF31188D6F834
:1053E80000A0994404FB0AF3A3EB0B03B3FBFAF305
:1053F80004FB0933DAE700BFD8560020D456002052
:1054080010E000E0D056002000ED00E02DE9F04F5C
:10541800DFF830C1474A4849484E494D8046102771
:1054280018F1FF38C0F08480DCF80430C3F30803B7
:10543800002B5CD1EFF31183002B58D10B689468D3
:1054480000BF08688342F9D1D6F800904FF47A700B
:1054580000FB09FEAEEB040EBEFBF9FE00FB03EEFB
:10546800DCF80430C3F308034FF47A740120FBB965
:10547800EFF31183E3B90B68D2F808A000BFD1F8A5
:1054880000904B45F7D1D6F800B004FB0BF9A9EB17
:105498000A09B9FBFBF904FB0393A3EB0E03B3F56D
:1054A8007A7FBDD2DCF80430C3F30803002BDFD0C9
:1054B800EFF3118A87F31288D2F808B01368DB0378
:1054C80044BF2860D2F808B00B68D5F800905FFA9E
:1054D8008AFA8AF31188D6F800A0994404FB0AF3E3
:1054E800A3EB0B03B3FBFAF304FB0933D5E7EFF3A4
:1054F800118487F31288D2F808901368D80303D56B
:1055080001232B60D2F808900B682868E4B284F372
:105518001188D6F800A04FF47A7400EB030E04FB50
:105528000AF3A3EB0903B3FBFAF304FB0E3E97E778
:10553800BDE8F08F10E000E0D4560020D8560020D7
:10554800D056002000ED00E030B4EFF311831022B4
:1055580082F312880649074C0A6807480132002579
:105568000A602560DBB2026883F3118830BC70479B
:10557800D4560020D056002010E000E01D4B70B536
:105588005C68236D626BDD69C2B1A36B2BB12B071D
:1055980002D5236D08221A6270BD2A06F7D5A26AC1
:1055A800616A8A4220D0511CA069A162825C20698C
:1055B800266D81423285EAD3A362E8E7A906E4D5DD
:1055C800E26A22B1988C216B80B29047DDE7E169ED
:1055D8009B8C6069DBB24E1CE6614354E169E36869
:1055E800994228BFE261D0E7226D136823F0800357
:1055F8001360CCE7C42900201D4B70B51C68236DCF
:10560800626BDD69C2B1A36B2BB12B0702D5236D89
:1056180008221A6270BD2A06F7D5A26A616A8A4210
:1056280020D0511CA069A162825C2069266D81424C
:105638003285EAD3A362E8E7A906E4D5E26A22B193
:10564800988C216B80B29047DDE7E1699B8C60699B
:10565800DBB24E1CE6614354E169E368994228BF16
:10566800E261D0E7226D136823F080031360CCE772
:10567800C429002070B4EFF31186502383F31288F5
:10568800836B1A68D20720D45D686DB9446A826A50
:10569800944217D081691144D9600ED9A21A5A6070
:1056A8008462002280F854201A6842F00102F1B2A4
:1056B8001A6081F3118870BC704701698A1A5A60B0
:1056C8008562EEE7012380F85430F1B281F3118846
:1056D80070BC704703682DE9F041DF691FB13B4694
:1056E800BDE8F0411847002A164611DD04460D466C
:1056F8000E4400E023689B68204698470028F9D0AC
:10570800236815F8011B1B6820469847AE42F1D163
:10571800BDE8F08103689B69184700BF03685B69AF
:10572800184700BF0368DB68184700BF03685B6859
:10573800184700BF03681B68184700BF054B53F89C
:10574800203033B11A689B88918A0B4218BF1B041A
:1057580093617047A0560020036803F138422DE991
:10576800F04F920A584DAA5C02F01F055209012415
:10577800022A04FA05F400F08C80032A00F08E80D7
:10578800012A3CD001F003077A1E012AC1F3810CDB
:10579800C1F300188088C1F3411135D9C60700F15B
:1057A8009780850700F1A380440700F1B1800207C4
:1057B80000F1BF80C60600F1CD80850600F1DB80D0
:1057C800440600F1E980020600F1F780C60500F101
:1057D8000581850500F11381440500F12181020549
:1057E80000F12F81C60400F13D81850400F14B8151
:1057F800440400F15981020455D4BDE8F08F334ABE
:1058080055692C435461BDE7002422464FF0010E30
:105818004FF0030904E00132102A04F10204ECD02D
:105828000EFA02F636EA0005F5D1D3F808A009FA0F
:1058380004F5ED430AEA050AC3F808A0D3F808B04E
:105848000CFA04FA4AEA0B0AC3F808A0B3F804A051
:105858001FFA8AFA2AEA06069E80B3F804A008FA14
:1058680002F646EA0A06B6B29E801E682E401E6000
:10587800D3F800A007FA04F646EA0A061E60D3F831
:105888000CA001FA04F605EA0A0A46EA0A05DD60F0
:10589800C1E70E4A95692C43946173E70B4AD569B1
:1058A8002C43D4616EE71A6822F040421A601A68E5
:1058B80042EA87771F60DA6822F0404242EA817143
:1058C800D960BDE8F08F00BFB85B03080010024044
:1058D8001A6822F003021A601A683A431A60DA68F2
:1058E80022F003020A438507DA607FF55DAF1A6884
:1058F80022F00C021A601A6842EA87021A60DA6813
:1059080022F00C0242EA81024407DA607FF54FAFC9
:105918001A6822F030021A601A6842EA07121A60FE
:10592800DA6822F0300242EA0112DA6002077FF5F3
:1059380041AF1A6822F0C0021A601A6842EA871258
:105948001A60DA6822F0C00242EA8112C606DA60FA
:105958007FF533AF1A6822F440721A601A6842EA77
:1059680007221A60DA6822F4407242EA01228506A8
:10597800DA607FF525AF1A6822F440621A601A6867
:1059880042EA87221A60DA6822F4406242EA8122F7
:105998004406DA607FF517AF1A6822F440521A609D
:1059A8001A6842EA07321A60DA6822F4405242EA78
:1059B8000132DA6002067FF509AF1A6822F4404224
:1059C8001A601A6842EA87321A60DA6822F440429A
:1059D80042EA8132C605DA607FF5FBAE1A6822F426
:1059E80040321A601A6842EA07421A60DA6822F4FA
:1059F800403242EA01428505DA607FF5EDAE1A6869
:105A080022F440221A601A6842EA87421A60DA6869
:105A180022F4402242EA81424405DA607FF5DFAE93
:105A28001A6822F440121A601A6842EA07521A6089
:105A3800DA6822F4401242EA0152DA6002057FF580
:105A4800D1AE1A6822F440021A601A6842EA8752F4
:105A58001A60DA6822F4400242EA8152C604DA6027
:105A68007FF5C3AE1A6822F040721A601A6842EADB
:105A780007621A60DA6822F0407242EA016285041D
:105A8800DA607FF5B5AE1A6822F040621A601A68CB
:105A980042EA87621A60DA6822F0406242EA81626A
:105AA8004404DA607FF5A7AE1A6822F040521A6003
:105AB8001A6842EA07721A60DA6822F0405242EA2B
:105AC8000172DA6097E600BF2DE9F04F4A484B4B68
:105AD8004B4C4FF090414FF0010A4FF002094FF044
:105AE80004084FF0080C4FF0100E202740268025A0
:105AF80030F8022B12F0010F03D01960A3F804A0AC
:105B0800083312F0020F03D01960A3F80490083389
:105B180012F0040F03D01960A3F80480083312F0C0
:105B2800080F03D01960A3F804C0083312F0100F4F
:105B380003D01960A3F804E0083312F0200F02D054
:105B480019609F80083312F0400F02D019609E80C0
:105B5800083312F0800F02D019609D80083312F4C8
:105B6800807F05D04FF4807B1960A3F804B0083318
:105B780012F4007F05D04FF4007B1960A3F804B03D
:105B8800083312F4806F05D04FF4806B1960A3F8C6
:105B980004B0083312F4006F05D04FF4006B19609D
:105BA800A3F804B0083312F4805F05D04FF4805B8B
:105BB8001960A3F804B0083312F4005F05D04FF45D
:105BC800005B1960A3F804B0083312F4804F05D0C5
:105BD8004FF4804B1960A3F804B00833D20B04D0FB
:105BE8004FF4004219609A80083301F58061A142A0
:105BF8007FF47EAFBDE8F08FA45B0308147B002020
:105C080000180048002852D0036803F138422DE9F3
:105C1800F04F920A504DAA5C02F01F055209012468
:105C2800022A04FA05F443D0032A00F09080012ADE
:105C380043D001F003077A1E012AC1F3810CC1F396
:105C480000188088C1F341113CD9C60700F188804B
:105C5800850700F19480440700F1A280020700F153
:105C6800B080C60600F1BE80850600F1CC804406EF
:105C780000F1DA80020600F1E880C60500F1F6803E
:105C8800850500F10481440500F11281020500F147
:105C98002081C60400F12E81850400F13C81440472
:105CA80000F14A81020400F15881BDE8F08F704785
:105CB8002A4A95692C439461BBE7284A55692C43C5
:105CC8005461B6E7002422464FF0010E4FF0030955
:105CD80004E00132102A04F10204E6D00EFA02F6BA
:105CE80036EA0005F5D1D3F808A009FA04F5ED4322
:105CF8000AEA050AC3F808A0D3F808B00CFA04FAAF
:105D08004AEA0B0AC3F808A0B3F804A01FFA8AFAF3
:105D18002AEA06069E80B3F804A008FA02F646EAC4
:105D28000A06B6B29E801E682E401E60D3F800A0F8
:105D380007FA04F646EA0A061E60D3F80CA001FA30
:105D480004F605EA0A0A46EA0A05DD60C1E7034ADD
:105D5800D5692C43D4616CE7B85B03080010024096
:105D68001A6822F003021A601A683A431A60DA685D
:105D780022F003020A438507DA607FF56CAF1A68E0
:105D880022F00C021A601A6842EA87021A60DA687E
:105D980022F00C0242EA81024407DA607FF55EAF26
:105DA8001A6822F030021A601A6842EA07121A606A
:105DB800DA6822F0300242EA0112DA6002077FF55F
:105DC80050AF1A6822F0C0021A601A6842EA8712B5
:105DD8001A60DA6822F0C00242EA8112C606DA6066
:105DE8007FF542AF1A6822F440721A601A6842EAD4
:105DF80007221A60DA6822F4407242EA0122850614
:105E0800DA607FF534AF1A6822F440621A601A68C3
:105E180042EA87221A60DA6822F4406242EA812262
:105E28004406DA607FF526AF1A6822F440521A60F9
:105E38001A6842EA07321A60DA6822F4405242EAE3
:105E48000132DA6002067FF518AF1A6822F4404280
:105E58001A601A6842EA87321A60DA6822F4404205
:105E680042EA8132C605DA607FF50AAF1A6822F481
:105E780040321A601A6842EA07421A60DA6822F465
:105E8800403242EA01428505DA607FF5FCAE1A68C5
:105E980022F440221A601A6842EA87421A60DA68D5
:105EA80022F4402242EA81424405DA607FF5EEAEF0
:105EB8001A6822F440121A601A6842EA07521A60F5
:105EC800DA6822F4401242EA0152DA6002057FF5EC
:105ED800E0AE1A6822F440021A601A6842EA875251
:105EE8001A60DA6822F4400242EA8152C604DA6093
:105EF8007FF5D2AE1A6822F040721A601A6842EA38
:105F080007621A60DA6822F0407242EA0162850488
:105F1800DA607FF5C4AE1A6822F040621A601A6827
:105F280042EA87621A60DA6822F0406242EA8162D5
:105F38004404DA607FF5B6AE1A6822F040521A605F
:105F48001A6842EA07721A60DA6822F0405242EA96
:105F58000172DA6002047FF5A8AE1A6822F04042A6
:105F68001A601A6842EA87771F60DA6822F04042AE
:105F780042EA8171D960BDE8F08F00BF10B10368B3
:105F880082881A85704700BF10B1036882889A61B9
:105F9800704700BF38B100298388026814BF002108
:105FA80010218B40936170470E4B1B8801463BB90B
:105FB8000D4B0E4A1B7810680BB981F00101E9E717
:105FC8000B4B5A691AB118B91A681060587470479F
:105FD800084A18681188084A92FBF1F20121026008
:105FE80059747047AC560020AE560020B0560020B9
:105FF800B4560020CC56002020A1070010B40A4B4C
:106008000A4A1C7801238340234052F8200029B90A
:10601800B3FA83F149095DF8044BBBE7191C18BFB3
:1060280001215DF8044BB5E79C560020A0560020DE
:1060380008B501210220FFF7E1FF094B1B7803F0A7
:106048000503052B08D000210120FFF7D7FF002109
:106058000846FFF7D3FFFEE717F05EF8F3E700BF47
:10606800C02900202DE9F041044618460D46164681
:1060780098462AF08BFF2768E6722844A0722946C2
:106088007D69434632462046AC46BDE8F04160474C
:10609800036810B504461B689847236820469B6828
:1060A8009847A37B0133A37310BD00BF2DE9F04FC0
:1060B800BF4B1E788BB0002E40F0BC80BD4BBE4C51
:1060C8001D78DFF814A3DFF81493DFF8148305F0C4
:1060D8000105A4F10A0B54F80A3CBBB1CC2707FB15
:1060E80006B71846FFF722FB80B154F80A0CFFF7F1
:1060F80019FB14F8023C8BB9242831D0F5B154F8B7
:106108000A3C1846FFF712FB0028EED10136032E91
:1061180004F1CC04DFD10BB0BDE8F08F012B23D004
:10612800022B2BD0032B37D0042B67D0052B40D064
:10613800062B4FD054F80A2C1346D2E754F80A3CE1
:1061480023281A4600F087819C4991F82A10814239
:10615800C7D19B4BCAF80090C3F80C801346C0E720
:10616800012304F8023CCAE74D2854F80A2C0CBF56
:106178000223002304F8023C1346B2E700233C281C
:1061880004F8023C45D03E28D4D10122032304F868
:10619800012C04F8023CB2E7C02814D800220423DA
:1061A80004F8050C04F8040C04F8062C04F8023C66
:1061B800A5E714F8063C14F8052C9A422FD814F8D1
:1061C800043C834203D0002304F8023C97E70623EB
:1061D80004F8023C14F801ECBEF1000F00F07E81D7
:1061E800BEF1010F00F0C28101360023032E04F82E
:1061F800023C04F1CC047FF46EAF8CE714F8043C45
:1062080004F8030C5840052304F8040C04F8023C75
:1062180075E7032204F8013C04F8022C6FE714F830
:10622800042CF9184240013304F8042C04F8063C05
:10623800887264E7634B186800283FF46CAFFAF77C
:10624800CBFFDFF8A0A1604DDFF89C91DAF80000E1
:10625800FFF76CFA00283FF45EAFDAF80000FFF7AA
:1062680061FA09281BD03F2819D02B68002B66D16A
:10627800042800F0A6810C2800F0E6807F28E5D0ED
:10628800A0F12002D2B25E2AE0D80BB92028DDD0D6
:106298005A1C09F803002A600FF062FFD6E72C6841
:1062A800002C5AD1494B264603F5887B002E08BF9F
:1062B8001E4608335B45F9D1002E00F07681A3F124
:1062C80008083068D8F80020075D135D9F42204415
:1062D80002EB040140F06781671E4F4422460BB968
:1062E800FD2A5CD907F8013F01322A6010F8013F06
:1062F80011F801EF9E45F2D00AB1B04512D03448EA
:106308000FF036FFB04508D356F8080B0FF030FFF2
:1063180009200FF025FF4645F6D92E480FF028FF33
:106328002A680024944291D2661E4E4416F8010F42
:106338000FF016FF2B6801349C42F7D386E70C2830
:1063480000F082800A2851D00D284FD07F2800F015
:10635800FA80FF2B3FF67AAF92E71C4F4FF0000808
:1063680007F5887B464602E008375F450DD0224690
:1063780039684846FBF708FB0028F5D1B846002ED7
:10638800F2D13E4608375F45F1D1002E99D1B8F1D8
:10639800000F3FF45BAF0E480FF0EAFEB4E7511C64
:1063A800202009F80200296009F801300A46A4E70C
:1063B800593B0020EF3A0020EE6B0020147A0020B1
:1063C80000ED00E0882A0020902B00209438030874
:1063D800E85B0308F05B0308FC9F0020EFBEADDE1E
:1063E8000400FA058C2A0020902A00200FF041FFB3
:1063F80023217C482CF077FE002800F0E080A0EBF9
:106408000900286088B1431E19F80310202940F0BC
:10641800E68009EB030204E012F8011D202946D1A9
:106428000346581E002BF7D12B604FF480720021D1
:1064380048462CF041FE6C4B1B78002B3FF46BAEAA
:106448006A480FF095FE01E769480FF091FE67482A
:106458000FF08EFEFAE667496748C978674ADFF8A1
:10646800CCE11360003118BF01210170644951600B
:106478004021936011735573624963480B6004327D
:10648800CEF80020584A0123137010F00DFA57482F
:106498000FF06EFE4FF400600CF0B8FC5B4B93F805
:1064A8002A30232B00F0938014F8023C40E62B603E
:1064B800574C002204F5887B09F8032002E00834D1
:1064C8005C4578D0216848460FF0B2FC0028F6D029
:1064D8005C4570D2636898470023A5E74D4BADF83B
:1064E80022E00FCB0DF1280C02AF87E80F004CF823
:1064F80024ED14F8051C14F8033C069404EB010E73
:10650800624639464FF0010C06A8CDF81CE0ADF8FC
:1065180020308DF824C00AF02DF8E8B9019F002337
:1065280004F8023C002F3FF4F1AD54F80A0C1FF0B8
:10653800C7FB013654F80A0CB847032E04F1CC0403
:106548007FF4C9ADE7E5013B002233482B6009F829
:1065580003200FF00DFE79E6029A304B039239467C
:10656800A4F10A0002930DF0B7FBD7E714F8053C35
:1065780014F8032C0694234407936E2A4FF0000363
:1065880008930993ADF820207FF42EAE06A8FBF7F8
:106598007DFA06A8FBF76EFA06A8FBF76BFA06A8C1
:1065A800FBF768FA20E62246A6E61D48A3F108088C
:1065B8000FF0DEFDA8E61B480FF0DAFD8CE728682F
:1065C80020E708480EF0A8FC0BB0BDE8F08F164A8B
:1065D80014F8023CC2F80C80CAF80090A8E50346FB
:1065E80066E700BF902A0020593B0020F05B0308B3
:1065F800F85B0308283E0020F0240020901D0020AE
:10660800313800088C2A0020245C0308147A002002
:10661800943803081C330308205C0308187F002003
:10662800E85B0308045C030800ED00E0882A00200A
:106638002DE9F04F2DED068BAB4BAC4A1C7897B08B
:1066480000F59C41203181460B911160002C00F02F
:10665800E886A74A1268904240F28380A54A0692CB
:106668001668A549A54A0591013C1C70A44B0492E3
:1066780006F480560893002E40F08180A14B1B78C9
:10668800022B01F08E81042B01F07D81012B01F09A
:1066980031819D4B9945089B9B7800F29685002B8C
:1066A80040F09785994B0793069B1E6816F4805710
:1066B80040F08586DFF894A2049BB3F90610059B89
:1066C8005D8BA942B4BF00250125914B1B6813F0CF
:1066D80080535ED0079A127812F001025FD00598B5
:1066E800408C884241F3B082002D5ED1894C94F8E9
:1066F8008C10002959D188488849006890F82D00E5
:1067080000240C604C608C60854900284ED10870CC
:10671800002A4FD0F1064DD5824A1278D20649D4C4
:10672800002F47D1002B45D1740243D47E4B1B78F0
:10673800002B02F033827D4B9B78002D42F0C782FC
:106748003BB17B4A7B4B12681B689B1A002BC2F239
:10675800B68210206F4C1FF0E9FF012384F88D30BA
:1067680028E0644B06931E68644B634A049306F45E
:106778008056634B05920893002E3FF47FAF0021AB
:106788006348FBF795FC00287FF478AF14F016F9FE
:1067980074E770029ED4079A127802F001025D4CE9
:1067A800002184F88C10002DA5D05D4901200870C7
:1067B800002AAFD1604B1A78002A79D10599049C38
:1067C800488BB4F90070898BB4F90240B842B4BF61
:1067D8008026002646F04003B942D8BF33469B08BE
:1067E80043F08006A042B8BF3346049F43F04006FA
:1067F800A142C8BF33469B08B7F90440B7F9066001
:1068080043F08007A042B8BF3B4643F04007A1428F
:10681800C8BF3B469B0843F080073E4C8642C8BF32
:106828003B4643F0400794F88EE08E42B8BF3B46A3
:106838009E4501F06184A4F8902084F892203A499A
:1068480084F88E300E78002E01F058835F2B01F00B
:10685800D5836F2B01F01784079B1B78DA0727D4A1
:1068680094F8921021BBB4F99030322B20DD94F8C3
:106878008E200120572A84F8920001F08C87069B0D
:106888001B685F0741F1A6825A2A41F0A38294F857
:106898009430002B42F09C8194F8963083F00103E9
:1068A80084F89630002B42F0FE810C201FF03EFF4A
:1068B800224B0993224B234D0A93069B1B685C07C6
:1068C80000F1F3860DF150091F4E0B950022C9F80F
:1068D80004203446149240F6330B4FF0190840F266
:1068E8008337049D37E000BFF8380020D0370020F8
:1068F800F4380020184C0020E87900207C7700202C
:10690800783E002042400020404B4C00EF3A0020E7
:10691800FC560020E01D00206034002014570020A1
:106928006020002004570020681B0020E05500204C
:10693800D4560020A43400200B3D00200034002051
:10694800643400205C34002060390020B039002015
:106958000434544520D0A178E378994218FB01709B
:10696800F6D26178043118FB037335F911105945D3
:10697800A8BF5946B1F5617FB8BF4FF46171814234
:10698800E6DD9942E4DC21782729E1D84846043439
:10699800FBF77EFB5445DED1674A0B9D1378674AA7
:1069A80099E8030082E80300002B40F0BC85644BA3
:1069B8001A78002A00F0F88501216048FBF778FB77
:1069C800002840F0E682089BDB78002B40F0E1824B
:1069D8002B881FB227F001071FFA87F84345A5F84F
:1069E800008001F00D80574F4FF002090E204FF044
:1069F800140B4FF0FF0A87F8009087F801B087F86A
:106A080002A01FF093FE49464C48B5F80080FBF7FA
:106A18004FFB002800F0D88228F001039BB24345C1
:106A28002B800AD00E2087F8009087F801B087F8ED
:106A380002A01FF07BFEB5F8008018F0020F01F0ED
:106A4800B581414B414A197850680C9318F0030FEF
:106A580008BF81F00201C1F340010B92FFF79AFAD7
:106A680024213648FBF724FB30B9079A13785907D5
:106A780044BF23F004031370099B1B6813F00A0F2B
:106A88001BD005212D48FBF713FB002801F0B2802D
:106A98002F887B0741F1478228480621FBF708FB2E
:106AA800002801F09480780641F1358207212348B7
:106AB800FBF7FEFA002840F0B0870C211F48FBF7CF
:106AC800F7FA2A88002800F0938242F480739A42E9
:106AD8002B8009D01B4B022214211A700E20FF2292
:106AE80059709A701FF022FE194B1B78082B00F082
:106AF8008B820E2B00F08882069BD3F8008018F456
:106B0800806F5FD0134B1B79002B00F02482142177
:106B18000A48FBF7CDFA002840F022821AF00EFE50
:106B280001201FF049FD002849D0DFF82CA00027DC
:106B38004FF0CC0BA14614E03C4E0020FC56002040
:106B4800593B0020205500209C560020A0560020CC
:106B58001059002024320020E46B0020DFB2022FFD
:106B68002CD80BFB07F87B1C5AF80840002CF5D1F1
:106B7800032290F9023002940192C278E24951F856
:106B88002220009218462246234601211FF05EF972
:106B9800034607EB470000EB0010099353B1214669
:106BA8000AEB8000CC222CF087FA099B4AF80830BF
:106BB8000137FFB229F022FC0028D0D14C46069BB1
:106BC800D3F80080079B93F800A0D04B1AF0010A75
:106BD80000F06D8201221A700A9B04991B68B1F9B2
:106BE80006105A89CA4801279142077080F24582E7
:106BF800C84B4FF07E521A60059BC74FB3F81890E8
:106C0800049B97F90420B3F90030387897F801C04D
:106C1800002AA3EB090714BF01224FF0FF32002F0F
:106C2800B8BF7F42B7F5FA7FA8BF4FF4FA77B842EA
:106C380080F2BB823F1A07EE907AF8EEE77AB74FF8
:106C48004B45C7ED007A03DAF1EE677AC7ED007AB3
:106C5800049BB3F902E0AEEB0903002BB8BF5B421B
:106C6800B3F5FA7FA8BF4FF4FA73984280F2028214
:106C78001B1A07EE903AF8EEE77AF145C7ED017A6C
:106C880003DDF1EE677AC7ED017A049BB3F90400DE
:106C9800A0EB0903002BB8BF5B42B3F5FA7FA8BF8E
:106CA8004FF4FA736345CCBFA3EB0C03002302FB3C
:106CB80003F207EE902AF8EEE77A4845C7ED027A24
:106CC800BCBFF1EE677AC7ED027A18F4805800F07D
:106CD800AE81B1F5FA6F924BA8BF4FF4FA61B1F5E6
:106CE8007A7F1A78B8BF4FF47A71A1F57A71002AC1
:106CF80041F056818B4ADFF844E282FB0130CB1722
:106D0800C3EB6013581C6FF0630C3EF910003EF99A
:106D180013E00CFB0313A0EB0E0003FB00F382FB54
:106D28000312DB17C3EB62139E440FFA8EFE07EEC5
:106D380090EAB8EEE78A87ED038AB8F1000F40F0D1
:106D4800B2832B885A0640F1FB807749774A91ED48
:106D5800018AD2ED019A92ED026A91ED034A92ED11
:106D6800030A91ED029A92ED007AD1ED005AD7ED1F
:106D7800011A97ED002A6E4A6E4938EE445A79EEA8
:106D8800C63A77EE007A65EE233A75EEC96A75EE73
:106D9800890A37EE401A66EEA76AB0EE633AA0EEAB
:106DA800813A13F00303B0EE665A78EE044A79EE9E
:106DB800867AA0EE815AF0EE638AA4EEA73AD4EE62
:106DC800A78AA4EEE75A33EE263AF0EE687AF0EE98
:106DD800674AF6EE008A35EE88AAE0EEC14A28EE48
:106DE800C33A35EE635A77EE293A77EEE67AAAEE99
:106DF800233A25EE285A76EE403A34EE49AAE0EED8
:106E0800817A74EEA64AAAEE235A34EE094A37EE7E
:106E1800697A64EEA84A63EE036AE4EE074A75EEFF
:106E2800C85A36EE006A67EEA87AB0EE667A95EE32
:106E3800057AE5EE056AE5EE867AB1EE648AF0EE4B
:106E4800665AF0EE476AB1EE674AE8EE246A63EEE6
:106E5800270A67EEA43AE4EE275AB1EE450AB0EEE7
:106E6800609AB0EE631AA4EE277A23EE244AE7EE7E
:106E7800A76AA5EE249AA0EE031AE8EE245AB0EE0B
:106E8800448A31EEA16AE0EE240AA5EE278A66EE6E
:106E9800A16A72EE028AE5EE033A61EE211A26EE45
:106EA800096AA4EEA47AA0EE274A0CBFD7ED022AFD
:106EB800DFED212A82ED005AA2EE256AE8EEA06AEB
:106EC800E2EE081A73EEA33A27EE227A34EE044A69
:106ED800F0EE005AE3EEA26AA4EE226AA1EEA57AC9
:106EE800C7ED016AC1ED366A81ED356A87ED006A42
:106EF80081ED377A82ED013AC2ED027AC2ED034A9A
:106F0800F3B987ED027A1BE0983A0308F03A0020BB
:106F18009820002014200020B8550020343200208A
:106F2800682400201F85EB51B80E0020C80E0020F1
:106F3800000F0020E01D002000000000FC360020AB
:106F4800BAF1000F40F0348129F07AFB17B0BDEC9C
:106F5800068BBDE8F08F079B1B78D9077FF5DEAD60
:106F68004FF40F7027F0D4FE00283FF428AE0CF041
:106F78001BFF4FF40F7027F07DFE00283FF41FAE73
:106F88000CF012FF4FF40F7027F074FE0028EED1BA
:106F980015E6099B1B6898077FF51AADB5F80080C0
:106FA80018F0010F10D148F0010398452B800BD041
:106FB8009A4B022214211A700E20FF2259709A70DF
:106FC8001FF0B4FBB5F8008028F002039BB24345DC
:106FD8002B803FF436AD914B02201421FF2218700C
:106FE8000E2059709A701FF0A1FBB5F8008028E5B3
:106FF80022F480739BB29A422B807FF46BAD884B4E
:107008001B78082B7FF475AD2A8822F040039BB2C9
:107018009A422B803FF470AD804B022214211A70E3
:107028000E20FF2259709A701FF080FB64E5059BC3
:107038005A8B9142C0F2E184B1F5FA6FD4BFC2EB2A
:107048000101C2F5FA614FF47A7303FB01F1754847
:107058000378C2F5FA62B1FBF2F1002B3FF44AAEB5
:107068004378714A01FB03F182FB0123C917C1EB85
:1070780063113FE6DFED6D7AFFE5B1F5FA6F80F257
:10708800B584187A8B1A03FB00F3C2F5FA6293FBF6
:10709800F2F3C3F1640307EE903AF8EEE77A9FED56
:1070A800647A644B67EE877AC3ED007AA4E51B78AF
:1070B8000693002B7FF490AD5F4A1268002A3FF4D4
:1070C8008BAD5E4A079212F8030CDFF8A4B11146A3
:1070D800D71E16F0E9FC9BF80090079A002800F0EC
:1070E8000C86069BB9F1000F53D107F10801787996
:1070F80016F0DAFC002841F031855149B87A16F0CB
:10710800D3FC002800F00C86B9F1020F41F02E855F
:107118004C49F87B16F0C8FC002841F023854A4901
:10712800387D16F0C1FC002800F00C86B9F1040F78
:1071380041F02C854549787E16F0B6FC002841F0D0
:1071480021854349B87F16F0AFFC002800F00C8673
:10715800B9F1060F41F012853E4997F8230016F061
:10716800A3FC002841F006853B4997F8280016F053
:107178009BFC002800F00C86B9F1080F41F0DB8475
:10718800364997F82D0016F08FFC00283FF424ADFF
:1071980009231A4602EB82021744314A7878B978F3
:1071A8008BF800301070517016E5DFED207A46E557
:1071B8000C9B19780B9B01F001011868FEF7EAFE99
:1071C80017B0BDEC068BBDE8F08F13B9089A012300
:1071D8009370244B089A1D7892F8214007931B203E
:1071E80016F08CFC012C05F00108814600F0488758
:1071F80005F00205089A1C4E92F82030DFF874A0BA
:107208001A4F09959346052B00F2B487DFE813F06F
:10721800BC00B2003400FA00FC00EF00205500204A
:1072280010590020682400201F85EB510000000041
:107238000AD7233C14200020F43A0020EE54002002
:10724800F8540020FD540020025500200755002066
:107258000C55002011550020165500201B55002004
:10726800F83A0020EF3A0020F43600205834002085
:1072780000000020681B0020012C04BF05238BF8A8
:107288002030B8F1000F12D0059B3088B3F91810E0
:107298000022134661F30F0260F31F4261F30F03EC
:1072A800049861F31F430360032342600993B14DBF
:1072B800DBF814102A68914280F0108647F23051AA
:1072C8000322CBF81C108BF8202002200BF09EFD27
:1072D80013F074FB2968DBF81C200A440421CBF85E
:1072E80018208BF82010012C40F08A872A68DBF8D8
:1072F8001810914280F03E879AF8000020B916F0E5
:10730800FDFB002840F036873A6822F002023A6016
:107318002A687388642101FB03234FF480600022EC
:10732800CBF810308BF820208BF803200BF03EFDB3
:107338009BF8203067E716F0E7FB012807D18D4D51
:1073480072882B68642101FB0233CBF81030B9F145
:10735800000F02D0B379002B4BD1012C00F00A8723
:10736800844DDBF810102A689142C0F0568701233B
:107378008BF82030012C3AD0F379012B46D016F047
:1073880051FB9BF820303EE7B8F1000FD3D1099D9F
:107398004FF48060B9F1000F00F03C830BF01EFD44
:1073A800089A00231361002D3FF47EA928461FF098
:1073B800BDF9069B1E6816F480573FF47BA91D2172
:1073C8006D48FAF775FE00287FF474A96B4B03F13A
:1073D800500A03E004339A4500F0D2861A78262A28
:1073E800F8D19978DA789142F4D2FFF765B9614D0E
:1073F8008EE716F017FB03224FF47A738BF82020E0
:10740800CBF81C305B4D60E75A4D6CE716F00AFB71
:10741800032240F6B8338BF82020CBF81C30554DAA
:1074280053E7574F3B78002B01F08982554BDFF823
:107438006C81DFF86CB1DFF86CA1059345465E46B8
:10744800049099460EE019F804109847032C28DC9C
:1074580088B93B782AF8020F01349C4205F10405EB
:1074680080F24881072CE1B23046DBF80430EADDCF
:10747800984700B2EDE738F824206B88801A4FF45B
:107488007A719B1A01FB00F040F6CA0290FBF3F0F8
:107498000844904240F2EE23A8BF10469842B8BF75
:1074A800184600B2D5E71D213348FAF701FE28B186
:1074B80000F03ABE0436B4423FF443AC3178262992
:1074C800F8D1B278F3789A42F4D2089BDB78002B93
:1074D8007FF437AC2848FAF7EBFDDFED2B7A00286C
:1074E80001F0358238EE678A284A2949FDEEC87AC4
:1074F800CDED047ABDF910301B0382FB0302DB17C4
:10750800C3EBA212C9F57A731BB203FB02F343F370
:107518000F334B4407EE903AF8EEE77A0123C7EDB4
:10752800037A0B700DE4154B03E00433A3423FF4D8
:107538003EAA19782329F8D19878DA789042F4D2BB
:107548000D48FAF7B5FD00283FF431AA114B1B6826
:1075580013F4003341F0E68200220F4B1046995C89
:10756800142902F10C0201F0938101301828F6D198
:10757800FFF71DBAD4560020FC56002060390020C1
:10758800243A0020E879002000007A44D34D6210A4
:107598008C200020F85300203C500308383A002083
:1075A800583E0020DE1D0020DFF8F092DFF8F0A240
:1075B800AB4F0B9209F15A084FF0010B494619F8E5
:1075C800010C16F071FA00B399F8040099F802302A
:1075D80099F803E000EB400107EB8101013BD1F88A
:1075E800A02003EB4303534493420ED097F8CC20DA
:1075F800C1F8A0300BFA00F022EA00000B9B81F8DA
:107608009CE0C1F8A43087F8CC0009F10609C1450F
:10761800D4D1944B944A1B780B930A9BDFF884A22D
:1076280012681B680C93AAF19C094FF0000B904656
:10763800DAF8043083B31F7877B3DAF80820A8EBB8
:107648000202002A0CDB99F8CC20012101FA0BF187
:1076580022EA010208F5FA7189F8CC20CAF8081064
:107668000B9ACAB19AF8002059780432D2B200298C
:1076780040F02E8305990498098B30F9122001F106
:10768800C800824240F38E8599F8CC109A7841FA66
:107698000BF3D90740F119860BF1010BBBF1040F6D
:1076A8000AF10C0AC4D1FFF787B96D4C94F89630EB
:1076B8005BB1079B1B78D80707D5049BB3F9062055
:1076C800059B5B8B9A4200F3F28511216748FAF714
:1076D800EFFC002800F0A68294F89A302BB994F8B1
:1076E800943013B93223A4F89830012384F89A30DF
:1076F800FFF7E8B8DDF810905D4A06925D49126818
:1077080042F2010AA1FB091B12EA0A0A4FEA9B1B73
:1077180000F08582584D5948524C59492E780078C6
:10772800267008701EB156490E7886F001064C4C3A
:107738000F2184F82410002B00F01284059D514B72
:10774800B5F826C0B5F824E0059D109318462D8B92
:1077580000784D4B129594F8255009954B4D04959A
:10776800A3FB00535B0803EB4303C31ADBB20F9080
:10777800CDF834C002F480520C9304F128000BF5C4
:107788009673CDF8449097F80080DDF82490DFF8E0
:1077980018C109943D4C0E91139200210A93089642
:1077A800CDF81CE0089B002B00F03A83099B079D4D
:1077B80033F911201FFA82FEAE454FEA410303D385
:1077C8000D9DAE4540F271835CF82120934580F011
:1077D8003183E25EBAF1000F40F046830131414542
:1077E800E25200F10600DDDB0E9A099C284B84F872
:1077F80024200F2A49460CBF01220022DDF84490BC
:1078080084F825101A7000F0B283224B1B491C4AD9
:10781800DFF854B008931C46042001230B70137042
:107828000BF0F4FADBF80030A1686268E3605B1AD9
:10783800934284BF002384F82130069B3C781E685D
:10784800002C01F08080059A134DB2F824E0178BC4
:107858000E4916F48056284640F0B283324634E08A
:10786800E01D00209C3E0020D4560020FC5600203D
:10787800184C0020D34D6210AC370020100F0020A8
:10788800110F002015390020ABAAAAAA7C77002086
:107898009D3E0020783E00206C3A002005540020D0
:1078A8002C3303087C1E002018390020437803EB92
:1078B800830303EB830303F2EE239BB20132A2425C
:1078C80021F8023B00F102000ED015F81230002B0F
:1078D80000F0EF82022BE9D001320B8821F8023B3D
:1078E800A24200F10200F0D1109A1378013313700C
:1078F800FEF7C1BED74CD4F88830A9EB0303002BA0
:10790800FEF6C7AED44AD54B527C059933F81230EF
:107918008A7DDFEDD36A9FEDD36AC97D9BB207EEFE
:10792800102A07EE903AB8EEC77AF8EEE77A27EE13
:10793800267A67EE867A0B9AC4F88820C7EE876A9B
:1079480040F2FF32FCEEE67ACDED077ABDF81C3046
:10795800934228BF134609B1D31A9BB2C248C34DFC
:107968000178C34C35F81160226825F81130921B54
:1079780013440131BF4D236001F00F021B0902704F
:107988002B80FEF786BEFDF79BFCBB4BBB4A1B68F2
:10799800C31A93427EF77DAEB64B00221A80FEF7DB
:1079A80078BE059A0499537DD27D013B31F9133095
:1079B8001AB1C3F53B6308331BB2A3F57A7307EE1C
:1079C800903A9FEDAF7AAB4AF8EEE77A40F2FF3192
:1079D80067EE877AFCEEE77ACDED077ABDF81C30C2
:1079E8008B4228BF0B461380FEF753BE1B7AC3F1A8
:1079F800640307EE903AFFF750BB4146FFF727BBF9
:107A08000221A048FAF754FB00283FF4DDAA2F8092
:107A1800FFF713B80BF0CAF9C2E49B4AB2F9003079
:107A2800002BB8BF5B42B3F5E17FBFF646A8B2F9B9
:107A38000230002BB8BF5B42B3F5E17FBFF63DA82B
:107A4800924B93ED096AD3ED076A93ED057AD3ED6E
:107A5800037A76EE866A77EE877A76EEA66AB7EECE
:107A6800007A37EE666A77EEA77AB0EEC66AF0EE6D
:107A7800E75AB4EEE56AF1EE10FAB4BFB0EE655A13
:107A8800B0EE465AB5EE405AF1EE10FA40F0DF83F8
:107A98009FED7F7AB4EEE56AF1EE10FA44BF9FEDF0
:107AA8007D6A36EE477AB7EE006AF4EEC66AF1EE02
:107AB80010FAC8BFDFED786AF5EEC07AC8BF36EEB7
:107AC800C77AF1EE10FA48BFB1EE477AF6EE007ABF
:107AD80027EE677ADFED6F7A77EE276ABDEEE66A02
:107AE80016EE103A2033402B40F28A86DFED6B6A9F
:107AF8006B4ADFED6A7AC2ED006AFDEEC76AC2ED35
:107B0800017A16EE903A2033402BC2ED027A49D81A
:107B1800DFED617AB4EEE77AF1EE10FA41F34E80C8
:107B28009FED606ADFED606A01E0B0EE677AB4EE5F
:107B3800E67AF1EE10FA77EE467AF6DC9FED5B7A9C
:107B4800F4EEC77AF1EE10FA41F124809FED556A00
:107B5800DFED576A01E0F0EE477AF4EEE67AF1EEEF
:107B680010FA37EE867AF6D4DFED4A7AB4EEE77A81
:107B7800F1EE10FA40F3C486DFED477A37EEC77AA4
:107B880027EE076ADFED4B5ADFED4B6ADFED4B7AE4
:107B9800E6EE256A67EE065AE6EE267AA5EEA77A9D
:107BA800F0EE477A464BC2ED037A1A6812F40032B7
:107BB80040F09E86434B1046995C0A2902F10C025C
:107BC80000F08E8501301828F6D1FEF776BF27F031
:107BD80040039BB2BB422B803EF468AF3A4B022273
:107BE80014211A700E20FF2259709A701EF09EFD03
:107BF800FEF75CBF2B8823F00407BFB2BB422F807F
:107C08003EF44AAF304B022214211A700E20FF2294
:107C180059709A701EF08AFD2F88FEF73DBF2B49D8
:107C28000E787FE594F89430002B3EF44BAE079B1A
:107C38001B7813F001037EF445AE012284F89430DA
:107C480084F89520FEF73EBE024C012184F88C1082
:107C5800FEF7ABBDE01D00204C5600206C560020FE
:107C68000000C842000080444340002048400020F3
:107C78004440002058570020D023002060E316001D
:107C88006F12833FFC5600200C340020D80E0020D1
:107C9800A7DFA834DB0FC93FDB0F49400000000015
:107CA800B80E0020DB0FC940E4CB1641DB0F49C0FA
:107CB800E4CB16C192E741B99730083C15A82ABE13
:107CC800F85300203C500308205500209C3E00201B
:107CD800012900F0238599F8CC20012303FA0BF33E
:107CE8000BF1010B1343BBF1040F89F8CC300AF1F7
:107CF8000C0A7FF49DACFEF75FBE511D787915F034
:107D0800D3FE00283FF4F9A9B9F1010F40F0268706
:107D180007F10D01B87A15F0C7FE002840F0268754
:107D2800C149F87B15F0C0FE00283FF4F8A9B9F165
:107D3800030F40F01787BD49387D15F0B5FE0028C0
:107D480040F02487BA49787E15F0AEFE00283FF44B
:107D5800F8A9B9F1050F40F01587B649B87F15F0B5
:107D6800A3FE002840F00A87B34997F8230015F0CE
:107D78009BFE00283FF4F8A9B9F1070F40F0FA86F6
:107D8800AE4997F8280015F08FFE002840F0D386FA
:107D9800AB4997F82D0015F087FE00283EF41CAF7C
:107DA800B9F1090F3EF418AFFFF7F2B948F0020332
:107DB80043452B803EF445AEA24B022214211A7093
:107DC8000E20FF2259709A701EF0B0FCB5F80080A2
:107DD800FEF737BE5D2A00F07D825B2A00F0D88569
:107DE8005E2A00F06B86562A00F06C86972A00F00F
:107DF800A686A72A00F05686934D2B889E0740F04A
:107E08001586A2F1B703072B00F29E82DFE813F074
:107E18008E029C029C029C0280029C0272027202E8
:107E2800079B002B3FD05CF8212093454FEA410384
:107E3800FFF4CFAC854A854DD25C05EB030E002AD2
:107E480000F0B180022A47D19EF8012002EB82029D
:107E580002EB820202F2EE2292B2032933DD12B261
:107E6800BAF1000F3FF4BAAC0C9D20F81520B9F117
:107E7800000F03D10F9D022D7FF6B0ACB0F8029031
:107E88000288B0F804E04A449644714A0FFA8EFE1C
:107E980082FB0E526F4DA2EBEE7225F803E012B290
:107EA8004FF001099AE41A464B000A9D4CF82150FC
:107EB80090E4D3B2022B04D9032B7FF40DAD7346A3
:107EC800FCE43B46FAE4012505FA01FE0E9D25EA8D
:107ED8000E0512B20E957DE4E25ABEE75E4A1278AC
:107EE800002A7FF4EBA9B8F1000F3FF4E7A9012CB1
:107EF80040F040819BF82030FFF785B9314657485C
:107F0800FAF7D6F8002800F0D38084F8936013F0CD
:107F1800CDF9FEF7A1BC47F04003BB422B807FF4AC
:107F28005DAEFEF7C3BD47F004039F422B800AD025
:107F3800444B022214211A700E20FF2259709A70A5
:107F48001EF0F4FB2F88464B464AB3F904304649E5
:107F580082FB0302DB17C3EBA2030B80FEF79CBD79
:107F6800424B434A109201221A70424B04931B2140
:107F78003A48FAF79DF800287FF447AC3E4BDFF803
:107F8800FCB008931946DBF80030CA688B609B1A6E
:107F9800C82B00F20185069B1E6806F48056A3E4F0
:107FA8005B78FFF75EB8CAB2022A40F2B483032AAC
:107FB80092D1129A139D079E002D08BF32464CE7B6
:107FC80000220FE0437803EB830303EB830303F200
:107FD800EE239BB20132A24221F8023B00F10200DB
:107FE8003FF482AC15F812301BB1022BEAD00B8893
:107FF800F0E7D3B2032BFAD83B46EBE7B2F5FA7FAA
:10800800FEF656AC94F89230002B7EF451AC079BE8
:108018001B7801210B4084F8921000F0D98312F0EC
:10802800CDFCFEF745BC00BFFD54002002550020E2
:10803800075500200C55002011550020165500202A
:108048001B550020205500205C3400206C3A00208D
:1080580056555555501E002050200020FC56002033
:108068000C340020676666668E2000209D3E002046
:10807800153900207C770020783E0020D456002057
:108088000025FFF7B7B8B2F5FA7FFEF611AC94F801
:108098009230002B7EF40CAC079A1278012184F8F8
:1080A8009210D10700F1428413F000F9FEF700BCEA
:1080B800079BBA4A1B781060D8077EF5D1ABB84B3E
:1080C8001B78002B3EF4F4AB089BDB78002B7EF486
:1080D800EFAB94F893300133DBB2032B84F8933081
:1080E8007EF6E6ABAF4B5B7813B9002D7EF4E0ABC0
:1080F80012F064FCFEF7B0BBAB4AAC491068B4F9A7
:108108009020C66981FB06018911F617701A00F5DF
:10811800FF407F3082423EF792AB891B0A4412B27D
:10812800A4F89020FEF78BBB089BDB78002B7FF42C
:10813800C5A9DFED9F7A9D4938EE678AC9F5FA63CC
:10814800FDEEC87A1BB2CDED047ABDF910201203FA
:1081580081FB0201D217C2EBA11203FB02F343F326
:108168000F334B4407EE903AB8EEE78A87ED038A5F
:10817800FFF7A4B9099D002D3EF496AAFFF716B99A
:108188008C4A059BD588049A1B8BB2F906105A1B9A
:10819800914240F389802B449942B4BF00250125C0
:1081A800FEF793BAC8398A4242DA99F8CC109A781D
:1081B80041FA0BF3DB073FF56FAA524201200D92FB
:1081C8001EF0A8FB7B1E0D9A162B00F25181DFE8EA
:1081D80013F0230237020A025C024B027002F50117
:1081E800E001CB01B601A1014F015C028E017002D2
:1081F800F501E0017A01660152013F0129011501EB
:10820800AB460899DBF80020CB69099D13448B61C4
:10821800002D3EF449AAFFF7C9B815F003FC032165
:1082280040F6B8328BF82010CBF81C20FFF74DB879
:1082380099F8CC30012202FA0BF223EA020308F57E
:10824800FA7289F8CC30CAF80820FFF725BAB4EEDC
:10825800E56AF1EE10FA8CBFB0EE654AB0EE464A18
:10826800C4EE054A9FED542A9FED545ADFED541A87
:10827800DFED542A9FED543ADFED543A9FED544A0E
:10828800A4EE825AE4EEE12AA4EE857AA4EEA23A9C
:10829800B0EE475AB0EE637AA4EE837AA4EE874A2A
:1082A80084EE057AFFF7F6BB0125FEF70EBA00212A
:1082B8004848F9F7FDFE00287FF407AA322384F81E
:1082C8009600A4F89830FFF700BA002A0CBF0120E6
:1082D800022074E7404B002201204049404C0B60CB
:1082E800404B0993404B2270404D0A931EF012FBFD
:1082F800FEF7E3BA3C4A3A4B0A9211463C4A0A60F6
:1083080002225A70374B099315F05CFCFEF7D5BA78
:10831800354A334B0A921146364A0A6000225A708F
:10832800304B099315F04EFCFEF7C7BA2E4A2C4B7A
:108338000A921146304A0A6001225A70294B099361
:1083480015F040FCFEF7B9BA792A00F08C847A2A35
:1083580000F07E849E2A00F073849D2A00F06884D1
:10836800AE2A00F05D84AD2A00F05284EF2A00F0B6
:108378004C84FD2A00F03784FB2A00F09D84FE2AF5
:1083880000F09784F72A00F091847B2A00F0768425
:10839800144B0993144B0A93FEF78FBAA8340020A4
:1083A8009C3E0020E0550020383D0020D34D62104F
:1083B80000007A44D836002099FB243F69A2163E73
:1083C80039094E3DE3B59E3E88FA163E45FE7F3F8D
:1083D800A7DFA834FC560020862D0020603400203A
:1083E800283E002000340020643400205C34002043
:1083F8004C3E0020343E0020403E0020D9F8D000FA
:10840800B64B90F836109B7811446429A8BF6421B4
:1084180021EAE17180F83610002B40F0918414F0C5
:1084280037FC58E4D9F8D000AC4B90F837109B785B
:108438001144FE29A8BFFE2121EAE17180F8371016
:10844800002BECD0162015F0A3FBD9F8D000E6E7F6
:108458000C98A24B41781144B1F5967FA8BF4FF410
:10846800967121EAE17141709B78002B40F061849C
:10847800D9F8D000D3E7D9F8D000984B81781144C7
:10848800C829A8BFC82121EAE17181709B78002B17
:10849800C5D0142015F07CFBD9F8D000BFE7D9F877
:1084A800D0008E4B41781144C829A8BFC82121EAC1
:1084B800E17141709B78002BB1D0132015F068FB57
:1084C800D9F8D000ABE7D9F8D000844B0178114433
:1084D800C829A8BFC82121EAE17101709B78002B47
:1084E8009DD0122015F054FBD9F8D00097E77B4BAC
:1084F8000C989B78417911446429A8BF642121EA2A
:10850800E1714171002BB3D00E2015F041FBD9F871
:10851800D00084E7D9F8D000704B017A9B781144D9
:10852800C829A8BFC82121EAE1710172002B3FF4D4
:1085380076AF0B2015F02CFBD9F8D0006FE7D9F8EF
:10854800D000664BC1799B781144C829A8BFC821BF
:1085580021EAE171C171002B3FF461AF0A2015F0E7
:1085680017FBD9F8D0005AE7D9F8D0005B4B8179CE
:108578009B781144C829A8BFC82121EAE1718171FB
:10858800002B3FF44CAF092015F002FBD9F8D000BE
:1085980045E7D9F8D000514B417993F802E01144EE
:1085A800C829A8BFC82121EAE1714171BEF1000FB5
:1085B80040F0AD83112F7FF461AF30E7D9F8D000D8
:1085C800464B017993F802E01144C829A8BFC82195
:1085D80021EAE1710171BEF1000F40F08E83102F86
:1085E8007FF460AF1BE70C993C4B0F790D93174450
:1085F800642FA8BF642727EAE7770F7115F0E2FA1E
:108608000D9B9B78002B3FF433AF0320394615F0C0
:10861800BFFAD9F8D00002E70C98304B0178114422
:10862800FA29A8BFFA2121EAE17101709B78002B91
:108638003FF41EAF012015F0ABFAD9F8D000EEE6F2
:108648000C98264B817811446429A8BF642121EA3B
:10865800E17181709B78002B3FF40AAF022015F07E
:1086680097FAD9F8D000DAE60C981C4BC1799B78B8
:10867800114481F30801C171002B3FF4F9AE0520C4
:1086880015F086FAD9F8D000C9E60C98134B817911
:1086980093F802E011446429A8BF642121EAE1713A
:1086A8008171BEF1000F40F03C830D2F7FF420AFA5
:1086B800DEE6D9F8D000094BC17893F802E01144FE
:1086C800C829A8BFC82121EAE171C170BEF1000F15
:1086D80040F009830F2F7FF4F9AEA0E6A62E002004
:1086E800B549D1F800E04200BEF1000F08D01718D4
:1086F80003EB87079EF801E07F787745BEF4DDA994
:108708001044AE4FAE4A03EB800300200B60388064
:108718001060FEF7D2B9129AFFF79FBB04999B78B5
:1087280031F91220B2F5617F4FF4966191FBF3F3B2
:10873800C0F2F38040F633019142A8BF11460C2FD6
:10874800A1F5617191FBF3F100F0CB81182F7FF453
:10875800C2AAC9B2C8290B46A8BFC823D9F8D020D5
:10876800D77DD8B2B8423FF4B6AADF1B954BD07577
:1087780048BF0737FF109B780137FFB23BB9002F7E
:108788003FF4A9AA38461EF0C5F8FFF7A4BA182086
:1087980015F0FEF9F3E78C4A8C4B099210461A68DB
:1087A8008B494FF47A73B3FBF2F3C3EB431203EB39
:1087B80082030268DB00A1F8A83053077EF57AA887
:1087C800844B854D0A221A80844B0A93FEF775B8AC
:1087D8008349096811F4003140F09D81814B0846B6
:1087E8005D5C0F2D01F10C016DD001301828F7D117
:1087F800FA3A0023A4F8902084F89230FEF758B88B
:10880800B4EEE77AF1EE10FA40F3DF81DFED765A45
:108818009FED766A01E0F0EE676AF4EEC66AF1EE63
:1088280010FA76EEE57AF6DCDFED716AF4EEE67AB8
:10883800F1EE10FA40F1C681DFED6B5A9FED6D6ADB
:1088480001E0F0EE667AF4EEC67AF1EE10FA77EE11
:10885800A56AF6D4DFED687AF4EEE76AF1EE10FA6D
:1088680040F31481DFED657A77EEE66A66EEA65A84
:108878009FED635A9FED636ADFED637AA5EE856A23
:1088880026EEA55AE5EE867AE5EE276AFFF730B9B7
:108898004949D1F800E04200BEF1000F08D017188E
:1088A80003EB87079EF801E07F787745BEF47FA841
:1088B8000244424F424803EB820300220B603A8095
:1088C8000260FEF774B83C490F68450037B12E18AE
:1088D80003EB86067F787678BE4289D20544374E08
:1088E800374803EB850300250B60358005607FE77B
:1088F800464B1B78032B00F02D810022FFF75AB955
:10890800DFED437AB4EEE77AF1EE10FA44BFDFED1B
:10891800387A37EEC77AFFF733B90C2F00F0F880B2
:10892800182F7FF4D8A900210B4617E7394A2649A2
:1089380013602A4B0991284D0A93FDF7BEBF364AAA
:108948000592FEF7D9BE06F48056FEF7CDBF38EE85
:10895800678A324B32491870FDEEC87AC9F5FA6356
:10896800CDED047ABDF91020120381FB0201D21764
:10897800C2EBA1121BB203FB02F343F30F334B44C8
:1089880007EE903AF8EEE77AC7ED037AFEF7D9B921
:10899800244B01220220A0E4234A069B1E68136888
:1089A80023F004031360089A012306F4805682F822
:1089B8002130FEF799BF00BF0C200020F4200020D2
:1089C800F8200020A62E002000340020084C0020AB
:1089D80090490020E67D00205C34002064340020AB
:1089E800F85300203C500308DB0FC940E4CB164184
:1089F800DB0F49C0E4CB16C1DB0FC93FDB0F494091
:108A080092E741B99730083C15A82ABE24520020A5
:108A1800DB0FC9BFA8340020E87900208C20002093
:108A2800D34D6210D42D0020583400200023BB2AD7
:108A3800149300F02E81B72A00F02781BE2A00F097
:108A48002B81BD2A7FF480AC4FF6FE71BF4AC04827
:108A5800D6890990908933440144D381918116F0D5
:108A68007DFAF8F793FC16F061FAFBF743FA012058
:108A78001DF050FFB4F89030B64A0A92FA3B002233
:108A8800A4F8903084F89220FDF717BFDFEDB27A92
:108A9800F4EEE76AF1EE10FA44BFDFEDB07A77EE54
:108AA800E66AE3E6AE4AAA4B09931378AD4D43F064
:108AB80004031370A74B0A93FDF7FFBEAA4B0222CB
:108AC80003200AE416F04AFAF8F760FC16F02EFACA
:108AD800FBF710FA01201DF01DFF94F88E20FFF718
:108AE80085B9CFB2A14B0E915B78BB423FF4F3A896
:108AF8009F4B0D9338460AF0BFFE0D9B0E999B784D
:108B08001BB1C9B20C2015F043F80137FFB236E6A5
:108B180000273946E6E797490978032900F0BE801F
:108B280019465BE6934B1B78032B7EF415AD1DF0BD
:108B3800DFFDFDF73CBF08231A46FEF72BBB8E4B23
:108B4800834A09924FF4C8721A80824B854D0A9362
:108B5800FDF7B3BE1DF0CCFDFDF7AFBF01231A46EC
:108B6800FEF718BB03231A46FEF714BB02231A4666
:108B7800FEF710BB07231A46FEF70CBB06231A465E
:108B8800FEF708BB05231A46FEF704BB04231A4662
:108B9800FEF700BBB0EE677AFEF7E6BF002D3DF4A6
:108BA800D8AD764C94F88D30002B3DF403AE1DF013
:108BB8009FFD002384F88D30FDF7FCBDF0EE477A69
:108BC800FEF7BCBFF0EE676A44E6F0EE667A2BE685
:108BD8005F4B09935F4B84F8941084F89500614DBE
:108BE8000A93FEF763BD002101200AF06BFDB4F87B
:108BF8009030574A0992963B564AA4F89030002381
:108C08000A9284F89230FDF758BE00210846ECE736
:108C1800FF21002018F04AF894F88E20FFF7A6BB31
:108C28000121002018F042F894F88E20FFF79BBB32
:108C38000021FF2018F03AF894F88E20FFF790BB37
:108C48000021012018F032F894F88E20FFF785BB38
:108C58004B4A3F4B0993137A43F0010313723D4B80
:108C68000A93FDF72ABE464A394B0993137A23F033
:108C780001031372374B0A93FDF71FBE4FF4FA61D5
:108C880002200AF01FFDFFF783BB19464FF6FE735B
:108C9800DCE619460223D9E60221D7E61DF028FDB5
:108CA800B4F99020A4E50B20FDF700BE00210420B4
:108CB8009BE70021032098E70021022095E72F4C2D
:108CC80011F07CFE002384F88D30FDF773BD002B76
:108CD8003FF467AF2B492C4A09684FF47A7000FBC0
:108CE800031313605DE70F200E930D9214F050FFED
:108CF800D9F8D0000E9B0D9AECE410200E930D923B
:108D080014F046FFD9F8D0000E9B0D9A67E41120A5
:108D18000E930D9214F03CFFD9F8D0000E9B0D9ADB
:108D280048E40D200E930D9214F032FF0E9B0D9A1D
:108D3800BBE4152014F02CFFD9F8D000FFF76FBB67
:108D4800172014F025FFFFF793BB00BFC055002084
:108D58000034002064340020DB0FC9BFDB0F49C09A
:108D6800045700205C340020222E0020283E0020DA
:108D7800A62E002024520020E87D0020E01D0020BF
:108D8800C03D0020D4560020A43400202DE9F0472F
:108D9800C74C636820469847002800F0C380C54B3D
:108DA8001B780122042B84F83C2000F0BD80B4F924
:108DB8001610B4F91820B4F91A3021636263A3635A
:108DC800BD4B1B88002B69D0BC4DD4ED0C7AD5ED7A
:108DD800004A95ED050A95ED015A95ED067AD5ED0F
:108DE800035A95ED026AF8EEE76AD5ED047AA4EE27
:108DF800A60AA5EE267A67EEC07AA5EEC07AE6EE58
:108E0800267A85ED057AC5ED067A29F08FF9D4ED35
:108E18000D6AD5ED094A95ED0E0A95ED0A5A95EDBC
:108E28000F7AD5ED0D7AD5ED0C5A95ED0B6A2063C6
:108E3800F8EEE66AA4EEA60AA5EE267A67EEC07AF0
:108E4800A5EEC07AE6EE267A85ED0E7AC5ED0F7AA4
:108E580029F06CF9D4ED0E6AD5ED124A95ED170A92
:108E680095ED135A95ED187AD5ED167AD5ED155A74
:108E780095ED146A6063F8EEE66AA6EEA40AA6EE1B
:108E8800857A67EEC07AA0EE657AE6EE867A85ED99
:108E9800177AC5ED187A29F049F9A063884FA17FA0
:108EA80088481CF079FC3B88002B40F08480864E73
:108EB800D6F8E050854B1B685B0743D4B5F90070C2
:108EC800216B636BA06B824A824E92ED026AD2EDEF
:108ED800006AD2ED015AC91B2163B5F90270DB1B88
:108EE8006363B5F904703568C01B07EE900AB8EEE5
:108EF800E75A07EE901AB8EEE77A07EE903AF8EEDE
:108F0800E77A36EE056A36EE877A77EEA57A013586
:108F1800A06382ED026A82ED007AC2ED017A3560C3
:108F2800BDE8F087BDE8F0876B4BB4F91600B4F9DB
:108F38001810B4F91A2018802063598061639A8048
:108F4800A2633DE7B6F89820322A00F08880002A0C
:108F580066D196F89530002BB0D06048D6F8FC2042
:108F68005F4980FB0273D217C2EB23122A80D6F81E
:108F7800002180FB0273D217C2EB23126A80D6F855
:108F88000431A78A80FB0302DB17C3EB2213DB1B28
:108F9800AB800023CB6086F8953015F0DFFFF8F73B
:108FA800F5F915F0C3FFFAF7A5FF01201DF0B2FC93
:108FB800D6F8E05082E7444E226BD6F8E050B3F57D
:108FC800C87F4FF0000323632B80398818BFD6F879
:108FD800E400B7F8008008BF0020B1F5C87F18BFCB
:108FE800D6F8E830616B02440B440020B8F5C87F1E
:108FF8006063C6F8E420C6F8E830688052D0D4F838
:1090080038E0D6F8EC10A0637144B8F1010FA880DD
:10901800C6F8EC1068D008F1FF38A7F8008049E7D7
:10902800D6F8FC00236B00210344C6F8FC3021630A
:109038002980D6F80001636B61630344C6F80031E8
:109048006980A36BD6F80401A1630344012AC6F81A
:109058000431A98075D0013AA6F8982079E72B88C1
:1090680020491F48276BA6F8F0300023B5F802E026
:10907800B5F804C0C0684B608B602363C6F8FC7009
:109088002B80616BC6F8001163636B80A16BC6F817
:109098000411A363A6F8F2E0A6F8F4C0C6F8F80035
:1090A800AB80D8E7A36BC6F8EC30A063A880B2E722
:1090B800143400200C320020EC430020F043002040
:1090C800E87D002044340020E01D0020184C0020DA
:1090D800E8340020E4340020103200201F85EB51D2
:1090E800C0550020DC1E0020DFF804C1DFF8F0E0E6
:1090F800C8328CFB02A9C833D217C2EBE9128CFB29
:1091080003A9DB17C3EBE913C8316B802A808CFBFA
:10911800013CA28ACB17C3EBEC139B1AAB80CEF8A9
:109128000C0015F01BFFF8F731F915F0FFFEFAF700
:10913800E1FE40461DF0EEFBB7F80080D6F8E0509F
:1091480069E7254B86F89A101B6886F8942013F473
:10915800003334D119462148475C0B2F01F10C012B
:1091680010D00133182BF7D1B6F8F0101C4B29801A
:10917800B6F8F270B6F8F400D6F8F8106F80A88048
:10918800D96068E7174FD7F800C05900BCF1000F45
:1091980009D001EB030E00EB8E0E9CF801C09EF87F
:1091A80001E0E645E0D20B44DFF848E00E4900EB69
:1091B800830000233860AEF800300B60D4E70B4B17
:1091C8001B78032B01D00B46C5E71DF091FAD6F8A2
:1091D800E050B6F89820C7E7F85300203C50030841
:1091E800C05500200C200020F82000202452002028
:1091F8001F85EB51F42000202DE9F0478C4B1B789C
:10920800DB07074644D58B4B8B4D1C788B4E012CC6
:1092180059D01CD3022C07D189498A4A0988128857
:10922800914201D901241C70EB7AE3B12B89D3B1A7
:10923800854B1B78BBB10AF041FB002800F09B80EE
:109248002B7B83422CBF0121002131700CE07C492B
:109258007E4A098810886A7B801A8842E2DAEB7AAB
:109268000024002BE2D131782A79632A06D8022C0F
:10927800774E00F0BA803378002B5DD1754AAB7A0F
:109288008C4238BF0C461470002B4CD1BDE8F087D7
:109298006B4B694D19885B88E878CB1A83EAE372CF
:1092A8008142A2EBE3721DD32B788B421AD3614B18
:1092B8001C78E01E012861D96749097802294FD036
:1092C800012C5E4EA5D15F4A5D491288687B0988EA
:1092D800121A914239DD5D4A12888A42A4D20024CA
:1092E8001C70A1E7B1EB400FE1DC524B1C78E11E8A
:1092F800012940F29480022ADEDC57494F4E087853
:10930800DFF84481DFF844C1DFF838E100210324A5
:10931800022834701C7088F80010ACF80010AEF801
:10932800001081D11FE0012C71D0022C0BD1072035
:10933800BDE8F0471DF0FAB97068381A474B9842F3
:1093480058DD72709AE7BDE8F08702241C706BE75D
:10935800022AD2DD4049097802294FF0040464D179
:109368003949364E09783E48022ACCBF00220122EC
:10937800C28081804BE70221317075E7022A9BDCAD
:1093880095F800C091FBFCFC0CF1010CBCF1080F36
:10939800DFF8B4A0304EA87895F801E096F8008080
:1093A8002A4CDFF8A090254EA8BF4FF0080C8AF889
:1093B80000C01FFA8CFA10FB0AF01EFB0AFE80B2EE
:1093C800DFF88CA02080A9F800E000244FF0640E9C
:1093D800B8F1020F34701C70CAF804408AF801E032
:1093E8007FF439AF0FFA8CF1BDE73078A0B90123CB
:1093F80077603370C2F164021A4B00FB02F083FB02
:109408000023C017A0EBA3506430707036E7082023
:10941800BDE8F0471DF08AB97368F81A8EE7032C87
:1094280096D10D49097802299AD0044EFCE600BF6E
:10943800EF3A002060240020F03300207024002040
:109448001C320020642400203232002062240020D4
:1094580068240020245200200C3200207F969800B7
:10946800103200206BCA5F6B2DE9F04F2DED0E8B8B
:10947800DFF8F4B093B0DBF8042004905846904726
:10948800002800F08E82BBF8A87000218BF85110DC
:10949800002F6DD1BBF93A00DBF82450DBF8281017
:1094A800BBF93860DBF82040BBF93C20DFF8BCA0F2
:1094B800401B521A341BCBF830009BF85210CBF8E3
:1094C8002C400BF12C00CBF834201CF065F9DAF8AD
:1094D8000020940041F15087DBED0C5A1F4CDBED66
:1094E8000B7A1F4994ED406AD4ED416A94ED427AB3
:1094F800D4F80C2109681B4B0293B8EEE58ADBED22
:109508000D5AF8EEE77AF8EEE58A013277EE867AB8
:1095180038EE268A78EE878A8A42C4ED407A84ED4E
:10952800418AC4ED428AC4F80C2101F0568393F8AD
:1095380000E0BEF1140F03F001800023D4F81451A9
:109548000393062D01F2A384DFE815F036172317DD
:109558008D156A160E0CD316EF1500BFE81E0020F5
:10956800B44000200C32002090490020184C002004
:10957800DE4BDF481A6805934FF47A75B5FBF2F2B3
:10958800C2EB421502EB8502D500DA4BDFF8C8833F
:1095980044780293ADB2AF421E78B8F9060003F0E2
:1095A800E880DBF87C30BBF93810DBF8602003F189
:1095B800010E07EE901A0A44BEF1010FCBF87CE0C9
:1095C800CBF86020F8EEE77A03F0E080DBED1B5A79
:1095D800DBED1D6A07EE10EA37EEE56AB8EEC75A0A
:1095E800012F86EE057A37EE257A77EEC77A8BED6E
:1095F8001C7AE7EE866A8BED1B7AF0EE667ACBED85
:109608001E6ACBED1D6A03F05384DBF89030BBF97A
:109618003A10DBF8642003F1010E07EE901A0A44B1
:10962800BEF1010FCBF890E0CBF86420F8EEE77AB2
:1096380003F0C780DBED205ADBED226A07EE10EA63
:1096480037EEE56AB8EEC75A012F86EE057A37EE8F
:10965800257A77EEC77A8BED217AE7EE866A8BED6D
:10966800207AF0EE667ACBED236ACBED226A03F01E
:109678004784DBF8A430BBF93C10DBF8682003F121
:10968800010E07EE901A0A44BEF1010FCBF8A4E0D0
:10969800CBF86820F8EEE77A03F0AE80DBED255AC8
:1096A800DBED276A07EE10EA37EEE56AB8EEC75A2F
:1096B800012F86EE057A37EE257A77EEC77A8BED9D
:1096C800267AE6EE276A8BED257AF0EE667ACBED00
:1096D800286ACBED276A03F0DE83874CA8F80600DA
:1096E800BBF8A820029B013A1E78ABF8A820059980
:1096F8000022072E4A608A60CA6040F05981FBF751
:10970800DFFD029BDFF850821E78049BC01A94F894
:109718002831A8F800000693002B40F04F81744AC6
:109728005279002A01F08681744A1278013AD2B23D
:10973800072E84F8282102F05E8200230793704BDD
:10974800D4F83421D3F800A0684B0593049B9FED0F
:109758006D6AD4ED4C9A6C49C4F834319A1A07EE04
:10976800902AF8EE677AB7EE007AC6EE278A0025C7
:10977800664BDFF8E891DFF8E881654F03932E46E2
:10978800D1ED006A94ED4BDA9FED629ADFED62AAA3
:109798009FED62CA9FED62AADFED62BA9FED62BAE1
:1097A80077EE69CA6CEEA6CAF4EEC7CAF1EE10FAF3
:1097B80088BFF0EE47CA5D4B99ED008A2B44D3ED84
:1097C800007AF5EE407AF1EE10FA17D0584B2B4498
:1097D80093ED007A78EE476AB0EEE66AF4EEC67A60
:1097E800F1EE10FA08D5F5EEC06AF1EE10FACCBF2A
:1097F80037EE878A37EE678A83ED008A4D4B1A88E1
:10980800910739D0022E37D09AF82E104A4B07EE1E
:10981800901A2B4493ED007A4B42F8EEE76A07EE74
:10982800903A26EE877AF8EEE77AB4EEE77AF1EE28
:1098380010FA0AD407EE901AF8EE677AF4EEC77AAF
:10984800F1EE10FA88BFF0EE477A3C4B3C4903EB47
:10985800460331F91600B3F90C30C31A07EE103A73
:10986800B8EEC77AD307E7EE497A41F17F80354BE6
:1098780093ED008A27EE888A059B94F868212B448B
:1098880093ED01EA78EE4EDA002A00F0F7802E4BCD
:10989800D4F86C2104991B688A1A9A4240F3EE8026
:1098A8009AF84830022B02F0F581022E04F009855F
:1098B800264B1B68980700F19780254B87ED00CA57
:1098C8001B689342C0F2CA80F7EE007AF4EEE79A7A
:1098D800F1EE10FA40F1D28005991E4BD1ED017AD4
:1098E80093ED007AF0EEE77A3CE000BF084C0020E8
:1098F8007C4900200C320020E81E0020B4550020CE
:1099080060340020002474492436002008570020C1
:1099180014570020CDCCCC3DAE47813F000000005D
:109928000000C84200003443610BB63B18360020E3
:109938002C2000205C34002038200020C055002056
:109948000C340020003600202C3600200034002083
:109958002836002034360020103200202020002035
:1099680020570020F4EEC77AF1EE10FA40F1868015
:10997800D1ED027AF0EEE77AB4EEE77AF1EE10FA7A
:109988007CDDD1ED037AF0EEE77AB4EEE77AF1EE1A
:1099980010FA73DD0F4B1B6899075FD50E490F4B03
:1099A80043E00F4B0F4C1E780293072E3FF4A7AEEF
:1099B80094F828310693002B3FF4B1AE013B84F8AC
:1099C8002831012E01F0B58213B0BDEC0E8BBDE835
:1099D800F08F00BF003400200C340020C055002058
:1099E8000C320020E81E0020D34BD449DFF8C8E32E
:1099F80031F916C09EED008ADFF8C0E387ED00CA92
:109A080003EB460028EE098AB0F90C00A0EB0C0025
:109A180007EE900AF8EEE77ADEF8000027EE888A6B
:109A2800904278EE4EDABFF64FAFB3F90C20B1F999
:109A380000E0C348AEEB020E00688EEAEE72A2EBBD
:109A4800EE7282421ADAB3F90E30B1F90220D21A54
:109A580082EAE273A3EBE27398420FDDB94B1A88EE
:109A6800002384F86831002A43F0E085B64AB74BF2
:109A78001178186881F00101FCF78CFAB44B2B447B
:109A880093ED000A039B2DEE000A022E20EE2D0A0C
:109A9800A3EC010A039304F03C84AE4BD7ED006AB3
:109AA80093ED007AAC4BD3ED007AAC4B93ED006AA2
:109AB800AB4B67EE277A2B4427EEAC7AD3ED007ACE
:109AC80067EE277AF0EE665AEDEEA75AB1EE467ABF
:109AD800B4EEE57AF1EE10FA08DCB4EEE56AF1EEE0
:109AE80010FA8CBFB0EE657AB0EE467A94ED4C6A07
:109AF800F7EE007AB4EEE76AF1EE10FAACBF012394
:109B0800002343B1F0EEE66AF0EEC77AF4EEE67AA7
:109B1800F1EE10FA01D587ED007A022E04F02B83BE
:109B2800904A914B52F826001B68B0EE4E0A9847AF
:109B38008E4A8F4B52F826001B6898479AF83730A0
:109B480023B18C4B1B88002B00F07787B0EE4C8A32
:109B5800894B38EE400A2B4493ED008A83ED000AC6
:109B68009AF8483030EE480A20EE288A002B33D085
:109B7800824B1B7813F0010300F0C386F7EE007ADE
:109B8800F4EEE79AF1EE10FA94F86831C1F27285B2
:109B9800002B00F0F787D4F86C31049AD31A784A6E
:109BA80012689A4218DD774BD3ED007AF0EEEDDAC1
:109BB800F4EEE7DAF1EE10FA42F17D80614B1A8893
:109BC800002384F86831002A00F0A7866E494A69A4
:109BD80012B10A6813604B746C4B94F878212B44CB
:109BE80093ED000A2DEE000A20EE088A88ED008A1F
:109BF80032B9039B87ED00CA03ED01CA88ED00CA9C
:109C08000136032E09F1040908F1040807F10407D5
:109C180005F104057FF4CFAD029B1A78072A01F0FD
:109C28003F85012A01F0D4870023039394F880210B
:109C3800002A41F08B81DFF888A1554BDAF8002023
:109C48001968D20491F82C0000F11287DFF874919A
:109C5800504AB9F81A3092ED006A4F4A4F4ED2ED89
:109C6800005AD6ED036A4E4A84ED646A07EE103A4C
:109C78004C4B92ED005AD3ED007AD3ED013AD3ED77
:109C8800024A84ED626AB8EEC77A35EEC64A012206
:109C980036EEC77A84ED614AC4ED655A84F8982196
:109CA800C7EE055A0A8D534206EE103A3E4BDFEDD9
:109CB8003F6A93ED005A3E4B93ED004AB7EE007AA7
:109CC800F4EEC75A35EE045AF1EE10FA88BFF0EEFA
:109CD800475A35EE275AB8EEC66AF4EEE65AF1EE60
:109CE80010FA07EE902AB4EEC65AB8BFF0EE665ADC
:109CF800F1EE10FAC4ED685AB8EE677A01F13883CC
:109D0800B4EEC75AF1EE10FA88BFB0EE475A264BA8
:109D1800DFED286AD3ED017A254B93ED014A77EE02
:109D2800847A25EE265A77EEA37AB4EEE76AF1EE46
:109D380010FA52DC48E000BFC05500200C34002067
:109D480030360020AC560020AE560020B056002019
:109D5800D4350020103500200400002048360020AB
:109D6800E035002018350020143500206C3500201F
:109D7800683500205C34002058200020EF3A00208D
:109D88002C36002038360020B4560020EC35002050
:109D980060340020885500208C5500203432002083
:109DA800E03600201457002008570020000000006B
:109DB800205700206F12833A0036002028360020F2
:109DC800184C0020E8790020B4EEE77AF1EE10FA9A
:109DD8008CBFB0EE676AB0EE476AED4B4A8DD3EDA3
:109DE800027A9FEDEC7A534204EE103A74EEA77AA9
:109DF800B8EEC44A26EE076AF4EEC47AF1EE10FA19
:109E08000AD407EE102AB8EE474AB4EEE74AF1EE54
:109E180010FA88BFB0EE674ADF4ADFEDDE7A527883
:109E280024EE274A0AB9B1EE444A002841F0748664
:109E3800B7EE003AD94E3278002A02F0A586D84902
:109E4800DFEDD87AD1ED024AD1ED016A91ED037ABE
:109E580066EE244AE5EE264AE4EE074A63EE244A13
:109E6800F4EEE74AF1EE10FAB4BFF0EE673AF0EE1E
:109E7800643A98BFF0EE647A012ACDED0A4A02F0FE
:109E8800D68691ED067AD1ED052AD1ED076A26EE40
:109E9800077AA5EE227AA4EE267A23EE077AB4EEA4
:109EA800E77AF1EE10FAB4EEE37A8CBFF0EE676A67
:109EB800F0EE476AF1EE10FA88BFF0EE676AB4BFB9
:109EC800F0EE637AF0EE477A022A8DED0B7A00F015
:109ED800DE8091ED0A7AD1ED092AD1ED0B3A26EE12
:109EE800077AA5EE227AA4EE237A23EE077AB4EE57
:109EF800E67AF1EE10FAB4EEE77A8CBFF0EE663A45
:109F0800F0EE473AF1EE10FA98BFF0EE636AA8BF98
:109F1800F0EE477A032A8DED0C7A00F0B88091EDC7
:109F28000E7AD1ED0D2AD1ED0F3A26EE077AA5EE7D
:109F3800227AA4EE237A23EE077AB4EEE67AF1EEDB
:109F480010FAB4EEE77A8CBFF0EE663AF0EE473AD4
:109F5800F1EE10FA98BFF0EE636AA8BFF0EE477A08
:109F6800042A8DED0D7A00F09280D1ED123AD1EDF0
:109F7800112A91ED137A66EE233AE5EE223AE4EEE1
:109F8800073A63EE233AF4EEE63AF1EE10FAF4EE0D
:109F9800E73A8CBFB0EE667AB0EE637AF1EE10FA6B
:109FA80098BFF0EE476AA8BFF0EE637A052ACDEDB8
:109FB8000E3A6CD0D1ED163AD1ED152A91ED177AFB
:109FC80066EE233AE5EE223AE4EE073A63EE233AE8
:109FD800F4EEE63AF1EE10FAF4EEE73A8CBFB0EEA2
:109FE800667AB0EE637AF1EE10FA98BFF0EE476A3F
:109FF800A8BFF0EE637A062ACDED0F3A47D0D1ED2F
:10A008001A3AD1ED192A91ED1B7A66EE233AE5EE5C
:10A01800223AE4EE073A63EE233AF4EEE63AF1EE3A
:10A0280010FAF4EEE73A8CBFB0EE667AB0EE637AD7
:10A03800F1EE10FA98BFF0EE476AA8BFF0EE637A27
:10A04800072ACDED103A22D091ED1E7AD1ED1D2AC6
:10A05800D1ED1F3A26EE077AA5EE227AA3EE847A8E
:10A0680027EE037AB4EEE67AF1EE10FAB4EEE77A68
:10A078008CBFB0EE666AB0EE476AF1EE10FA8DED6D
:10A08800117A98BFF0EE466AA8BFF0EE477A77EEED
:10A09800E67AF7EE006AF4EEE67AF1EE10FAC4ED2D
:10A0A8004C7A43F3FA8586EEA77A022ADDED0B7A1D
:10A0B80067EE244A67EE877ACDED0A4ACDED0B7A32
:10A0C8002DD0DDED0C7A67EE877A032ACDED0C7A78
:10A0D80025D0DDED0D7A67EE877A042ACDED0D7A6D
:10A0E8001DD0DDED0E7A67EE877A052ACDED0E7A62
:10A0F80015D0DDED0F7A67EE877A062ACDED0F7A57
:10A108000DD0DDED107A67EE877A072ACDED107A4B
:10A1180005D0DDED117A27EE877A8DED117A224987
:10A12800096811F0805801F05882F6EE005AC4ED23
:10A13800685A002A02F04B851C4B94ED656A1C494D
:10A148001C4F1D78DFF874E094F9983194ED645A47
:10A15800B7F90670C878DAF80010DEED004A0597FE
:10A16800BDEEC66A07EE103AB9F81A70124B079797
:10A1780016EE10EABDEEC56A05F0010C01F4805731
:10A1880001F0100501F4800108911B7818E000BF68
:10A19800085700206F12833A10590020BA31002066
:10A1A8005036002000000000FC560020EF3A002046
:10A1B800783E00207C7700203C4E00204C36002062
:10A1C800D4ED616AD4ED627AB8EEC77A16EE101A49
:10A1D800002840F03587002D41F06D83D54D9DED69
:10A1E8000A5A95ED006AD44825EE866AA5EE076AF4
:10A1F800B0EE675AA6EE265ABDEEC56A16EE108A6C
:10A2080016EE107AF045A8BF77464145C8BF0F46FD
:10A2180006EE107AB8EEC66A012A80ED006A00F0F0
:10A22800DC8095ED046A9DED0B5A25EE866AA5EE55
:10A23800076AB0EE675AA6EE265ABDEEC56A16EE54
:10A24800108A16EE107AF045A8BF77464145C8BF78
:10A258000F4606EE107AB8EEC66A022A80ED016A49
:10A2680000F0BB8095ED086A9DED0C5A25EE866AD4
:10A27800A5EE076AB0EE675AA6EE265ABDEEC56A85
:10A2880016EE108A16EE107AF045A8BF77464145BB
:10A29800C8BF0F4606EE107AB8EEC66A032A80EDEC
:10A2A800026A00F09A8095ED0C6A9DED0D5A25EE34
:10A2B800866AA5EE076AB0EE675AA6EE265ABDEE84
:10A2C800C56A16EE108A16EE107AF045A8BF7746D2
:10A2D8004145C8BF0F4606EE107AB8EEC66A042A92
:10A2E80080ED036A79D095ED106A9DED0E5A25EE42
:10A2F800866AA5EE076AB0EE675AA6EE265ABDEE44
:10A30800C56A16EE108A16EE107AF045A8BF774691
:10A318004145C8BF0F4606EE107AB8EEC66A052A50
:10A3280080ED046A59D095ED146A9DED0F5A25EE1B
:10A33800866AA5EE076AB0EE675AA6EE265ABDEE03
:10A34800C56A16EE108A16EE107AF045A8BF774651
:10A358004145C8BF0F4606EE107AB8EEC66A062A0F
:10A3680080ED056A39D095ED186A9DED105A25EEF5
:10A37800866AA5EE076AB0EE675AA6EE265ABDEEC3
:10A38800C56A16EE108A16EE107AF045A8BF774611
:10A398004145C8BF0F4606EE107AB8EEC66A072ACE
:10A3A80080ED066A19D095ED1C6A9DED115A65EE8F
:10A3B800865AE7EE055AE6EEA57AFDEEE77A17EE3D
:10A3C800905AAE45A8BFAE46A942D8BF714607EE1F
:10A3D800901AF8EEE77AC0ED077ABCF1000F00F0AA
:10A3E8003C87564A1268002A40F04487544A12783B
:10A3F80092B1307868B1504FDFF868810025E8B233
:10A40800D8F80030B7EC010A984730780135854212
:10A41800F5DB4C4A12689047029B1A78072A01F02C
:10A428002E810025DAF80020560500F1BD87464B3D
:10A438001B68180700F1C687444B1B78BBB1444A18
:10A44800B9F81A30B2F906209A4210DC414B1B7851
:10A45800012B01F0E583192B01F0E2830E2B06D0C6
:10A46800082B04D03C4E0023B360C4F8403194F864
:10A47800AA6126B1394B1B889F0741F0938394F852
:10A48800B021002A40F0F98799F81E70002F00F0DB
:10A498003184022F01F07583032F41F06E8399F800
:10A4A8002030C3EB431103EB8101C90089B299F84D
:10A4B8001F300233DBB2002A00F08485002900F047
:10A4C800818527480768B1FBF7F10FB2A4F8E0715E
:10A4D800002B03F0BB8007EE907AF8EEE77AF7EEF0
:10A4E800006A86EEA77A1C4E012BD4ED7D6AD6ED64
:10A4F800007A77EEE67A67EE877AC4ED797A3DD00E
:10A50800D6ED017AD4ED7E6A77EEE67A022B67EE15
:10A51800877AC4ED7A7A31D0D6ED027AD4ED7F6AA3
:10A5280077EEE67A032B67EE877AC4ED7B7A25D03F
:10A538001AE000BF503600206C570020682D00201C
:10A5480064510020384E002000340020681B002091
:10A558007C77002010590020343200205C34002021
:10A56800F8580020304E0020D6ED037AD4ED806AEA
:10A5780077EEE67A67EE877AC4ED7C7A02990978F5
:10A58800092903F09F81002F40F3BA839BB394ED10
:10A598007D7AD4ED797A77EE877A012BC4ED7D7ACE
:10A5A800C6ED007A21D094ED7E7AD4ED7A7A77EEF2
:10A5B800877A022BC4ED7E7AC6ED017A15D094ED28
:10A5C8007F7AD4ED7B7A77EE877A032BC4ED7F7A96
:10A5D800C6ED027A09D0D4ED807A94ED7C7A77EED4
:10A5E800877AC4ED807AC6ED037A013B022BB8BFA7
:10A5F8000223DBB20693069B002A18BF02239E465D
:10A60800CB4BDFEDCC6A1A68029B917818781378E7
:10A6180007EE903AF8EEE77AB0EE007A67EEA67A9F
:10A62800F4EEC77AF1EE10FA40F38D86DFEDC26AD8
:10A6380037EEC77AB0EE676AA7EE266AF0EE466A8A
:10A6480096ED007A9FEDBD6A27EE066AF0EEC65ACF
:10A6580084ED546AC4ED575A99B107EE101AB8EE52
:10A66800C75A9FEDB47A66EE064A25EE075AB7EE4A
:10A67800007A37EE457A64EEA54AA4EE857A26EE8E
:10A68800076A9FEDAF7A537926EE877A27EE067A26
:10A69800CBB1DFEDA86A9FEDAB6A65EEA65A06EE70
:10A6A800903AF8EEE66A66EEA56AF4EEC66AF1EE4E
:10A6B80010FA01F31B82F7EE005A75EEE66A85EE92
:10A6C800A66A27EE067A0C289FED9F8ADFED9F6A1F
:10A6D80000F08A87B4EEC87AF1EE10FA98BFB0EEAF
:10A6E800478AB4EEE68AF1EE10FAB8BFB0EE668A91
:10A6F80084ED4E8ABEF1000F00F0DD80B0EE007AE6
:10A70800F4EEC77AF1EE10FA05DD37EEC77ADFED21
:10A718008A6AE7EE267A96ED017ADFED886A27EEF7
:10A72800267AF0EEC75A84ED557AC4ED585A99B195
:10A7380006EE901A9FED7F6AF8EEE66A27EE075A52
:10A7480066EE866AB7EE006A36EE666A25EE255A28
:10A75800A5EE266A27EE067ADFED796A937967EE29
:10A76800A67A67EE877AABB107EE103AB8EEC77AE9
:10A778009FED706ADFED736A27EE257A27EE067A79
:10A78800B4EEE67AF1EE10FA41F3A281DFED706AD9
:10A7980067EEA67A0C2800F04587DFED6B6A9FED1F
:10A7A8006B7AF4EEE67AF1EE10FA88BFF0EE667A8C
:10A7B800F4EEC77AF1EE10FAB8BFF0EE477ABEF1C0
:10A7C800010FC4ED4F7A76DD5378DFED5A6A07EE54
:10A7D800903AF8EEE77AB0EE007A67EEA67A537A06
:10A7E800F4EEC77AF1EE10FA05DD37EEC77ADFED41
:10A7F800526AE7EE267A96ED027ADFED506A27EE86
:10A80800267AF0EEC75A84ED567AC4ED595A9BB1B0
:10A8180006EE903A9FED476AF8EEE66A27EE075A89
:10A8280066EE866AB7EE006A36EE666A25EE255A47
:10A83800A5EE266A27EE067ADFED416AD37967EE40
:10A84800A67A67EE877AFBB107EE103AB8EEC77AB8
:10A858009FED386ADFED3B6A27EE257A27EE067A08
:10A86800B4EEE67AF1EE10FA01F32E81B5EEC07A75
:10A87800F1EE10FA02F17083B7EE006A36EE477A0D
:10A88800C6EE076A67EEA67A0C2800F0EB86DFEDC5
:10A898002E6A9FED2E7AF4EEE67AF1EE10FA88BF72
:10A8A800F0EE667AF4EEC77AF1EE10FAB8BFF0EE81
:10A8B800477AC4ED507A092800F0828699F8216019
:10A8C800002E40F03786002384F8B03120F060FC79
:10A8D800002840F051831F4B1B7823B91E4B9B78EF
:10A8E800002B41F05A81029B1E78072E7FF469A83D
:10A8F800FAF7E6FC194B029A401B1678D880FFF746
:10A9080060B894F86821002A3FF466A9144A84F8CC
:10A9180068311288002A7FF459A9124A124B11781B
:10A92800186881F00101FBF735FBFFF755B900BF47
:10A93800643400200AD7233CD7A368416F12033B35
:10A9480000004843A4707D3F00C0F94400C0F9C42A
:10A958000000C842593B0020A62E002010320020DB
:10A96800AC560020AE560020B056002094ED577A21
:10A97800B1F90000D4ED586AB1F902E0E24AF4EE08
:10A98800C76A80EAE0738EEAEE71A3EBE073F1EE3A
:10A9980010FAA1EBEE71B8BFF0EE476A8B42B8BF70
:10A9A8000B4607EE103A1378B8EEC77A27EE097A05
:10A9B800002B40F0B880D54B93ED006AB4EEEA6AFC
:10A9C800F1EE10FA41F1E480F7EE005A75EEC65A3E
:10A9D8003BEEC77A65EE8B5ACD4BA7EE256A93ED11
:10A9E800007A26EE076AB5EEC06AF1EE10FA40F278
:10A9F800F085CAEE065AB7EE007AB0EE476AA6EEC0
:10AA0800E56AF0EE466AF4EEC76AF1EE10FA88BF1E
:10AA1800F0EE476AF5EEC06AF1EE10FAB8BFF0EE54
:10AA28004C6ABC4B93ED007A67EE877AA7EEA68A4C
:10AA3800FEF722BF0122FEF77BBEB74BB74A2B4475
:10AA480093ED007AD2ED007AB54B67EE277AF7EEF0
:10AA5800006AF4EEE67AF1EE10FA93ED007A88BF18
:10AA6800F0EE667A67EE877A27EE888AFFF770B885
:10AA7800AC4BDFF8EC921A78AB4ED3075CBFB9F851
:10AA88001820A4F88C21A94AD6ED037A128807EE7B
:10AA9800102AB8EEC77AF4EEC77AF1EE10FA42F24D
:10AAA8004380A34D2B8807EE103AB8EEC77AF4EE30
:10AAB800C77AF1EE10FAC1F2BF809E4A9E4D92ED20
:10AAC800006AD5ED006A94F99821C4ED646A76EEBF
:10AAD800665A012AC4ED626AC4ED615A84ED656A5A
:10AAE80001F04186049BC4F89C31002537EEC77AF3
:10AAF800FCEEE77A914E84ED687A17EE902AA4F876
:10AB08008C21012296ED005A84F898218C4A9542AE
:10AB180041F2F7878B4BD3ED007AD3ED013AD3EDB1
:10AB2800024AFFF7BDB87A4B93ED005AB5EEC05A0A
:10AB3800F1EE10FA40F34D85834BD3ED004AF5EE64
:10AB4800C04AF1EE10FA40F3448534EEC77A66EE57
:10AB5800CA5A87EE246AC5EE856AB7EE007AB4EE63
:10AB6800C76AF1EE10FA88BFB0EE476AB5EEC06A60
:10AB7800F1EE10FA76EE876AB8BFB0EE4C6A66EE70
:10AB8800266A40E7714AD2ED007AB0EEC87AB4EE90
:10AB9800E77AF1EE10FA7FF71FA86D4AD2ED007A36
:10ABA800B0EEED7AB4EEE77AF1EE10FA7FF714A87A
:10ABB800684AD9ED007A92ED007AF0EEE77AF4EE81
:10ABC800C77AF1EE10FA7FF507A801220499C4F8B4
:10ABD8006C1184F86821FEF7E2BF07EE102A197895
:10ABE800DFF88081C4F80C71B8EEC77AF7EE006A16
:10ABF800132986EE879AB8F90400B4F810619BED22
:10AC0800070A01F03C85544A544992ED001AD2EDE6
:10AC1800053A92ED122A92ED173AD2ED091AD2EDC1
:10AC28000E4A92ED016A92ED064A92ED0A7AD2ED49
:10AC38000F5AD2ED132AD2ED186A92ED045AD2EDCA
:10AC4800030A67EE897A69EE288A29EE088AE1EE16
:10AC5800273A01EB86070025A2EE283AC4F80051EE
:10AC6800C4F80451E1EE884AA6EE274AE7EE085AEE
:10AC780092ED167A92ED0D6A92ED021AD2ED0C1A47
:10AC8800C7ED003AE2EEA86A25EE635A27EE437A4A
:10AC980092ED0B2AD2ED152AC7ED204AA0EEE34A21
:10ACA80026EE646AD2ED143A82ED054AA1EE275ADF
:10ACB800F0EE477AE1EEE45AA2EE086AE2EEC36AE1
:10ACC800E3EEA87A82ED065AC2ED0E5A82ED0F6ABB
:10ACD80087ED403AC2ED176AC2ED187AC4F80851F8
:10ACE800721C02F01F02A4F81021A8F80400029BAD
:10ACF800FEF71DBCA4F8E071002A3FF4E7AD0A4E48
:10AD08004FF0020E7CE400BF0C3600201436002001
:10AD1800083600200436002044200020FC3500209E
:10AD2800F8350020EF3A002034320020E4360020C5
:10AD3800E63600208C550020D0360020EC36002066
:10AD48008FD0030014570020103600203C36002016
:10AD5800383600204036002044430020D8400020E8
:10AD6800E8790020103200209C4A1178D4F8187134
:10AD78009B4B9FED9C7AFE009A1982ED007A002980
:10AD880079D09948B0EE476AF0EE476A0022F0ECB5
:10AD9800017A013267EEA77A05EE902AB4EEE77AD7
:10ADA800F1EE10FAF8EEE55AB8BFB0EE677A8A42CB
:10ADB80076EEA76AA7EEA56AE9D1F5EEC06A9A19F8
:10ADC800F1EE10FA82ED007A55DDC6EE265A874A72
:10ADD80087490988F7EE007A75EEE75AD2ED007ACE
:10ADE80065EEA77AFDEEE77A17EE902A812A42F3FC
:10ADF800C6808A42A8BF0A4607EE902AF8EEE77A8C
:10AE08007C4AF01902EB800292ED057AD2ED003A05
:10AE180092ED066A92ED014AD2ED046AD2ED034A38
:10AE280092ED025AA3EEA77AA4EE276A66EEC76AE5
:10AE3800A7EE646ABDEEC77AE5EE276A17EE100A38
:10AE4800812882ED056AC2ED066A42F39580814247
:10AE5800A8BF014607EE901AF8EEE77AFCEEE77A0B
:10AE6800CDED057ABDF8142099198A801FB9BEF175
:10AE7800130F02F00487BEF1150F41F046811E44FE
:10AE8800DFF89081B28828F81720D4F814515A4A6C
:10AE9800013582FB05325119EA17C2EBA102C2EB58
:10AEA800C202AD1AC4F814515448D4F81C11049BBA
:10AEB800534D02682D78C4F81C31591A0A440260AF
:10AEC800002D40F0DB8107EE901A4E4EDFF86491BA
:10AED8004D4FB8EEE78A06F5F07506F51378F6ECEF
:10AEE800017A9BED070ADBF80832F8EEE77A284684
:10AEF80027EE800A9847A5F1E000DBF8283198474B
:10AF0800A5F17000DBF898319847D6F8EC00DBF82B
:10AF1800AC309847D7ED007AA9EC010AE0EE087A40
:10AF28002435A845E7EC017AD9D1029B1E78FEF7B3
:10AF38003CBD364B364A19681288364BC9691980A8
:10AF48005A8013B0BDEC0E8BBDE8F08F324B334EF8
:10AF58001A7812F0010F327840F0DC83002A00F0F2
:10AF6800D58592002E492F48DFF8CCA0DFF8CC9089
:10AF780028F07DF8FFF735BA2B4C1FF0C5FF637832
:10AF8800022B00F03D86032B7FF4A5AC41F2B813E9
:10AF9800E35C002B41F06E8341F2A403E35C002BD9
:10AFA80041F0638341F2E803E35C002B41F05883EE
:10AFB80041F22C13E35C002B3FF48DAC1B4821F0CD
:10AFC80021FC88E4B4F8E071013F3FB2002FA4F8F7
:10AFD800E0717FF791AE164EFFF7D8BABA4000205D
:10AFE800B043002000000000E81E0020BC40002004
:10AFF800B8400020D842002093244992D43400203D
:10B00800B0400020BC490020D8340020383D002042
:10B018002A52002010320020EF3A0020BA310020D6
:10B028002C5200206C57002094590020C06A002040
:10B03800343200200C4C0020184C0020E879002005
:10B04800002D00F02787BCF1000F42F00983CC4D9A
:10B05800002B42F09D8195ED006A9DED0A5AC94882
:10B0680025EE866AFDEEE44AA5EE076AB0EE675A59
:10B07800A6EE265A14EE901ABDEEC56A16EE10CA50
:10B0880016EE107AF445A8BF77466145C8BF0F464B
:10B0980006EE107AB8EEC66A012A80ED006A00F062
:10B0A800DF8095ED046A9DED0B5A25EE866AA5EEC4
:10B0B800076AB0EE675AA6EE265ABDEEC56A16EEC6
:10B0C80010CA16EE107AF445A8BF77468C45B8BF6B
:10B0D8000F4606EE107AB8EEC66A022A80ED016ABB
:10B0E80000F0BE8095ED086A9DED0C5A25EE866A43
:10B0F800A5EE076AB0EE675AA6EE265ABDEEC56AF7
:10B1080016EE10CA16EE107AF445A8BF77468C459D
:10B11800B8BF0F4606EE107AB8EEC66A032A80ED6D
:10B12800026A00F09D8095ED0C6A9DED0D5A25EEA2
:10B13800866AA5EE076AB0EE675AA6EE265ABDEEF5
:10B14800C56A16EE10CA16EE107AF445A8BF7746FF
:10B158008C45B8BF0F4606EE107AB8EEC66A042AC8
:10B1680080ED036A7CD095ED106A9DED0E5A25EEB0
:10B17800866AA5EE076AB0EE675AA6EE265ABDEEB5
:10B18800C56A16EE10CA16EE107AF445A8BF7746BF
:10B198008C45B8BF0F4606EE107AB8EEC66A052A87
:10B1A80080ED046A5CD095ED146A9DED0F5A25EE8A
:10B1B800866AA5EE076AB0EE675AA6EE265ABDEE75
:10B1C800C56A16EE10CA16EE107AF445A8BF77467F
:10B1D8008C45B8BF0F4606EE107AB8EEC66A062A46
:10B1E80080ED056A3CD095ED186A9DED105A25EE64
:10B1F800866AA5EE076AB0EE675AA6EE265ABDEE35
:10B20800C56A16EE10CA16EE107AF445A8BF77463E
:10B218008C45B8BF0F4606EE107AB8EEC66A072A04
:10B2280080ED066A1CD095ED1C6A9DED115A65EEFD
:10B23800865AE7EE055AE6EEA57AFDEEE77A17EEAE
:10B24800905AAE45A8BFAE46A942D8BF714607EE90
:10B25800901AF8EEE77AC0ED077A002A3FF4C1A801
:10B2680092004949474827F002FF484A1268002AD5
:10B278003FF4BCA80BF070FDFFF7B8B807EE901AC2
:10B28800434D444BDFF81881DFF818910394F8EE2A
:10B29800E78A05F5B87600271C46CDF81880029B8A
:10B2A800DBED077A1B78172B56D095ED007AB8EEB0
:10B2B800C78A082B28EE278A07D1B0EE480A0593DB
:10B2C80026F034FF059BA8F80000DAF8002090006B
:10B2D8000BD5002F02F0A287B0EE480ADBF808323F
:10B2E80006F170009847B0EE408AB0EE480ADBF8E5
:10B2F8002831A6F170009847DBF898313046984716
:10B30800029B1B78032BB0EE408A20D0D5F8F000C2
:10B31800DBF8AC30B0EE480A9847D9ED007AA4ECD7
:10B32800010AE0EE287A0137032F06F1240608F116
:10B33800020805F10405E9EC017AB0D1029B039CEF
:10B348001E78FEF732BBF0EE676AFFF779B926F090
:10B35800EDFEA8F80000D9E795ED007A0BEB47025F
:10B36800B8EEC78A128FA8F8002028EE278AACE723
:10B37800B0EE465AFEF7CBBC074B0293074C93E559
:10B38800503600206C5700202C520020682D0020D9
:10B39800BC4900200C4C00200C320020E81E002084
:10B3A80010320020D8340020DBF80830002B3FF49E
:10B3B8003EA8C649A1F14C009847C54B1B68180721
:10B3C8007FF53AA8C34ED6ED027AB2EE0E7AF0EEC9
:10B3D800E76AF4EEC76AF1EE10FA41D5BE4B1B8856
:10B3E80059073DD5BD4BBE49B3F90430B4F8A62181
:10B3F80081FB0301DB17C3EBA1039B1A9BB219B2B4
:10B4080011F1B30FBCBF03F5B47319B2B329C4BFAC
:10B41800A1F5B47319B2B34BB34A1B791278002B58
:10B428004FF6FF7318BF012312077FF505A8AF4A2F
:10B43800126811FB03F3117EAD4A9BB211FB03F3B3
:10B4480082FB03121A44DB17C3EB221307EE103AF0
:10B45800B8EEC77A77EEC77AC6ED027AFEF7ECBF88
:10B468009E4B9F4AB3F9043082FB0312DB17C3EBF0
:10B47800A203A4F8A631FEF7DFBF9E499E4BD1F880
:10B48800EC101B6844F620608142A8BF0146B1F564
:10B498007A7FB8BF4FF47A7189B213F0100FA4F80D
:10B4A800B211DAF8003000F0C283DB0441F15D85A7
:10B4B8008E4BD3F800E0BEF832707F08854E8F4877
:10B4C800D4F8B431D6ED037AA0FB010188096421D0
:10B4D80091FBF0F11429BDEEE77A04EB4306A8BF0F
:10B4E800142101339942C4F8B43117EE10CADCBFF5
:10B4F8000023C4F8B43104EB4303A6F8B8C1B3F988
:10B50800B83107EE103AB8EEC77A77EEC77AFDEE93
:10B51800E77ACDED037ABDF90C1081EAE173A3EB6C
:10B52800E173BB4201F3EE8675494FF07E530B6021
:10B53800FEF7AABF1E217048F6F7BAFD00283FF4AF
:10B54800C2A9654B1B885A063FF5BDA994F8043279
:10B55800B34242F0D9816A4BD4ED827AD3ED016AC5
:10B5680094ED505ADFED675A9FED676A27EEC57A6A
:10B5780068EE277AA8EE267AE5EE267AB4EEE57A22
:10B58800F1EE10FA88BFB0EE657AB4EEC67AF1EE45
:10B5980010FAF4EEE57AB8BFB0EE467AF1EE10FA9A
:10B5A80088BFF0EE657AF4EEC67AF1EE10FAB8BF0D
:10B5B800F0EE467A84ED4E7AC4ED507AFFF783B9FF
:10B5C800FDEEC87A514A17EE903A9780D380FFF77C
:10B5D80075B9DFED4F6AFFF724BADAF800104F02A9
:10B5E8003EF5A3ADFEF7A5BDB4EEC87AF1EE10FAAC
:10B5F80098BFB0EE478ABDEEC77AB4EEE68ADFF8A8
:10B608000CC1F1EE10FA17EE103AB8BFB0EE668A28
:10B6180084ED4E8AACF80030BEF1000F7FF46EA8BE
:10B62800FFF74CB99FED377ADFED376A3749F4EE0B
:10B63800C77AF1EE10FA98BFB0EE677AFDEEE77AB6
:10B64800B4EEE67AF1EE10FA17EE903AB8BFB0EE23
:10B65800667ABEF1010F84ED4F7A4B803FF7B4A8AC
:10B66800FFF72CB9BDEEE77A284B17EE102A9A801F
:10B67800FFF70DB9002B3EF4AFAAFEF78CBAF9F725
:10B688001FFE029B21491A78039B072AA0EB03009F
:10B6980088807EF4C6AEF9F713FE0546FEF7C2BEF3
:10B6A800F9F70EFE029BDFF864801A78079B012ADF
:10B6B800A0EB0300A8F8020000F08C82072A7EF4B1
:10B6C800B3AAF9F7FDFD0390FEF7B0BADC490020F4
:10B6D80000340020343200205C3400200C34002078
:10B6E80067666666B855002004570020603400205D
:10B6F80089888888800F0020FC560020D34D62106E
:10B708000400002000C0F94400C0F9C41032002031
:10B7180000000000002A00F0F981D4ED583A94EDB9
:10B72800574AD4ED627AF34994ED617A91ED005A63
:10B73800D4ED555A94ED546AEF4DF048F4EEC43AFE
:10B74800F3EE046AF1EE10FA77EEA64A00F1C2822F
:10B7580095ED026A26EE656AB0EE674AA6EE074ADC
:10B76800B4EEE44A34EE666AF1EE10FA48BFB0EE81
:10B77800456A012A80ED006A00F0C88195ED066AE5
:10B7880026EE656AB0EE674AA6EE074AB4EEE44ACA
:10B7980034EE666AF1EE10FA48BFB0EE456A022A46
:10B7A80080ED016A00F0B28195ED0A6A26EE656ABD
:10B7B800B0EE674AA6EE074AB4EEE44A34EE666A8B
:10B7C800F1EE10FA48BFB0EE456A032A80ED026A2E
:10B7D80000F09C8195ED0E6A26EE656AB0EE674A28
:10B7E800A6EE074AB4EEE44A34EE666AF1EE10FAC1
:10B7F80048BFB0EE456A042A80ED036A00F08681EE
:10B8080095ED126A26EE656AB0EE674AA6EE074A1B
:10B81800B4EEE44A34EE666AF1EE10FA48BFB0EED0
:10B82800456A052A80ED046A00F0708195ED166A74
:10B8380026EE656AB0EE674AA6EE074AB4EEE44A19
:10B8480074EE666AF1EE10FA48BFF0EE456A062A11
:10B85800C0ED056A00F05A81D5ED1A6A66EEE56A10
:10B86800B0EE674AA6EE874AB3EE046AB4EEE44A3D
:10B8780074EE466AF1EE10FA48BFF0EE456A072A00
:10B88800C0ED066A00F04281D5ED1E6ADFF874A2A9
:10B89800DFF8749266EEE55AE5EE877AF4EEE47A1C
:10B8A80077EEC67AF1EE10FA48BFF0EE457AC0EDB1
:10B8B800077AFEF796BD904D9DED0A5A95ED006A00
:10B8C800BCF1000F41F0E48125EE866A8B48A5EEB5
:10B8D800076AB0EE675AA6EE265ABDEEC56A16EE9E
:10B8E80010CA16EE107AF445A8BF77466145C8BF5E
:10B8F8000F4606EE107AB8EEC66A012A80ED006A95
:10B908003FF4AEAC95ED046A9DED0B5A25EE866AC0
:10B91800A5EE076AB0EE675AA6EE265ABDEEC56ACE
:10B9280016EE10CA16EE107AF445A8BF77466145A0
:10B93800C8BF0F4606EE107AB8EEC66A022A80ED36
:10B94800016A3FF48DAC95ED086A9DED0C5A25EE21
:10B95800866AA5EE076AB0EE675AA6EE265ABDEECD
:10B96800C56A16EE10CA16EE107AF445A8BF7746D7
:10B978006145C8BF0F4606EE107AB8EEC66A032ABC
:10B9880080ED026A3FF46CAC95ED0C6A9DED0D5AA2
:10B9980025EE866AA5EE076AB0EE675AA6EE265A25
:10B9A800BDEEC56A16EE10CA16EE107AF445A8BFA9
:10B9B80077466145C8BF0F4606EE107AB8EEC66AEC
:10B9C800042A80ED036A3FF44BAC95ED106A9DEDB7
:10B9D8000E5A25EE866AA5EE076AB0EE675AA6EEFD
:10B9E800265ABDEEC56A16EE10CA16EE107AF44550
:10B9F800A8BF77466145C8BF0F4606EE107AB8EE75
:10BA0800C66A052A80ED046A3FF42AAC95ED146AEB
:10BA18009DED0F5A25EE866AA5EE076AB0EE675AC5
:10BA2800A6EE265ABDEEC56A16EE10CA16EE107AB4
:10BA3800F445A8BF77466145C8BF0F4606EE107AA1
:10BA4800B8EEC66A062A80ED056A3FF409AC95EDA2
:10BA5800186A9DED105A25EE866AA5EE076AB0EEC3
:10BA6800675AA6EE265ABDEEC56A16EE10CA16EE3D
:10BA7800107AF445A8BF77466145C8BF0F4606EE61
:10BA8800107AB8EEC66A072A80ED066A3FF4E8AB7A
:10BA980095ED1C6A9DED115A65EE865AE7EE055A3A
:10BAA800E6EEA57AFDEEE77A17EE905AAE45A8BF06
:10BAB800AE46A942C8BF8E4607EE90EAF8EEE77A8E
:10BAC800C0ED077AFFF7C9BBDFED0D6AFEF7DABEF6
:10BAD800B5EEC07AF1EE10FA01F13A82B7EE006ADB
:10BAE80036EE477AC6EE076AFEF752BE9FED046A45
:10BAF800FEF7E7BD4C360020503600206C5700207A
:10BB08000000C842184C0020E8790020DFF878A32C
:10BB1800DFF87893FEF765BCC8494A79002A3EF4F5
:10BB280087A9C74A1278002A3EF482A90B78C5492A
:10BB3800DFEDC54A07EE903A0B88B8EE677A07EE54
:10BB4800902A06EE903AF8EEE77AF8EE666A67EE23
:10BB5800277AB7EE007A87EEA63AB4EEE43AF1EE29
:10BB680010FA88BFB0EE643AB4EEC73AF1EE10FAB4
:10BB7800B8BFB0EE473AFEF75DB9B44B5988FEF747
:10BB880096BCB4F8B21101F57A7189B2FEF78FBC90
:10BB9800AF4B93ED006AFEF726BF04981DF0F6FE42
:10BBA800FEF7A1BEAB4B9FEDAC7AD3ED087AF4EE6D
:10BBB800C77AF1EE10FA00F2F7849FEDA87AA84E42
:10BBC800D6ED037A77EE877AC6ED037AFEF757BC8F
:10BBD800DFF8BC82F9F774FBA249D4F87C21096824
:10BBE8000390821A511AC4F87C01A8F80420A8F816
:10BBF8000610FEF71BB8F9F763FB0790FDF79FBD2A
:10BC0800A3784FF0010A072B3EF665AEDFE813F084
:10BC1800560656073F074B076E0628073207520697
:10BC2800914B9B7B002B3EF41DACFEF720BCD8004B
:10BC38003FF53BACFEF728BCB4F88C51954240F276
:10BC4800FE8494F8A451002D40F0C787874A884E97
:10BC580092ED007AD6ED007A94F99821C4ED647AD1
:10BC680077EE676A012AC4ED627AC4ED616A84EDF1
:10BC7800657A02F01A80049BC4F89C317D4A9FEDD6
:10BC8800777A92ED005A84ED687A012284F8982137
:10BC9800FEF73CBF784B1B88002B40F0F385774AB2
:10BCA800774B11781868FAF775F9D4F86C21049B6A
:10BCB8009A1AFDF7FABD734BD9ED007A93ED007A25
:10BCC800F0EEE77AF4EEC77AF1EE10FA7DF784AF7A
:10BCD800FDF774BFD5ED015A65EEC65AB0EE674A56
:10BCE800A5EE874AB4EEE44A74EE665AF1EE10FA0D
:10BCF80048BFF0EE455A012AC0ED005A3FF406AF9E
:10BD0800D5ED055A65EEC65AB0EE674AA5EE874AE4
:10BD1800B4EEE44A74EE665AF1EE10FA48BFF0EE5B
:10BD2800455A022AC0ED015A3FF4F0AED5ED095A42
:10BD380065EEC65AB0EE674AA5EE874AB4EEE44A05
:10BD480074EE665AF1EE10FA48BFF0EE455A032A2F
:10BD5800C0ED025A3FF4DAAED5ED0D5A65EEC65A7B
:10BD6800B0EE674AA5EE874AB4EEE44A74EE665A26
:10BD7800F1EE10FA48BFF0EE455A042AC0ED035A16
:10BD88003FF4C4AED5ED115A65EEC65AB0EE674A17
:10BD9800A5EE874AB4EEE44A74EE665AF1EE10FA5C
:10BDA80048BFF0EE455A052AC0ED045A3FF4AEAE3E
:10BDB800D5ED155A65EEC65AB0EE674AA5EE874A24
:10BDC800B4EEE44A74EE666AF1EE10FA48BFF0EE9B
:10BDD800456A062AC0ED056A3FF498AED5ED196AA2
:10BDE80066EEC66AB0EE674AA6EE874AF3EE045AD4
:10BDF800B4EEE44A74EE656AF1EE10FA48BFF0EE6C
:10BE0800456A072AC0ED066A3FF480AED5ED1D6A83
:10BE1800DFF874A0DFF8749026EEC66AE6EE077ABB
:10BE2800F4EEE47A77EEE57AF1EE10FAB8BFF0EEC8
:10BE3800457AC0ED077AFEF7D4BA00BFF033002088
:10BE4800323200201C320020713DAA3F583E0020AB
:10BE580008360020AC3400208FC2753C000000007A
:10BE680034320020F8580020447A00208C550020F5
:10BE7800D0360020EC360020AC560020AE5600200C
:10BE8800B056002040360020184C0020E8790020E9
:10BE980010320020D94D002B41F09E8095ED006AAC
:10BEA8009DED0A5AD64825EE866AFDEEE44AA5EECF
:10BEB800076AB0EE675AA6EE265A14EE901ABDEE3F
:10BEC800C56A16EE108A16EE107AF045A8BF7746B6
:10BED8004145C8BF0F4606EE107AB8EEC66A012A79
:10BEE80080ED006A3EF479AA95ED046A9DED0B5A3F
:10BEF80025EE866AA5EE076AB0EE675AA6EE265AC0
:10BF0800BDEEC56A16EE108A16EE107AF045A8BF87
:10BF180077468845B8BF0F4606EE107AB8EEC66A6F
:10BF2800022A80ED016A3EF458AA95ED086A9DED53
:10BF38000C5A25EE866AA5EE076AB0EE675AA6EE99
:10BF4800265ABDEEC56A16EE108A16EE107AF0452E
:10BF5800A8BF77468845B8BF0F4606EE107AB8EEF8
:10BF6800C66A032A80ED026A3EF437AA95ED0C6A88
:10BF78009DED0D5A25EE866AA5EE076AB0EE675A62
:10BF8800A6EE265ABDEEC56A16EE108A16EE107A8F
:10BF9800F045A8BF77468845B8BF0F4606EE107A29
:10BFA800B8EEC66A042A80ED036A3EF416AA95ED37
:10BFB800106A9DED0E5A25EE866AA5EE076AB0EE68
:10BFC800675AA6EE265ABDEEC56A16EE108A16EE18
:10BFD800107AF045A8BF77468845B8BF0F4606EEE9
:10BFE800107AB8EEC66A052A80ED046A3EF4F5A90F
:10BFF80095ED146A9DED0F5A25EE866AA5EE076A3F
:10C00800B0EE675AA6EE265ABDEEC56A16EE108A3D
:10C0180016EE107AF045A8BF77468845B8BF0F4698
:10C0280006EE107AB8EEC66A062A80ED056A3EF476
:10C03800D4A995ED186A9DED105A25EE866AA5EEED
:10C04800076AB0EE675AA6EE265ABDEEC56A16EE26
:10C05800108A16EE107AF045A8BF77468845B8BF13
:10C068000F46FEF798B9674ED4ED017A94ED006A51
:10C078003188726977EEA77AF0EE006AB0EE677AD7
:10C08800A6EE267A4E1E04EBC601D6EE267A0839AD
:10C098001032F6EE003A27EE237A67EEA37A84EDA3
:10C0A800207AC4ED217A584C274604F1800091ED9E
:10C0B800027A91ED036AD7ED036AD7ED027A52ED61
:10C0C800014A12ED025A37EE674A76EEC65A77EE03
:10C0D800277AE4EE845A013EA1F10801E5EE047ADC
:10C0E80007F1080702F1080236EE267A00F1080087
:10C0F800E4EE877AE5EE475A67EEA37A25EEA37A4F
:10C10800C0ED007A80ED017AD1D1BEF1140F7EF432
:10C11800BEAEF9F7D5F8039BDFF80081C01AA8F87E
:10C128000200D4F81451FEF7B2BED4F81831B4F8AE
:10C1380010C1364ACCF120095FFA89F90CEB431794
:10C1480002EB87075FEA990201F0FB8501321601CD
:10C158002F48304907EB060807F1100212ED024A92
:10C1680012ED035A12ED016A12ED047A50ED024AFB
:10C1780050ED035A50ED016A50ED047A64EE244AFA
:10C1880065EE255A66EE266A67EE277A10329045E4
:10C1980041ED024A41ED035A41ED016A41ED047A4D
:10C1A80000F1100001F11001D8D11B48A6F11001CF
:10C1B8000F4400EB0108214419F0030209D0B7EC41
:10C1C800017AF8EC017A67EE277A013AE1EC017A14
:10C1D800F5D1BCF1000F41F04280BEF1140F7EF49E
:10C1E80056AEF9F76DF8039BDFF83080D4F8145198
:10C1F800C01AA8F80200FEF74ABE00BF5036002059
:10C208006C570020C0400020E81E0020D8400020C5
:10C2180068420020F81E00205842002010320020FA
:10C22800D04E31785FEA910C01F07E86CE4F0CF14A
:10C2380001094FEA491907EB090807F12002A7F19C
:10C24800700012ED076A52ED056A12ED037A52ED9D
:10C25800017A52ED025A12ED084A52ED064A12EDE1
:10C26800045A26EE066A66EEA66A27EE077A67EE95
:10C27800A77AA4EE046A20329045E4EEA46A00F19D
:10C288001000A5EE057AE5EEA57AF1EEC65AB1EEF4
:10C29800E66AF1EEC76AB1EEE77A40ED085A00EDBA
:10C2A800076A40ED066A00ED057ACAD1A9F12002B5
:10C2B8003A4404EB0C1711F0030018BF08320FD0F2
:10C2C80052ED017A12ED027A67EEA77A0138E7EEAD
:10C2D800077A02F10802B1EEE77AA7EC017AEFD10A
:10C2E800BEF1140F01F034850135C4F81451FEF77E
:10C2F8003DBDD4F818519D499D489E4BEA00114414
:10C3080015448A88196800EE102A643AC82AA8BF1A
:10C31800C822782AB8BF782207EE902AB8EEC07AE9
:10C32800F8EEE77A00EB850577EE670A77EE876A1D
:10C3380067EE877A20EEA67AB8EE400AC7EE870A3B
:10C348002846D5F81490D5F81880EF692E6A23F09E
:10C3580001FD029BC5F8149093F800E0C5F8188019
:10C36800BEF1140FEF612E6201F00285D4F8182196
:10C37800814BD4F81451013283FB0213A3EBE2730F
:10C3880003EB4303D31A0135C4F81831C4F8145128
:10C39800CDE67A4E7A48B268B18924F08DFD029BC9
:10C3A80093F800E0BEF1140F01F0EF84D4F81451B3
:10C3B8000135C4F8145157E6704E318873684FEA56
:10C3C80051094FEA89005FEAD10C04EB000204EB43
:10C3D800810500F0A18000F110010CF1010C694FFA
:10C3E80002EB0C1C2944103203F1100E05F1100069
:10C3F80050ED032A50ED043A17ED043A17ED032ADD
:10C4080050ED026A10ED016A17ED021A57ED010AA4
:10C4180011ED044A11ED035A52ED044A52ED035A44
:10C4280012ED027A52ED017A51ED021A11ED010A6C
:10C4380073EE238A32EE228A47ED048A07ED038AD7
:10C4480071EE268A30EE868A47ED028A07ED018A68
:10C4580074EE848A35EE858A42ED048A02ED038AF9
:10C4680077EE218A37EE808A42ED028A02ED018A50
:10C4780073EE633A75EE655A1EED035A32EE623A70
:10C4880074EE644A25EE638A1EED044A23EE052AFB
:10C4980064EE652AA3EE048A1032944524EE843AA9
:10C4A800A3EE842A07F110070EF1100EA5EE853AC7
:10C4B80000F1100001F11001E4EE852A00ED078A71
:10C4C80000ED082A01ED073A41ED082A5EED055A0C
:10C4D8001EED065A71EE666A30EEC66A31EEC77A0C
:10C4E80070EE677A26EE253A65EEE63A25EE674A5B
:10C4F80067EE054AE6EE053AA6EE853AA7EE254A26
:10C50800E7EEA54A00ED063A40ED053A01ED064A88
:10C5180041ED054A7FF46CAF1FFA89F91A4649467E
:10C52800174822F0F9FF72684946284622F0F4FFBE
:10C53800029B1A78142A7FF4F4ADEAE5F8F7C0FEF6
:10C54800029B039093F800E0BEF1140F05BFDFF8DB
:10C558003880D4F81451D4F81451A8F80050FCF7D6
:10C56800F0BF00BFBA400020681F0020B043002081
:10C578009C4B0020084C002056555555C0400020C3
:10C58800E81E0020F81E002010320020306E99BCF2
:10C598002716983DA40DC93F843459BEDB0F494086
:10C5A800D06D393A00000000F0EEE76AB7EE005AA5
:10C5B80035EE665A1FED0B4A5FED0B5A1FED0A6AFE
:10C5C8001FED0C7A94ED6B0AF1EEC54AE6EE845A3B
:10C5D800F5EEC07AA6EEA56AF1EE10FAA6EE867A16
:10C5E80048BF5FED127A27EE247A48BF37EEC77A44
:10C5F80027EE000A25F09AFDB0F5617F00F39D86CD
:10C6080007EE900AF8EEE76A5FED1B7A66EEA76A16
:10C6180007EE906ABDEEE67AF8EEE77A17EE103A82
:10C628002033402B41F291841FED220A25F07EFD34
:10C6380000B207EE900AB8EEE77AFFF7C0BAC84A28
:10C6480002F1500503E00432954200F0C6821378E7
:10C65800262BF8D19678D3789E42F4D2FFF7F1BA18
:10C66800C04820F0CFF8FEF7A3BCBF4820F0CAF8B6
:10C67800FEF798BCBD4820F0C5F8FEF78DBCBC4D50
:10C68800BC4F95ED004A95ED057AD5ED014A95ED3B
:10C69800066AD5ED046A95ED035AD5ED025A67EEA0
:10C6A800897A07EB8602A4EE277AA4EEA76A66EEDB
:10C6B800C76AA5EE476AE5EEA76A20EE070A85ED88
:10C6C800056AC5ED066A82ED007A29EE088A25F02A
:10C6D8002DFD69EE288AD5ED0E5AD5ED176A95ED30
:10C6E800091AD5ED121A95ED0F5A95ED187A95EDB0
:10C6F8000A2AD5ED132A95ED0D6AD5ED167A95ED32
:10C708000C3AD5ED0B3A95ED154AD5ED144AE1EE04
:10C71800085A002207EB8601E8EEA16A00B2C4F8C5
:10C728000021A2EE085AC4F80421C4F80821A8EE92
:10C73800A27A26EE656A67EEE67AA3EE655AA3EE5C
:10C74800886AA6EEC47AE8EEA47A85ED0E5AC1EDA1
:10C75800205A85ED0F6AC1ED406A85ED177AC5ED5F
:10C76800187AFEF7BDBAD4F89C51049B5D1BFEF7FE
:10C77800BDB9BBF93820CBF8201007EE902A01216B
:10C78800F8EEE77ACBF86020CBF87C100022012F76
:10C79800CBED1C7ACBED1B7ACBF8742001F06782C5
:10C7A800AF427CF432AFBBF93A20CBF8642007EEF5
:10C7B800902A00210122F8EEE77ACBF82410CBF872
:10C7C80090200022012FCBED217ACBED207ACBF8F7
:10C7D800882001F05082AF427CF44BAFBBF93C207B
:10C7E800CBF8682007EE902A00210122F8EEE77ABC
:10C7F800CBF82810CBF8A4200022012FCBED267A05
:10C80800CBED257ACBF89C207CF467AF9FED5A8A54
:10C81800032E49D04CB107EE904AF8EEE77AF4EED1
:10C82800C87AF1EE10FA01F1D683544A544C1168D3
:10C83800DBF86820A8F8060094F8200102EB5502FE
:10C8480092FBF5F50022CBF828508A620A63CA6287
:10C8580028B14C4A126832F480637CF441AF4A4AEA
:10C86800126812F4003241F0FA8148481146835C9C
:10C87800012B02F10C0200F0908301311829F6D146
:10C88800FCF72EBF42494B69002B3DF40EA84148E6
:10C89800414B008893FBF0F00B684FF0010E1860D5
:10C8A80081F811E0FDF701B8B0EE480A25F03EFC2A
:10C8B80000B2AFE703236370FEF70DB800230AAE9A
:10C8C8003146184609221EF0FBF801287EF403A819
:10C8D8000A9B93F8FE21552A01F0F08141F2B41227
:10C8E80002210123A1546370FDF7F5BF2278237D4F
:10C8F8002A4FDFF8B490032A14BF4FF480784FF022
:10C908008008002B67D0012BFBD1254B6268196882
:10C91800386800234FEA412E4FF0FF31B1FBFEF19A
:10C9280012EB010B43F1000C0021614500F10200FC
:10C9380008BF584538BF83465A461A4902201EF098
:10C94800FFF9032801F2B78101A353F820F000BFD3
:10C95800DFA80008B5C90008DFA80008B5C90008A5
:10C96800603900207C6A0020386A00204C6B002067
:10C9780044430020D840002000000000383D00203B
:10C98800E81E002058340020F85300203C500308CB
:10C99800B4560020CC56002020A107009C6B002034
:10C9A800A46B00209C590020985900206268A36855
:10C9B8002669991AB14284BFE260216103281FD019
:10C9C8000133B3FBF8F208FB12320AB143449B1A55
:10C9D8000022636022753A684946023200201EF040
:10C9E800AFF9032801F2678101A353F820F000BFD3
:10C9F800DFA80008FFCA0008DFA8000809CA000865
:10CA080023690622652BA27034D92278032A14BF21
:10CA18006FF0FF026FF07F02A3F1650303EA0203E0
:10CA280003F1010314BF4FF4807280229A422361FC
:10CA380020D23A68E768023203EB0708904581F094
:10CA48002883844A6760D16FC4F80880490203FBD1
:10CA580001F30521176042F81C3C42F8183CA1700C
:10CA6800A2687D4901201FF003FC012841F01683CC
:10CA78000623A370002179481FF01AF8012841F015
:10CA88000D83A3780133DBB2A370FFF7BCB8744BF6
:10CA980000930320A0703023052272496F481FF0CD
:10CAA8002BFFFDF718BF41F27013E35C002B3DF438
:10CAB80012AF6A481FF0A6FEFDF70DBF0AAE41F29D
:10CAC800FC173146E059002309221DF0F9FF01281F
:10CAD8007DF401AF00230A9A2370B2F80B30B3F546
:10CAE800007F01F0E58241F2B41203210123A15431
:10CAF8006370FDF7F0BE636884F814A00133A36087
:10CB080003E7DFED597A594B94ED687AC3ED007A63
:10CB1800C3ED017AC3ED027A554BF0EE674AF0EEA9
:10CB2800673A1968FDF7BCB8524A534DD2ED006A0E
:10CB3800524A95ED006A1278C4ED646A84ED656A1C
:10CB4800002A00F00D8276EE665A94F99821C4ED19
:10CB5800615A0132C4ED626A00F07285049BC4F820
:10CB68009C31002537EE677AFCEEE77A444E84ED77
:10CB7800687A17EE902AA4F88C21FF2296ED005AC5
:10CB880084F89821FDF7C2BF3E49DFED3F7A096876
:10CB9800C4ED4C7A11F0805840F0C383DAF80010E5
:10CBA80011F4800800F0EF814FF00008B6EE007A2B
:10CBB80067EE877AF4EEE57AF1EE10FAC8BFF0EE88
:10CBC800675A40F3AE83C4ED685AFDF7B2BA2F4BEB
:10CBD8001D7805F0010CFDF700BC264A264DD2ED64
:10CBE800007A264A95ED007A1278C4ED647A84EDCD
:10CBF800657A002A00F02E8377EE676A94F9982107
:10CC0800C4ED616A0132C4ED627A00F05586049B76
:10CC1800C4F89C3100259FED147A194E84ED687A8A
:10CC2800FF2296ED005A84F89821FDF76FBF73EE46
:10CC3800E77AB7EE007AF4EEC77AF1EE10FAC4EDAF
:10CC48004C7A41F32A8084EEA77A8DED0A7AFDF7B3
:10CC580066BA00BF286B002098590020046B00209A
:10CC680011B802082C5C03080000000014570020CB
:10CC78006034002088550020D43600203C4E002027
:10CC8800E8360020FC56002000000080EF3A002023
:10CC9800002F00F0CB8625EE866ACC48A5EE076A01
:10CCA800B0EE675AA6EE265ABDEEC56A16EE10CA51
:10CCB80016EE107AF445A8BF77466145C8BF0F46FF
:10CCC80006EE107AB8EEC66A012A80ED006A3DF4D5
:10CCD80088AB95ED046A9DED0B5A25EE866AA5EEA4
:10CCE800076AB0EE675AA6EE265ABDEEC56A16EE7A
:10CCF80010CA16EE107AF445A8BF77466145C8BF3A
:10CD08000F4606EE107AB8EEC66A022A80ED016A6E
:10CD18003DF467AB95ED086A9DED0C5A25EE866AE1
:10CD2800A5EE076AB0EE675AA6EE265ABDEEC56AAA
:10CD380016EE10CA16EE107AF445A8BF774661457C
:10CD4800C8BF0F4606EE107AB8EEC66A032A80ED11
:10CD5800026A3DF446AB95ED0C6A9DED0D5A25EE41
:10CD6800866AA5EE076AB0EE675AA6EE265ABDEEA9
:10CD7800C56A16EE10CA16EE107AF445A8BF7746B3
:10CD88006145C8BF0F4606EE107AB8EEC66A042A97
:10CD980080ED036A3DF425AB95ED106A9DED0E5AC2
:10CDA80025EE866AA5EE076AB0EE675AA6EE265A01
:10CDB800BDEEC56A16EE10CA16EE107AF445A8BF85
:10CDC80077466145C8BF0F4606EE107AB8EEC66AC8
:10CDD800052A80ED046A3DF404AB95ED146A9DEDD7
:10CDE8000F5A25EE866AA5EE076AB0EE675AA6EED8
:10CDF800265ABDEEC56A16EE10CA16EE107AF4452C
:10CE0800A8BF77466145C8BF0F4606EE107AB8EE50
:10CE1800C66A062A80ED056A3DF4E3AA95ED186A0C
:10CE28009DED105A25EE866AA5EE076AB0EE675AA0
:10CE3800A6EE265ABDEEC56A16EE10CA16EE107A90
:10CE4800F445A8BF77466145C8BF0F4606EE107A7D
:10CE5800B8EEC66A072A80ED066A3DF4C2AA95EDC7
:10CE68001C6A9DED115A65EE865AE5EE075AE6EE04
:10CE7800A57AFDEEE77A17EE902A9645A8BF964662
:10CE88009142D8BF714607EE901AF8EEE77AC0EDE6
:10CE9800077AFDF7A6BABEF1010F7FF7B7AC07EE28
:10CEA800103AB8EEC77AC7EE876AB1EEE68AAFE401
:10CEB800BEF1010F40F3DB8607EE103AB8EEC77AF1
:10CEC800C7EE876AB1EEE68A032E13D04CB107EE9F
:10CED800904AF8EEE77AF4EEC87AF1EE10FA01F12A
:10CEE8007A80DBF8602002EB550292FBF5F2CBF872
:10CEF800202055E4B0EE480A25F018F900B2E5E71D
:10CF0800BEF1010F40F3B78607EE103AB8EEC77AC4
:10CF1800C7EE876AB1EEE68A032E13D04CB107EE4E
:10CF2800904AF8EEE77AF4EEC87AF1EE10FA01F1D9
:10CF38005280DBF8642002EB550292FBF5F2CBF845
:10CF4800242048E4B0EE480A25F0F0F800B2E5E7FE
:10CF5800F7EE006AFDF71CBCF7EE006AFDF792BC1D
:10CF680076EEC65AF0EE466AEFE5194BD3F800E0C4
:10CF7800BEF93270FEF7A2BA8222FDF775BFDFED67
:10CF8800157AFDF73DBFB6EE007AF4EEC75AF1EE1A
:10CF980010FA3FF70BAEFDF7CCB8D4F824614A007D
:10CFA8003EB1551800EB850576786D78B542BCF42E
:10CFB80097AB0A4400EB82000022C4F82401A4F8CD
:10CFC8000C22C4F81022FCF78BBB00BF6C57002062
:10CFD800603400200000024395ED006A9DED0A4A86
:10CFE800E34825EE866AFDEEE43AA4EE076AB0EE61
:10CFF800674AA6EE264A13EE901AB4EEC45AF1EE2A
:10D0080010FAB0EE446A88BFB0EE646ABDEEC66A34
:10D0180016EE108A16EE107AF045A8BF77464145FD
:10D02800C8BF0F4606EE107AB8EEC66A012A80ED30
:10D03800006A3DF4D2A995ED046A9DED0B4A25EEF0
:10D04800866AA4EE076AB0EE674AA6EE264AB4EEF0
:10D05800C45AF1EE10FAB0EE446A88BFB0EE646AC2
:10D06800BDEEC66A16EE108A16EE107AF045A8BF15
:10D0780077468845B8BF0F4606EE107AB8EEC66AFE
:10D08800022A80ED016A3DF4A8A995ED086A9DED94
:10D098000C4A25EE866AA4EE076AB0EE674AA6EE49
:10D0A800264AB4EEC45AF1EE10FAB0EE446A88BFCC
:10D0B800B0EE646ABDEEC66A16EE108A16EE107AF5
:10D0C800F045A8BF77468845B8BF0F4606EE107AE8
:10D0D800B8EEC66A032A80ED026A3DF47EA995ED92
:10D0E8000C6A9DED0D4A25EE866AA4EE076AB0EE3D
:10D0F800674AA6EE264AB4EEC45AF1EE10FAB0EE2C
:10D10800446A88BFB0EE646ABDEEC66A16EE108A3D
:10D1180016EE107AF045A8BF77468845B8BF0F4687
:10D1280006EE107AB8EEC66A042A80ED036A3DF46A
:10D1380054A995ED106A9DED0E4A25EE866AA4EE77
:10D14800076AB0EE674AA6EE264AB4EEC45AF1EE74
:10D1580010FAB0EE446A88BFB0EE646ABDEEC66AE3
:10D1680016EE108A16EE107AF045A8BF7746884565
:10D17800B8BF0F4606EE107AB8EEC66A052A80EDEB
:10D18800046A3DF42AA995ED146A9DED0F4A25EE2F
:10D19800866AA4EE076AB0EE674AA6EE264AB4EE9F
:10D1A800C45AF1EE10FAB0EE446A88BFB0EE646A71
:10D1B800BDEEC66A16EE108A16EE107AF045A8BFC4
:10D1C80077468845B8BF0F4606EE107AB8EEC66AAD
:10D1D800062A80ED056A3DF400A995ED186A9DEDD3
:10D1E800104A25EE866AA4EE076AB0EE674AA6EEF4
:10D1F800264AB4EEC45AF1EE10FAB0EE446A88BF7B
:10D20800B0EE646ABDEEC66A16EE108A16EE107AA3
:10D21800F045A8BF77468845B8BF0F4606EE107A96
:10D22800B8EEC66A072A80ED066A3DF4D6A895EDE1
:10D238001C6A9DED114A65EE865AE7EE045AE6EE41
:10D24800A57AB4EEE75AF1EE10FAC8BFF0EE647AA8
:10D25800FDF7B3B877EEC76AF0EE477ACEE4454AF1
:10D268004FEA89075FEA9C09384402EBC313274455
:10D2780037D009F101094FEA091903EB090803F14D
:10D28800100200F1100607F1100112ED024A12ED2A
:10D29800035A12ED016A12ED047A56ED024A56ED70
:10D2A800035A56ED016A56ED047A64EE244A65EE97
:10D2B800255A66EE266A67EE277A1032904541EDC8
:10D2C800024A41ED035A41ED016A41ED047A06F143
:10D2D800100601F11001D8D1A9F110094B444844B6
:10D2E8004F441CF0030C3EF478AFB3EC017AF0EC39
:10D2F800017A67EE277ABCF1010CE7EC017AF4D1E8
:10D30800FEF76BBFBEF834309FED1B7A07EE903AFC
:10D31800F8EEE77A194B67EE877AC3ED007AFDF7E6
:10D32800B3B8B7EE007A77EE677AF4EEE75AF1EE23
:10D3380010FA88BFF0EE675A45E407EE906ADFED11
:10D34800106AF8EEE77A66EEA65A9FED0E5A9FED40
:10D358000E6A9FED0E7AA5EE856A26EEA55AA5EE11
:10D36800867AE5EE076A26EEA70AFFF75FB900BFDF
:10D378006C570020D84000206F12833A0400002028
:10D3880084F9223F92E741B99730083C15A82ABE94
:10D3980095ED006A9DED0A4AAE4825EE866AFDEED7
:10D3A800E43AA4EE076AB0EE674AA6EE264A13EE00
:10D3B800907AB4EEC45AF1EE10FAB0EE446A88BF1F
:10D3C800B0EE646ABDEEC66A16EE10CA16EE101A02
:10D3D800F445A8BF71466745C8BF394606EE101A1E
:10D3E800B8EEC66A012A80ED006A3DF439AF95EDC2
:10D3F800046A9DED0B4A25EE866AA4EE076AB0EE34
:10D40800674AA6EE264AB4EEC45AF1EE10FAB0EE18
:10D41800446A88BFB0EE646ABDEEC66A16EE10CAEA
:10D4280016EE101AF445A8BF7146BC45B8BF394678
:10D4380006EE101AB8EEC66A022A80ED016A3DF4BB
:10D448000FAF95ED086A9DED0C4A25EE866AA4EEAD
:10D45800076AB0EE674AA6EE264AB4EEC45AF1EE61
:10D4680010FAB0EE446A88BFB0EE646ABDEEC66AD0
:10D4780016EE10CA16EE101AF445A8BF7146BC4540
:10D48800B8BF394606EE101AB8EEC66A032A80ED10
:10D49800026A3DF4E5AE95ED0C6A9DED0D4A25EE68
:10D4A800866AA4EE076AB0EE674AA6EE264AB4EE8C
:10D4B800C45AF1EE10FAB0EE446A88BFB0EE646A5E
:10D4C800BDEEC66A16EE10CA16EE101AF445A8BFCD
:10D4D8007146BC45B8BF394606EE101AB8EEC66AA2
:10D4E800042A80ED036A3DF4BBAE95ED106A9DED0C
:10D4F8000E4A25EE866AA4EE076AB0EE674AA6EEE3
:10D50800264AB4EEC45AF1EE10FAB0EE446A88BF67
:10D51800B0EE646ABDEEC66A16EE10CA16EE101AB0
:10D52800F445A8BF7146BC45B8BF394606EE101A87
:10D53800B8EEC66A052A80ED046A3DF491AE95ED11
:10D54800146A9DED0F4A25EE866AA4EE076AB0EECE
:10D55800674AA6EE264AB4EEC45AF1EE10FAB0EEC7
:10D56800446A88BFB0EE646ABDEEC66A16EE10CA99
:10D5780016EE101AF445A8BF7146BC45B8BF394627
:10D5880006EE101AB8EEC66A062A80ED056A3DF462
:10D5980067AE95ED186A9DED104A25EE866AA4EEF1
:10D5A800076AB0EE674AA6EE264AB4EEC45AF1EE10
:10D5B80010FAB0EE446A88BFB0EE646ABDEEC66A7F
:10D5C80016EE10CA16EE101AF445A8BF7146BC45EF
:10D5D800B8BF394606EE101AB8EEC66A072A80EDBB
:10D5E800066A3DF43DAE95ED1C6A9DED114A65EE67
:10D5F800865AE7EE045AE6EEA57AB4EEE75AF1EE5B
:10D6080010FAC8BFF0EE647AFDEEE77A17EE901ACA
:10D618008E45A8BF8E468F42D8BF774607EE907AD0
:10D62800F8EEE77AC0ED077AFDF717BE0A494A69AE
:10D63800002A3CF423AA0A6813604B74FCF71EBA4C
:10D64800D4F89C51049B5D1BFFF78CBA034EFCF782
:10D6580095BF00BF6C570020B4560020343200201C
:10D66800002F00F0AB83E04D9DED0A4A95ED006A6E
:10D6780025EE866AA4EE076AB0EE674AA6EE264A49
:10D68800B0EE446A33B1B4EE445AF1EE10FAC8BFB2
:10D69800B0EE646AFDEEE44ABDEEC66A14EE907A16
:10D6A80016EE101A8F4214EE90CA00F3EA84714500
:10D6B800A8BF714606EE101ACC48B8EEC66A012A11
:10D6C80080ED006A3CF48DAE95ED046ADDED0B4A01
:10D6D80025EE866AA4EE876AF0EE674AE6EE264AE9
:10D6E800B0EE646A002B00F0C284B4EEE45AF1EEA6
:10D6F80010FA40F3BC8439467145A8BF714606EE5E
:10D70800101AB8EEC66A022A80ED016A3CF469AEC6
:10D7180095ED086ADDED0C4A25EE866AA4EE876A67
:10D72800F0EE674AE6EE264AB0EE646A002B00F097
:10D738009484B4EEE45AF1EE10FA40F38E8439463C
:10D748007145A8BF714606EE101AB8EEC66A032ADC
:10D7580080ED026A3CF445AE95ED0C6ADDED0D4AAC
:10D7680025EE866AA4EE876AF0EE674AE6EE264A58
:10D77800B0EE646A002B00F06684B4EEE45AF1EE71
:10D7880010FA40F3608439467145A8BF714606EE29
:10D79800101AB8EEC66A042A80ED036A3CF421AE7A
:10D7A80095ED106ADDED0E4A25EE866AA4EE876ACD
:10D7B800F0EE674AE6EE264AB0EE646A002B00F007
:10D7C8003884B4EEE45AF1EE10FA40F33284394664
:10D7D8007145A8BF714606EE101AB8EEC66A052A4A
:10D7E80080ED046A3CF4FDAD95ED146ADDED0F4A59
:10D7F80025EE866AA4EE876AF0EE674AE6EE264AC8
:10D80800B0EE646A002B00F00A84B4EEE45AF1EE3C
:10D8180010FA40F3048439467145A8BF714606EEF4
:10D82800101AB8EEC66A062A80ED056A3CF4D9AD2E
:10D8380095ED186ADDED104A25EE866AA4EE876A32
:10D84800F0EE674AE6EE264AB0EE646A002B00F076
:10D85800DD83B4EEE45AF1EE10FA40F3D78339468B
:10D868007145A8BF714606EE101AB8EEC66A072AB7
:10D8780080ED066A3CF4B5AD95ED1C6ADDED114A04
:10D8880065EE865AE4EE875AE5EEA67A002B00F09C
:10D89800B583F4EEC57AF1EE10FA40F1AF833A465B
:10D8A8007245A8BF7246944607EE90CAF8EEE77A2A
:10D8B800C0ED077AFCF795BDD4F89C51049B5D1B1D
:10D8C800FFF7A9B996ED000A0593039224F02EFC00
:10D8D8004749DFF850E1D1F8EC10DFF84CC1039A62
:10D8E800ACF800008EFB013EC917C1EBAE1107EE84
:10D8F800901AF8EEE77A059BFDEEE77A17EE901A94
:10D90800ACF80210FCF73FBE07EE906ADFED396A0B
:10D918009FED397A84F80462F8EEE77A67EEA67A22
:10D9280077EE876ABDEEE66A16EE103A2033402B92
:10D9380040F2B182DFED316A314BBDEEE77AC3EDDB
:10D94800016A17EE103A2033402B00F2A1829FEDB6
:10D958002D7AF4EEC77AF1EE10FA40F31C84DFED6D
:10D968002A5A9FED2A6A01E0F0EE477AF4EEC67A69
:10D97800F1EE10FA37EEE57AF6DCDFED257AB4EE53
:10D98800E77AF1EE10FA40F10384DFED1F5A9FEDBC
:10D99800216A01E0B0EE677AB4EEC67AF1EE10FAC9
:10D9A80077EE257AF6D49FED147AF4EEC77AF1EE85
:10D9B80010FA40F3BE829FED137A77EE677A67EE2E
:10D9C800A75A9FED155A9FED156A9FED157AA5EE9A
:10D9D800856A27EEA55AA5EE867AE5EE077AC4EDA4
:10D9E800827AFDF7BDBD00BF503600206C5700207D
:10D9F800800F002035FA8E3CDB0FC93F0000000085
:10DA080004000020DB0F4940DB0FC940E4CB16417E
:10DA1800DB0F49C0E4CB16C192E741B99730083C07
:10DA280015A82ABED34D62101032002025EE866A52
:10DA3800A5EE076AB0EE675AA6EE265ABDEEC56A8D
:10DA480016EE100A814200F3B7817045A8BF7046F0
:10DA580006EE100AB8EEC66AB8F1000F00F0B283FD
:10DA6800DD48012A80ED006A3CF4BBAC95ED046A00
:10DA78009DED0B5A25EE866AA5EE076AB0EE675A49
:10DA8800A6EE265ABDEEC56A16EE107AB94200F324
:10DA980091817745A8BF774606EE107AB8EEC66A38
:10DAA800B8F1000F00F08383022A80ED016A3CF48C
:10DAB80098AC95ED086A9DED0C5A25EE866AA5EEA0
:10DAC800076AB0EE675AA6EE265ABDEEC56A16EE8C
:10DAD800107AB94200F36C817745A8BF774606EE05
:10DAE800107AB8EEC66AB8F1000F00F08183032AF5
:10DAF80080ED026A3CF475AC95ED0C6A9DED0D5A0B
:10DB080025EE866AA5EE076AB0EE675AA6EE265A93
:10DB1800BDEEC56A16EE107AB94200F34781774523
:10DB2800A8BF774606EE107AB8EEC66AB8F1000FBD
:10DB380000F05383042A80ED036A3CF452AC95ED5F
:10DB4800106A9DED0E5A25EE866AA5EE076AB0EEBC
:10DB5800675AA6EE265ABDEEC56A16EE107AB94285
:10DB680000F322817745A8BF774606EE107AB8EE13
:10DB7800C66AB8F1000F00F09983052A80ED046A9F
:10DB88003CF42FAC95ED146A9DED0F5A25EE866A8C
:10DB9800A5EE076AB0EE675AA6EE265ABDEEC56A2C
:10DBA80016EE107AB94200F3FD807745A8BF774694
:10DBB80006EE107AB8EEC66AB8F1000F00F04F838F
:10DBC800062A80ED056A3CF40CAC95ED186A9DEDCB
:10DBD800105A25EE866AA5EE076AB0EE675AA6EED9
:10DBE800265ABDEEC56A16EE107AB94200F3AE8029
:10DBF8007745A8BF774606EE107AB8EEC66AB8F140
:10DC0800000F00F00083072A80ED066A3CF4E9ABB8
:10DC180095ED1C6A9DED115A65EE865AE7EE055A98
:10DC2800E6EEA57AFDEEE77A17EE902A914203DC3C
:10DC38007245A8BF7246114607EE901AF8EEE77AC9
:10DC4800B8F1000F7FF434AE089B002B7FF430AEA0
:10DC5800059B079A9342B8BFF0EE647A28E65F4ABC
:10DC68001278032A00F011820022FEF7FEBD9FED14
:10DC7800628AFFF729B99FED608AFFF74DB99FEDDA
:10DC8800580ADFF8708125EE800A24F04FFAD4F89C
:10DC98001451A8F80600FDF7FAB85249096811F0BE
:10DCA80080587EF483AFFEF779BFD4F89C51049B6B
:10DCB8005D1BFDF7E3BF237DFEF723BE93F8FF212D
:10DCC800AA2A7EF40BAED3F8C61149B193F8C22143
:10DCD800A2F10B0001282DD902F0F702062A29D05B
:10DCE800D3F8D61149B193F8D221A2F10B0001283B
:10DCF80020D902F0F702062A1CD0D3F8E61149B160
:10DD080093F8E221A2F10B00012813D902F0F702DF
:10DD1800062A0FD0D3F8F61100293EF4DFAD93F8A8
:10DD2800F231A3F10B02012A04D903F0F703062B01
:10DD38007EF4D4AD41F2FC120123A150A370FEF78A
:10DD4800BEBE294829498046FEF736BA0F4652E733
:10DD5800F7F7B6FA029BDFF89C8093F800E0039B84
:10DD68003178D4F81451C01AA8F80400FEF7BCBAE8
:10DD7800F7F7A6FA029BDFF87C8093F800E0039B94
:10DD8800C01AA8F80200FEF7F1BAF7F799FA029B51
:10DD9800DFF8608093F800E0039BC01AA8F802003F
:10DDA800FEF704BB0F4603E70F46DEE60F46B9E66B
:10DDB8000F4694E60F466FE6084649E60AA9BDEE07
:10DDC800E46A01EB820294460948034D09941A4615
:10DDD80016EE107A434629E06C57002024520020A2
:10DDE8000000C842FC56002058420020E81E0020CF
:10DDF800503600201032002000000000E4CB16410D
:10DE0800DB0F49C0DB0FC940E4CB16C1DB0FC93FAC
:10DE1800DB0F494092E741B99730083C15A82ABE64
:10DE28006145A5EC016A00F110007AD090ED006A16
:10DE3800B1EC014A25EE866AA7EE046AB0EE674A9D
:10DE4800A6EE864AB0EE446A32B1B4EE445AF1EE18
:10DE580010FAC8BFB0EE646ABDEEC66A16EE108A44
:10DE6800474506EE107A04DCF045A8BFF04606EEFA
:10DE7800108AB8EEC66A002BD2D1089C002CCFD1EC
:10DE8800059CA046079CA045B8BFB0EE646AC7E7EA
:10DE98005FED277AA3E5F4EEC77AF1EE10FA40F3C6
:10DEA80074815FED285A1FED2B6A01E0F0EE476A96
:10DEB800F4EEC66AF1EE10FA36EEE57AF6DC5FEDBE
:10DEC800306AB4EEE67AF1EE10FA40F15B815FED6C
:10DED800335A1FED336A01E0B0EE667AB4EEC67AC3
:10DEE800F1EE10FA77EE256AF6D41FED387AF4EEE3
:10DEF800C76AF1EE10FA75DD1FED3B7A77EE666AB8
:10DF080066EEA65A1FED3D5A1FED3D6A1FED3D7A9C
:10DF1800A5EE856A26EEA55AA5EE867AE5EE076A8D
:10DF28000AE5099CFCF75DBAD24F07F18002FEF7BB
:10DF3800C2B99FEDD17AF4EEC77AF1EE10FA44BF78
:10DF48009FEDCE7A77EE677A39E59FEDCD7AF4EEDC
:10DF5800C76AF1EE10FA40F37F81DFEDCA5A9FEDF0
:10DF6800CA6A01E0F0EE476AF4EEC66AF1EE10FA0A
:10DF780036EEE57AF6DCDFEDC16AB4EEE67AF1EE6C
:10DF880010FA40F16681DFEDBF5A9FEDC06A01E0EB
:10DF9800B0EE667AB4EEC67AF1EE10FA77EE256A3C
:10DFA800F6D49FEDBB7AF4EEC76AF1EE10FA05DD00
:10DFB8009FEDB37A77EE666AFFF7C5B99FEDAE7A43
:10DFC800F4EEC76AF1EE10FA44BF9FEDAC7A77EE33
:10DFD800666AFFF7B8B9A8F80600ABF8A850A54CD0
:10DFE800FBF785BB9FEDA47AF4EEC76AF1EE10FA51
:10DFF80044BF9FEDA27A77EE666A81E7FDEEE77A85
:10E0080017EE902ABA42FFF64FAC49E4BDEEC66A55
:10E0180016EE101AB942BFF623AC394623E4BDEE1A
:10E02800C66A16EE101AB942BFF6F6AB3946FFF7C4
:10E03800F6BBBDEEC66A16EE101AB942BFF6C8ABFB
:10E048003946FFF7C8BBBDEEC66A16EE101AB942CC
:10E05800BFF69AAB3946FFF79ABBBDEEC66A16EE15
:10E06800101AB942BFF66CAB3946FFF76CBBBDEE70
:10E07800C66A16EE101AB942BFF63EAB3946FFF72C
:10E088003EBB14EE901AFFF715BB18F031FBFBF7F7
:10E0980027BB1DF0FBFB2369FEF7D3BC02287CF4E9
:10E0A8001AAC41F2B4120123A3546370FCF713BCF9
:10E0B800137C022B7EF417AD92F8FE31552B7EF4BB
:10E0C80012AD92F8FF31AA2B7EF40DADD689E7592F
:10E0D800704B37441F6092F80DE041F210210EF1A9
:10E0E800FF337F2B44F801E03EF6FDACCEF1000390
:10E0F8003EEA03037EF4F7AC4FEA4E2341F21821BF
:10E10800013B6350D08A00B9506A634941F2042345
:10E11800E050B2F811305B0103F2FF135B120B60A1
:10E12800B2F8131001B9116A40001E440644891B55
:10E1380041F2082C40F6F476B1FBFEF1B14244F806
:10E148000C1030D94FF6F476B14228D9032121704A
:10E15800D26A52493B44184441F20C2641F21C232E
:10E168000978A051E25009B923F05AFEA378013387
:10E17800A370FCF7B0BB94F87831002B7BF44CAD5E
:10E18800FBF737BDF0EE476AAFE6B0EE667A96E683
:10E19800F0EE477A07E4B0EE677AFFF7EEBB0222AB
:10E1A80022700022D5E701232370FEF79CBC089B50
:10E1B800002B7FF479AC059B079FBB42B8BFB0EE3C
:10E1C800646A71E4089B002B7FF44AAC059B0798AE
:10E1D8008342B8BFB0EE646A42E4089B002B7FF428
:10E1E800A9AC059B079FBB42B8BFB0EE646AA1E427
:10E1F800089B002B7FF47BAC059B079FBB42B8BFF5
:10E20800B0EE646A73E4089B002B7FF4FCAC059BBA
:10E21800079FBB42B8BFB0EE646AF4E4132B05D184
:10E22800B0EE480A23F082FF069B1880B0EE480A39
:10E23800DBF808321A489847029B1B78132BB0EE7C
:10E24800408A7DF452A823F071FF069B5880FDF7A1
:10E258004CB8F0EE476AA4E6B0EE667A8BE6089B07
:10E26800002B7FF4ADAC059B079FBB42B8BFB0EE57
:10E27800646AA5E4E81E0020DB0FC9BFDB0F49C0B4
:10E28800DB0F4940DB0FC940E4CB1641E4CB16C194
:10E29800DB0FC93F946B0020B46B0020746B002027
:10E2A8009C4B002000C0F84400C0F8C4089B002B19
:10E2B8007FF463AC059B079FBB42B8BFB0EE646AAE
:10E2C8005BE45FED087AB4EEE7EAF1EE10FA66DC9B
:10E2D8005FED0B7AB4EEE7EAF1EE10FA5FD4314B5A
:10E2E800D3ED007AB1EE677AF4EEC7DAF1EE10FA00
:10E2F80052D4F4EEE7DAF1EE10FA88BFF0EE67DAFE
:10E30800294B87ED00CA1B689342BBF6DDAAFBF7D1
:10E3180041BB264A264B10681B689847254BD7ED0A
:10E32800006A93ED007A244BD3ED007A234B83EDFA
:10E33800020A234B67EE277A2B4427EEAC7AD3EDFB
:10E34800007A204B67EE277AF0EE665AEDEEA75A70
:10E3580093ED006AB1EE467AB4EEE57AF1EE10FA82
:10E3680008DCF4EEC65AF1EE10FA8CBFB0EE467A2D
:10E37800B0EE657A144B1B78012B02D0192B7BF475
:10E38800B5ABDFED127AF4EEE7DAF1EE10FACCBFB6
:10E3980001230023FBF7B5BBF0EE47DAB0E7DFED6A
:10E3A8000CDAADE74436002028360020BC350020C2
:10E3B800D035002010350020040000200857002028
:10E3C800E035002048360020D02C0020000096427E
:10E3D800000000002DE9F04F2DED028B95B00646A8
:10E3E80013F0ACF9B74B1D7825B115B0BDEC028B15
:10E3F800BDE8F08FDFF834B3DBF800305805F4D50A
:10E40800B14F3A68002A00F02681B04CD4F8283180
:10E4180003F5F43348339E42C0F01D81DFF81083C2
:10E4280094F82C11D8F80030C4F82861013184F828
:10E438002C11990701F1D68113F0140F41F07B815B
:10E4480013F0080F94F82C3140F07881580701F048
:10E45800B580282B9E4B039301F0A8825E2090473D
:10E468009C4B1B78002B6BD0984C9B4AD4F83031CE
:10E47800F31A934201F20080DFF8B8A29AF80080FC
:10E48800B8F1000F33D1DFF86092D9F80000F7F740
:10E498004DF9C0B201280ED90228904F41F03D83B2
:10E4A8003B78002B41F00D85D4F83831F31AB3F5D9
:10E4B8007A6F81F096858A480268002A40D09AF8D7
:10E4C8000030BBB9874BD9F800001B689B781E3B0E
:10E4D800012B4FF0020141F2028504300BF056FC8B
:10E4E800012200238AF8002084F8443126E07C4881
:10E4F80002682AB3D4F8403140F6B731F31A8B4298
:10E508001ED994F83C31002B01F0FE82013BDBB2AE
:10E5180084F83C31002B01F0D08112F8011B94F8EB
:10E528004471026094F845316F48CA190133006894
:10E5380084F8442184F84531F7F7FCF8C4F84061C1
:10E548006A4A039B12781B68012A03F101030C93A2
:10E5580000F0DF86664B1B786BB1664F3B6853B1A2
:10E56800039B5A4CD3F80090D4F85831A9EB030315
:10E57800632B00F28586DFF8C08198F80090B9F126
:10E58800020F01F07681554F97F87430032B00F095
:10E59800D487594B1B7873B1584D2B685BB14B4CE2
:10E5A800F6F78EFED4F86431049044F61F62C31A5D
:10E5B800934200F20581524B1B78002B4ED1514BF0
:10E5C8001B7843B1414CD4F8B43203F50043E83327
:10E5D8009E4280F018874C4B1B78002B3FF405AF08
:10E5E8003A4E4A4C4A4D06F2BD272068F7F79EF886
:10E5F80000283FF4FAAE2068F7F794F82B788046A5
:10E608005A1E33B120682A70F7F790F80028F2D123
:10E61800EBE603223946781E24F034FD96F8BC3226
:10E6280096F8BD2286F8BF8283F47F4383F0FF0308
:10E638009B1A1FFA88F89BB2B8EB132FD5D196F81E
:10E64800BE22DBB29A42D0D1781E0AF0C7FE2B78E0
:10E6580018442870C9E71E4B039301E72D4C227814
:10E66800002A40F04D862C4F3C78002C40F09380D7
:10E678002A4D2878002841F0AF83144C284DD4F84F
:10E68800AC122A78274B93FBF2F30B449E4296D3A5
:10E6980094F8B032244AC4F8AC62D75CFB0701F1A5
:10E6A800BE84B90701F12E857A0701F1208494F818
:10E6B800B0322978013393FBF1F201FB123384F86D
:10E6C800B0327CE7593B00207C3400200021002038
:10E6D800D4560020EA3B00203F0D03000C00002028
:10E6E80074340020703400206C340020EB3B002090
:10E6F800F83B0020E06B0020003C0020043C002098
:10E70800443C0020553C00200A3C0020103C0020DE
:10E71800143C0020DC3B00204D3C00204C3C0020F9
:10E72800543C0020A0860100503C0020184C0020DA
:10E738000034002078340020E238002013F0030A67
:10E748007FF484AE5E2090473B6814209847184BAE
:10E75800184AB3F9043082FB03124FEAE379C9EB94
:10E76800A2090FFA89F95FFA89F00BF09FFBC9F348
:10E7780007200BF09BFB3B685E2098473B681C20FA
:10E78800984750460BF092FB50460BF08FFB94F8DD
:10E798002C313A685AE6084D286E002841F0E1808D
:10E7A8008146064B87F80090C3F8AC6207E700BFC4
:10E7B8000C340020676666665C3C0020002100205F
:10E7C80094F86A31002B41F08080DC4B1A6802F023
:10E7D8000803002B48F603414AF60B404BF60F435B
:10E7E80049F6074804BF0346884612F0040F4FF065
:10E7F800190118BF9846920684F86A1103D548F49F
:10E80800804848F0200805F04BF8C8F309090028AB
:10E8180041F07685CA4B9F79002F41F070866420BD
:10E828004FF0FF3A4FF0000CADF83E70ADF83CC029
:10E83800CDF842C0CDF846C0CDF84AC0CDF83080FA
:10E84800CDF83480CDF83890ADF840A08DF84E0062
:10E858000CAF0FCFDFF800E384F805C0AEE80F0077
:10E8680097E80F00AEE807002EF8023B71464FF01C
:10E87800010C1B0CFE271F20C82201F81E39A770A7
:10E88800A27184F807C0E07094F87A01207180F0D2
:10E89800F10383EA0313DAB2130983F0E70343EAC7
:10E8A800022383EAC2031BB283EA0312D2B2C3F380
:10E8B800072383EA121343EA022383EAC2031BB243
:10E8C80083F0C80282EA0212D2B2C3F3072383EAB2
:10E8D800121343EA022383EAC2031BB283EA0C073A
:10E8E80087EA0717FFB2C3F3072282EA171242EA40
:10E8F800072200EB0C0382EAC7070EEB0C0084F832
:10E908007A31278011F8013B7B4083EA0313DBB29D
:10E918001A0982EA172242EA032282EAC3031BB2D7
:10E928009FB281422780EDD183F07C0383EA0313F1
:10E93800DBB24FEA131E8EEA172E8EEA032E8EEAFA
:10E94800C30E0FFA8EFE1FFA8EF9DFF810C2A4F874
:10E9580000905FFA8EFE4FEA192984F8289084F80F
:10E9680027E00CF5D17804F1220ADCF80000DCF885
:10E978000410DCF80820DCF80C3047460FC70CF10F
:10E98800100CD445B846F0D1DCF8000038606D4F63
:10E998009CF8043088F8043007F1270884F8C9E1A6
:10E9A80084F8CA9117F8011F2868F6F7C3FEB8451E
:10E9B800F8D194F86B31002B40F08C876249039AA8
:10E9C800097812680A2084F86B01002901F07D811A
:10E9D8005E4F01293888089041F2B1850229B7F8BD
:10E9E80002E001F0A384B8880790032901F0A0850C
:10E9F800F8880690042901F095850529388901F0E1
:10EA08008C850629B7F80A9001F083850729B7F89D
:10EA18000C8001F07B85FB89059394F87A110C92A0
:10EA28000B4683F0300282EA0212D2B21709484933
:10EA3800099387F07A0747EA02270988237187EA4A
:10EA4800C202444FC1EB012187FB013A089B4FF0FA
:10EA5800000C63F30F0C079B6EF31F4C4FF0000E76
:10EA680063F30F0E069BCDF834C012B28A44002718
:10EA7800C91763F31F4EC1EB6A2A059BCDF838E02E
:10EA880082EA021160F30F070020C9B268F30F0091
:10EA9800C2F3072269F31F4782EA111263F31F408A
:10EAA8004FF000090F978DF845A010908DF844900D
:10EAB80042EA01220DF1300C82EAC107BCE80F00DE
:10EAC8003FB287F0C80888EA0818DFF88CE084F8B5
:10EAD80005905FFA88F8C7F30727AEE80F0087EAC2
:10EAE800181747EA08239CE8030083EAC8031BB207
:10EAF80083F023024EF8040B82EA0212D2B2C3F367
:10EB08000723099F83EA1213704643EA022383EA24
:10EB1800C20207F1010C20F814194FF0230816213E
:10EB2800FE27C82384F87AC1228084F807800EF172
:10EB3800020EA770E170A371114611E000340020A5
:10EB4800F0330020A3220020583E00207C770020CC
:10EB580058570020030820800821002002210020A7
:10EB680010F8013B4B4083EA0313DBB21A0982EA2F
:10EB7800112242EA032282EAC3031BB299B270450A
:10EB88002180EDD183F0F40383EA0313DBB24FEA6B
:10EB9800131E8EEA112E8EEA032E8EEAC30E0FFA8A
:10EBA8008EFE1FFA8EF8D44FA4F800804FEA182C76
:10EBB8005FFA8EFE84F81EE084F81FC07968BA6890
:10EBC8003868FB6807F5D178A8E80F0038697969D3
:10EBD800BA6904F2A317A8E8070004F2C11884F878
:10EBE800C1C184F8C0E117F8011F2868F6F7A2FD33
:10EBF800B845F8D194F87271002F40F07486BF4B75
:10EC080094F87AE1B3F90010B3F90220B3F90430AB
:10EC18009FEDBB6A677107EE103A039B1B680C9364
:10EC28008EF06A0383EA031306EE901AD9B20B0931
:10EC380083F0D50343EA012383EAC1031BB283EAC5
:10EC480003115242C9B207EE902AC3F3072383EA9D
:10EC5800111343EA0123F8EEE77AF8EEE66AB8EE14
:10EC6800C77A83EAC1031BB267EE867A66EE866AC4
:10EC780027EE067A002083F0C808CDED0E7ACDED98
:10EC88000D6A8DED0F7A10901190129088EA081C89
:10EC98000DF130095FFA8CFCC3F30728B9E80F00BF
:10ECA80088EA1C1848EA0C2888EACC08DFF86CC205
:10ECB8000FFA88F8ACE80F0088F01E0799E80700FB
:10ECC80087EA0717FFB2C8F3072383EA171343EA53
:10ECD80007238CE8070083EAC7071C20C8214FF0E8
:10ECE80005094FF01E08FE230EF10102E07084F8BA
:10ECF800729184F80780A3700CF10C00A171ACF13B
:10ED0800100184F804E0278084F87A2111F8013B87
:10ED18007B4083EA0313DBB21A0982EA172242EA2C
:10ED2800032282EAC3031BB29FB281422780EDD13E
:10ED380083F0270383EA0313DBB24FEA131E8EEA3C
:10ED4800172E8EEA032E8EEAC30E0FFA8EFE1FFAD6
:10ED58008EF9DFF8A4C1A4F800905FFA8EFE4FEA9E
:10ED6800192984F8259084F824E00CF5D17804F169
:10ED7800220ADCF80000DCF80410DCF80820DCF8D3
:10ED88000C3047460FC70CF1100CD445B846F0D1EB
:10ED98005C4FBCF80030A8F8003007F1240884F86C
:10EDA800C6E184F8C79117F8011F2868F6F7C2FC76
:10EDB800B845F8D194F873310393002B40F08F8550
:10EDC800514B1B68052213F0140F84F8732140F08F
:10EDD800AA86DFED4E7A94F87A81484B4C4AB3F90B
:10EDE8000410B2F906204B4F4B48CDED0E7A88F04F
:10EDF800220383EA03135FFA83FE4FEA1E1383F0AC
:10EE0800590343EA0E2383EACE03B2F5FA6F1BB225
:10EE1800A8BF4FF4FA6283EA031E5FFA8EFEB2F5CA
:10EE28007A7FC3F3072383EA1E13B8BF4FF47A72BD
:10EE38004FF0640C43EA0E23A2F57A720CFB02F23F
:10EE480083EACE0387FB02C780FB01C00FFA83FE6B
:10EE5800D217C9174FF0000AC2EBA712C1EBA001E5
:10EE68008EF0C8070DF13009ADF84220ADF840101A
:10EE7800CDF830A0CDF834A0CDF83CA0CC4687EA38
:10EE88000717BCE80F00FFB2CEF3072E8EEA171E55
:10EE98004EEA072E8EEAC707DFF880E0DCF800C0EC
:10EEA80084F80480AEE80F003FB287F04A0383EA93
:10EEB8000313DBB2C7F3072181EA1311724641EA53
:10EEC800032108F1010881EAC303142042F810C99C
:10EED800FE274FF04A0C002184F87A814FF0C808C9
:10EEE800E07023800EF1040E84F807C0A7706171EA
:10EEF80084F80680184613E0022100200C34002014
:10EF080088C3E43AA3220020003400200000000057
:10EF18007C770020D34D6210676666660821002062
:10EF280012F8011B414081EA0111C9B20B0983EAB9
:10EF3800102343EA012383EAC10109B288B272456A
:10EF48002080EDD181F0140181EA0111C9B24FEAA4
:10EF5800111E8EEA102E8EEA012E8EEAC10E0FFACD
:10EF68008EFE1FFA8EFC4FEA1C2ABF4BBE4884F85F
:10EF78001DA05FFA8EFE84F81CE0BB4F59689A68A2
:10EF88000068DB68A4F800C007F5D17CACE80F0086
:10EF980038697969B7F81880ACE8030004F2A31758
:10EFA800ACF8008084F8BFA1B84684F8BEE104F24A
:10EFB800BF1A18F8011F2868F6F7BCFBC245F8D13C
:10EFC800AA4BAB4A1B781278013B12F00100DBB266
:10EFD80014BFC0214021172B03D8A64A13441B7B1A
:10EFE8000393A54B1A8893071ABF002341F0100119
:10EFF800012312F4027F18BF022312F0100F18BF6A
:10F00800062312F0200F18BF1023002840F0D987DC
:10F018004FF0030C94F87AA10C938AF0460383EA24
:10F028000313DAB2130983F0920343EA022383EA53
:10F03800C2031BB283EA0310C0B2C3F3072282EAF9
:10F04800101242EA002282EAC00212B282F0C80E0E
:10F058008EEA0E1E00235FFA8EFE9DF80C808DF856
:10F0680034800320C2F307228DF837C082EA1E12CB
:10F078008DF835308DF836108DF8380042EA0E2CB0
:10F0880099E807008CEACE0E0FFA8EFEDFF8EC81C5
:10F09800E3718EEA0E1CA8E803005FFA8CFCCEF33D
:10F0A800072E8EEA1C1E4EEA0C2181EACC0C94F83D
:10F0B80008E088F800200FFA8CFC8EEA0C0E8EEA25
:10F0C8000E1E5FFA8EFECCF3072282EA1E1242EA77
:10F0D8000E22607AA17A94F80BC0637182EACE0E90
:10F0E8000FFA8EFE80EA0E0080EA0012D2B2CEF34A
:10F0F800072080EA121040EA022080EAC20000B22B
:10F10800414081EA0111C9B2C0F3072282EA111213
:10F1180042EA012282EAC10212B28CEA020C8CEAAB
:10F128000C1C5FFA8CFCC2F3072282EA1C1242EA2A
:10F138000C2294F80CE0607BA17B94F8109084F882
:10F1480004A082EACC0212B28EEA020E8EEA0E1EE9
:10F158005FFA8EFEC2F3072282EA1E1242EA0E22EC
:10F1680082EACE0212B2504080EA0010C0B2C2F366
:10F17800072282EA101242EA002282EAC00212B290
:10F18800514081EA0111C9B2C2F3072282EA111281
:10F1980042EA012282EAC102E17B13B281EA030258
:10F1A80082EA0212D2B2C3F3072383EA121343EAB4
:10F1B800022383EAC2031BB289EA030282EA02122B
:10F1C800D2B2C3F3072383EA121343EA022383EA82
:10F1D800C2031BB283F0320282EA0212D2B2C3F334
:10F1E800072383EA121343EA022383EAC2031BB20A
:10F1F8009AB24FF0FE0C0AF10101DBB222804FF007
:10F20800090EC82084F802C04FEA122CA8F10E0299
:10F2180084F803E0A07184F87A1184F812C003938B
:10F22800637458F80E0C5168926838F802AC9DF86F
:10F238000C3008F5CA7EAEE8070008F5D2788EF8DB
:10F248000290AEF800A084F8B4C184F8B33117F87E
:10F25800011F2868F6F76EFAB845F8D1049BC4F880
:10F268006431FFF7A8B900BF02210020105900201F
:10F27800EF3A0020743303085C3400200821002092
:10F28800DFF82CA3DFF82C8341200AF0D7FABAF96B
:10F29800023088FB0320DB17C3EBA00080B20AF022
:10F2A800B3FABAF9003088FB0320DB17C3EBA000E0
:10F2B80080B20AF0A9FABAF9043088FB0320DB17F8
:10F2C800C3EBA00080B20AF09FFAA64B3868197801
:10F2D800F6F730FA94F85C3113F0010800F0568420
:10F2E800A14AC4F858910133DBB2A2FB0312D20839
:10F2F80002EB8202A3EB420384F85C31FFF73BB9CF
:10F308009A4B9B491868F6F7E5F900232370FFF735
:10F31800AAB9984F386800283FF41CA94FF0000A92
:10F328002B46DFF89482944C049655469A46F6F795
:10F33800FDF9F8B1F5B94FF001092E463868F6F72E
:10F34800F1F983B27E2B00F0A98298F80120002AF7
:10F358004BD194F84811C1B11B2B84F8482100F017
:10F3680077820D2B47D0386888F80190F6F7DEF9D8
:10F378000028E3D15346AA4650460CAA7F49049E6A
:10F388001D460AF073FAFFF7E5B87D2B00F0938469
:10F3980094F84C2122B180F02003DBB284F84C11A0
:10F3A80094F84721062A10D8B4F84A113868194445
:10F3B800A4F84A11A118013281F8503184F8472184
:10F3C800F6F7B4F90028B9D1D4E7B4F84A2188F897
:10F3D800019013449BB21A0A52FA83F3FF2BA4F844
:10F3E8004A31386802D1664DA1E73868F6F79EF9C8
:10F3F8000028A3D1BEE73868A4F84A21F6F796F9A1
:10F4080000289BD1B6E794F8B832C4F8B462012B4F
:10F4180040F27E8394F8B9225A49981801EB80018A
:10F42800013202F001024F6A84F8B922BFB1564D89
:10F438000D950DF15009123DA52349F8205D802254
:10F4480084F8103115233146484684F8112184F890
:10F458001231B847002840F0E18294F8B8324B4A9C
:10F46800013382FB0312A2EBE37202EB42029B1A06
:10F4780084F8B832FFF7AFB8454A464B92F80BC04C
:10F48800039A1B88D4F83401126843495FFA83FE53
:10F498001F0A4FF47A73121A03FB0CF300209A42E6
:10F4A80081F81EE0CF7781F814E04F7588700871F5
:10F4B80080F01B83394BDFF8F4E01B68384A394881
:10F4C800176800689268C4F830618EFB038CDB17FC
:10F4D800C3EB6C13DFF8DCC08EFB008E8CFB079847
:10F4E8008CFB029CD217C2EBAC0203F5FA734FEA0D
:10F4F800E07C9BB2CCEB6E1CFF1700F5EA4EC7EB25
:10F50800A8070EF1300E8B761B0A0CF1780C4FEA27
:10F518002E2E3030CB764FEA272813120F7781F83A
:10F528001D8081F8202081F8213081F824C081F8DD
:10F5380023E081F82200FEF79FBF1B4B0493186855
:10F54800F6F7ECF800283FF424A8049B012118687A
:10F55800F6F7E0F80222002387F8742088F80030D4
:10F56800FFF717B8A4780020CDCCCCCC483C0020BD
:10F578009C3B002068340020002100204622002007
:10F588005022002074330308252200205655555573
:10F59800243200201C320020183C002004340020B3
:10F5A8006431002008340020FC3900201F85EB510D
:10F5B8000C340020676666660C0000205E209047C9
:10F5C8003B6802209847CA4BCA4A9B6A323382FB7F
:10F5D8000329DB17C3EB69195FFA89F00AF066FCA7
:10F5E800C9F307200AF062FC3B685E2098473B6835
:10F5F80003209847C04B1B78D90740F1A1810EF032
:10F6080083FABE4B9FEDBE7AD3ED037A67EE877A15
:10F61800FCEEE77ACDED037ABDF80C30002800F057
:10F628005684D8B24FEA13290AF040FC48460AF03B
:10F638003DFCB44B1B78042B73D0B34AB4F82E317D
:10F648001178DFF8F4A293FBF1F201FB123292B2C7
:10F65800BAF80030A4F82E211201642092B200FBFF
:10F6680003134900B3FBF1F342EA03295E20C3F315
:10F6780003221FFA89F93B6849EA020998473B685F
:10F68800062098475FFA89F00AF010FC4FEA192023
:10F698000AF00CFC9D49B4F82E214B7ABAF800A068
:10F6A8000132012BA4F82E2100F066864A7B0AEB72
:10F6B8008A031FFA83FA002A40F08D843B685E2093
:10F6C80098473B683A2098478A4BA3FB0A394FEA88
:10F6D80059191FFA89F3D8B203930AF0E7FB039B81
:10F6E800180A0AF0E3FB3B685E2098473B683B201A
:10F6F8009847642303FB19A39BB28548053380FB15
:10F708000320DB17C3EBA000C0B20AF0CFFB002038
:10F718000AF0CCFBDFF81C9299F80630002B40F079
:10F728001E84D8F80030180700F1D98294F82C31DB
:10F738003A68FEF78EBE5E2090473B6830209847B7
:10F74800744BD3F800905FFA89F00AF0AFFBC9F365
:10F7580007200AF0ABFB94F82C3113F003097FF46F
:10F7680018A86D49D4F828216C4B8A421B6840F2CE
:10F77800BA83002BB8BF5B425E4A1BB282FB0312FE
:10F78800D917C1EB62124FF0640909FB12390FFA5D
:10F7980089F913B25FFA89FADAB2C9F30729C3F310
:10F7A80007213B6804915E20039298473B6810202C
:10F7B8009847039A10460AF079FB049908460AF01C
:10F7C80075FB3B685E2098473B6821209847504668
:10F7D8000AF06CFB48460AF069FBD8F800303A6832
:10F7E800FEF72EBEDFF854919FED4D8A04944FF03A
:10F7F800240A5E20904750463B689847494BF9ECED
:10F80800016A9B8A07EE103AF8EEE66AB8EEC77A04
:10F818000AF1010AC6EE877A5FFA8AFA67EE887AF1
:10F82800FDEEE77ACDED037ABDF90C40E0B20AF0BF
:10F838003DFBC4F307200AF039FBBAF1270F01D0CA
:10F848003A68D6E7049CD8F800303A68FEF7F4BD69
:10F858003868F5F76BFF00287FF485AD386884F8C1
:10F86800469188F80190F5F761FF00287FF466ADAE
:10F8780080E5F5F725FD2C4B1B68A0EB030A40F645
:10F88800B8339A4500F25A81284B1B793A2B00F07D
:10F898007D84002388F80030FEF77BBE386884F842
:10F8A800466184F8476184F8489188F80160F5F763
:10F8B8003DFF00287FF442AD5CE594F8441194F8CC
:10F8C80045311B484A1CFEF731BE013B84F86A31BA
:10F8D800FFF76FB8013B84F86B31FFF78BB9013B39
:10F8E80084F87331BAE4013F84F87271FFF762BAA1
:10F8F8002C5700201F85EB51EF3A002034320020AE
:10F90800CDCC4C3E2452002032320020243200203C
:10F9180067666666083400203F4B4C0004340020BC
:10F9280000007A4414340020E8380020D038002041
:10F938006C340020F03300201C32002044340020B6
:10F94800844A854BB2F80890A3FB09394FEA990914
:10F958005FFA89F00AF0AAFA4FEA19200AF0A6FA23
:10F9680067E60024DFF81C82A1464FF0500A02E047
:10F97800DBB283F3118815F804B0601C594628449B
:10F9880009F056FE002840F00B820BF101031C44DD
:10F99800EFF311838AF312882A6E9442E8DB00227F
:10F9A800DBB22A6683F31188FEF7FBBE4FF0000A2C
:10F9B8005E20D3F8008084F82CA190473B68DFF8DC
:10F9C800C8911720984750460AF070FA634BA3FB7A
:10F9D80008239B0BA9FB03125209C2EB0212A3EBEB
:10F9E8008203D8B20AF062FA3B685E2098473B6807
:10F9F800182098475A4BA3FB08239B09A9FB03121D
:10FA08005209C2EB0212A3EB8203D8B20AF04EFAF3
:10FA180050460AF04BFA3A68FEF720BD0C9EAE42FB
:10FA28004FF000014FD941F2210015F8013B81EA5E
:10FA380003235A0013F4004F80EA020192B289B2FC
:10FA480008BF11464A0080EA020311F4004F99B238
:10FA580093B218BF0B46590080EA010213F4004F15
:10FA680089B293B208BF0B465A0013F4004F80EADC
:10FA7800020192B289B208BF11464A0080EA020325
:10FA880011F4004F99B293B218BF0B46590080EA9F
:10FA9800010213F4004F89B293B208BF0B46590014
:10FAA80013F4004F80EA010289B292B208BF0A46F5
:10FAB800530080EA030112F4004F9BB289B208BFD9
:10FAC8001946B542B1D14846F2F716F825490C9DBA
:10FAD80025486D1A152DA8BF15252A4623F0C7FA03
:10FAE800224A94F8B8321570B9E4214B039A1B786E
:10FAF8001268C4F83421013B012B3FF6DBAC10221D
:10FB080002238A700B71D5E40AF076F9FEF716BD68
:10FB1800184A02EB8302576A88E40AF05DF9012368
:10FB28003B70FEF7C8BC144B9FED147AD3ED007AF6
:10FB3800F8EEE77A67EE877AFFF74DB9104AB2F820
:10FB48005E3100210133A2F85E3188F80010FEF71B
:10FB580020BD00BFF0330020CDCCCCCC73B2E7453C
:10FB6800D34D6210102200209C3F0020B13F00209E
:10FB78002452002074330308043400200AD7233C9D
:10FB880000210020CD16020889888888894B1B88A7
:10FB9800DA0515D4D80600F1D183990600F1E98376
:10FBA8005A0600F1FC83180700F1FF83D90700F11A
:10FBB800F98313F0020F0CBF4FF004084FF00C0844
:10FBC8007D4B7E4A1B78D27803F001030AB143F0DB
:10FBD80002035320049309F031FE794A128802EB9C
:10FBE800820202EB8202900080B209F00DFE002032
:10FBF80009F00AFE7349744AB1F800A03868CAEBE4
:10FC0800CA1A4FEA4A0A82FB0A3252444FEAEA7A8F
:10FC1800CAEB622A5FFA8AFA5146F5F78BFD6B4BFD
:10FC280038681A78049B48EA0308684B8AEA020A8B
:10FC3800002183F800A0F5F77DFD41463868F5F707
:10FC480079FD624B614A1B78386888EA0303DBB2A6
:10FC580019461370F5F76EFD94F85C31002B7FF4AC
:10FC68003FAB4F2009F0EAFD1FF0CAF81FF0C8F8B3
:10FC78001FF0C6F801213868F5F75CFD544A534B6C
:10FC880092F800801B78514A386808F0010883F020
:10FC9800010341461370F5F74DFD4C4B4B4A1B7859
:10FCA800386888EA030319461370F5F743FD94F89A
:10FCB8005C31FFF715BB386884F84C91F5F736FDD1
:10FCC80000287FF43BABFFF755BB884689460846BA
:10FCD800069107918E4608910591FEF79EBE0CA9E4
:10FCE8003C480AF0A7F83B685E2098473B68132019
:10FCF8009847BDF930805FFA88F00AF0D7F8C8F362
:10FD080007200AF0D3F83B685E2098473B681B2021
:10FD18009847BDF932805FFA88F00AF0C7F8C8F34F
:10FD280007200AF0C3F83B685E2098473B68232009
:10FD380098474E200AF0BAF800200AF0B7F80CA944
:10FD480024480AF077F83B685E2098473B68122001
:10FD58009847BDF930805FFA88F00AF0A7F8C8F331
:10FD680007200AF0A3F83B685E2098473B681A20F2
:10FD78009847BDF932805FFA88F00AF097F8C8F31F
:10FD880007200AF093F83B685E2098473B682220DA
:10FD9800984745200AF08AF800200AF087F8C5E459
:10FDA80041463A2009F0A0FB40EA09095FFA89F9BF
:10FDB800EBE500BF5C340020EF3A0020783E0020DD
:10FDC8001C3200205857002003082080A478002007
:10FDD8000457002080969800B749B84B0093A1F1CA
:10FDE8003F07B74BB74A0B9101F8404C0CA8B649EE
:10FDF8000A97F1F759FF0A9F7B1C0A933C700A9BEC
:10FE08002922591C0A911A700A9BEA22591C0A9144
:10FE18001A700A9BC822591C0A910CA81A7021F062
:10FE2800B5F800F101080CA942460A9823F01FF919
:10FE38000A9A02EB080301330A9302F808400A9B66
:10FE48005A1C0A921C700A9B5A1C0A921C700A9B24
:10FE58005A1C0A921C700A9B5A1C0A921C700A9B14
:10FE68005A1C0A921C700A9B5A1C0A921C700A9B04
:10FE78005A1C0A921C700A9B5A1C0A921C700A9BF4
:10FE88005A1C0A921C700A9B5A1C0A921C700A9BE4
:10FE98005A1C0A921C700A9B5A1C0A921C700A9BD4
:10FEA8000122991814A80A911A7050F8283DDB1BF2
:10FEB8003B7011F0EDFB854B2C70C3F8AC62FEF77C
:10FEC8007EBBC4F8386187F80080FEF7F4BADBF827
:10FED8000020D2067FF5A5AB8146FFF7A5BBF5F755
:10FEE80019FCFEF7FDBACA4649464A4659E4724B20
:10FEF800774A0D93A3F140081268002103F8401CCB
:10FF0800212388F80230D30040F127827149032762
:10FF1800714B1B88580500F11D82DA0700F13C82FD
:10FF280003F002036D4A002B1CBF03271146DFF8BC
:10FF3800C8913A46484623F09AF807EB090314A8F3
:10FF48000133A9F1020140F8203D00225B1A07F8AD
:10FF5800092088F8013011F09BFBFEF7A8BB3B682D
:10FF6800DFF898A15E2098473B6828209847DAF880
:10FF780000305B4A82FB0312DB17C3EBA203D8B243
:10FF8800039309F093FF039BC3F3072009F08EFF47
:10FF98003B685E2098473B6804209847B9F80830CA
:10FFA800002B40F0CE81DAF8083083F310095FFAAD
:10FFB80089F009F07BFFC9F3072009F077FFFFF705
:10FFC800B0BB484AD278002A0CBF4FF0040C4FF05F
:10FFD800050CFFF71FB8444B1B789AFBF3FAFFF7A1
:10FFE8006DBB0123D9F800003B70F5F79BFB074672
:08FFF800D9F80000F5F796FBB3
:020000040801F1
:1000000079067EF45CAA8E287EF459AA9AF800300C
:10001000002B7EF470AA374B374A1A602D2384F8E0
:100020003C31FEF753BADFF8E0909FED348AB9F91E
:100030000230234A0D9207EE903AF8EEE77A0DF17E
:10004000500867EE887AA2F14003FDEEE77AA2F14C
:100050003D0148F8201D02F8400C0822CDED037A3E
:100060005A701E229A70BDF80C104046F1F722FD1E
:10007000B9F9003007EE903AF8EEE77A404667EEBD
:10008000887AFDEEE77ACDED037ABDF80C10F1F732
:1000900011FDB9F9043007EE903AF8EEE77A4046E0
:1000A00067EE887AFDEEE77ACDED037ABDF80C10A5
:1000B000F1F700FD404611F0EFFAFEF7F6BA00BF87
:1000C0009C3B00202E3E0020545C03085C5C03082F
:1000D000685C030800210020FC560020405C0308F7
:1000E0005C340020505C030867666666783E00203A
:1000F0003232002074340020183C002058A08B417C
:100100005F3B0020643100200C340020AA4AAB4B36
:100110000D920DF15008A2F13D0048F8200D19880C
:10012000DFF8A892A2F1400300204FF00A0E02F877
:10013000400C082283F801E040469A70F1F7BAFCBF
:10014000D9F800309E49DA1781FB0313C2EBA303F1
:1001500099B24046F1F7AEFC03F0B4FBD9F8089031
:100160000C9B4FEA1942591C0C911A700C9B4FEAD8
:100170001922591C0C911A700C9B5A1C0C9283F872
:1001800000900C9B5A1C0C921870404611F084FA97
:10019000FEF78EBA8B4B997818460FF0EFFE0028C9
:1001A0007FF47BAB854A884F884B12888849894CFD
:1001B0008948FA611A6809689B68FA62B4F85E2196
:1001C0000490C7F86CA0FB640068F963FA65F3F764
:1001D00003FB824600287EF4DBA9049B494618688D
:1001E000F5F79CFA774A94F86031D2780692642B3E
:1001F0004FF0040287F8742040F0008194F86131D8
:10020000072B08BF84F861A194F86131089307EBCC
:100210000319D9F804100591084620F0BBFED9F85F
:10022000081007915FFA80F9084620F0B3FE5FFAE4
:1002300080FA089B69480599059009EB0A02083283
:10024000C27123F00F028272644A03F00F035373EA
:10025000624B0AEBC900987318464A460F3022F0E9
:100260000AFF5F4B079909F109001844524622F032
:1002700002FF0598C37903F10109CBB1013B5FFA95
:1002800083FC0CF1080CDFF870E184440023073094
:1002900010F8012B5A409300D10883EA420301F081
:1002A000180153404EFA01F253408445DBB2EFD1BE
:1002B0004B4A069809F8023021F0E4FD94F86131C8
:1002C0000022013384F8613184F86021059BDDF858
:1002D00014909B785BB1049B19F805101868F5F72A
:1002E0002DFA013599F80230EDB2AB42F3D894F80B
:1002F00060310322013384F8603187F8742088F874
:100300000020049BFFF71FB92C4B364A1B889279BB
:1003100003EB830303EB83039F00BFB2002A00F0CB
:100320001B812A4B1B680FFA83FA03F0CBFA40B209
:10033000FEF77CBA984699461846069307930593AC
:10034000FEF76FBB4FF034083EE403F0BBFA09F050
:10035000B1FD002009F0AEFDFFF7E7B90327224900
:10036000E9E5DBF80030214A214903F48003002B42
:1003700016BF114604270327CEE54FF0240823E4D7
:100380003B685E2098473B68392098475FFA8AF0BF
:1003900009F090FD4FEA1A2009F08CFDFFF7BEB975
:1003A00014490427C7E54FF010080DE44FF0080882
:1003B0000AE44FF0200807E49C3B00201C32002098
:1003C00067666666D03800200C000020643100208B
:1003D0000434002000210020FC390020B86B0020EC
:1003E000BE6B0020F0330020445C0308405C03082F
:1003F000385C0308485C03080007090E97F87590FD
:100400005849594A059219F00F0F04BF09F1010923
:100410005FFA89F9B9F1070F28BF4FF001094FEAD8
:10042000091A07EB0A035FFA8AFC187C0023095CAF
:10043000937202F10D0307EB0A024CEA0000012956
:100440001870D26803F1010E0CD90239C9B2881CA8
:100450001844734603F8012B83424FEA1222F9D164
:1004600001318E44BA4422F0600309F101099AF87F
:1004700011205FFA89F91343B9F1080F8EF80030A3
:100480000EF101036BD04FEA091A07EB0A01374A54
:10049000087C3449095C9A1A02EB010E0CF1100C2D
:1004A000BEF1130F5FFA8CFCC5DDD2B2931DDBB237
:1004B0000598DFF8C4E043F04001C17103F1010C7D
:1004C000CBB105325FFA82FA0AF1080A82440023AE
:1004D0000EF1010010F8011B59408B0083EA410323
:1004E000CA084B40224902F0180241FA02F2534076
:1004F0008245DBB2EED106980CF80E3087F8759085
:1005000021F0C0FCE2E61B4B0746B3F900A06420D3
:10051000FEF78CB90593FEF784BA98460593FEF76B
:1005200080BA984699460593FEF77BBA9846994655
:1005300018460593FEF775BA9846994618460693ED
:100540000593FEF76EBA98469946184606930793A8
:100550009E460593FEF765BA4FF0FF33E3E6034A84
:100560009A1AA2E774330308B86B0020C56B002009
:100570000007090E64310020BE6B00202DE9F04712
:10058000B0F908400C81E4B2442C8CB00D4600F068
:10059000058406462FD9812C00F0508300F281801B
:1005A000542C00F0AD8040F2B7806E2C00F08083B8
:1005B000802C40F0B380924B1C780B3C14F0FF046D
:1005C00012D0904F00220A2629683B88481C2860D8
:1005D0000E702968FF2B02F10102A8BFFF23481CFF
:1005E000A24228600B70EFDB0124234620466B817A
:1005F0000CB0BDE8F087052C00F0BE831ED8022C9D
:1006000076D040F2EB80032C00F0AD83042C40F058
:1006100085807D4928462246F1F742FA0021284686
:10062000F1F76EFA2A680021531C01242B60204642
:10063000234611706B810CB0BDE8F087242C55D097
:1006400040F28480282C00F05383382C66D10A684D
:100650006E4B0124511C296014702A680521101961
:10066000286011702A680A211019286011702A6800
:1006700000211019286011702A6819781019286053
:1006800011702A6859781019286011702A689978B1
:1006900013192B602346117020466B810CB0BDE806
:1006A000F087A02C10D06FD9B82C00F05A83FE2C04
:1006B00034D1574C04F1080634F8021B2846F1F7F0
:1006C0001FFAB442F8D18FE7524B08461968F1F788
:1006D000FFF9514B28461968F1F7FAF94F4B1968A1
:1006E00028460124F1F7F4F923467FE74C4BF6E75F
:1006F00004224C4928460124F1F7D2F92346CBE7DE
:100700000B6800215A1C2A6019702A6801241319E9
:100710002B6023461170BFE7522C83D02946204618
:1007200001F0A6FB014600287FF45EAF742C00F0B8
:100730007B82772C40F08480336872689A4240F064
:100740003983394A284616F09FF94DE7202CE5D128
:100750000B68364C591C627829601A702B68227815
:10076000591C29601A702B68A278591C29601A70CC
:1007700021892846F1F7C4F92B686279591C296050
:100780001A702A68A1794FE7822CC7D10B68284AD2
:10079000284C1178254A581C286019701189284660
:1007A000F1F7AEF9244B2A681B88FF2B02F10101F7
:1007B000A8BFFF2329601370A16881F3100189B2DB
:1007C0002846F1F79DF9216801F30F0189B2284607
:1007D000F1F796F9194B2A68197825E7012C9DD174
:1007E0000B680022591C29601A702B685A1C2A6059
:1007F0001C702A682521531C2B60234611704BE77F
:10080000BA310020382400202E3E0020732D002015
:1008100010320020ACF7FF1FB0F7FF1FB4F7FF1F27
:10082000E4550020D45C0308495C0208F033002042
:1008300032320020643100201C320020245200207B
:10084000292C376800F0BA82392C01F09780212CCE
:1008500001F0748072680B3CD31BEF2C00F25B87B5
:1008600001A050F824F000BFD9170108171701089C
:10087000171701081717010817170108171701089C
:10088000171701081717010817170108171701088C
:10089000171701081717010817170108171701087C
:1008A000171701081717010817170108171701086C
:1008B000171701081717010817170108171701085C
:1008C00017170108171701086F18010817170108F3
:1008D0005518010817170108DF1801081717010834
:1008E0001717010817170108A7160108171701089D
:1008F00083170108171701081717010817170108B0
:1009000017170108171701087117010817170108B1
:100910002117010817170108CF160108171701083A
:10092000171701081717010817170108E90501082B
:1009300017170108291801081717010817170108C8
:100940000F180108171701080913010817170108E4
:1009500017170108171701081717010817170108BB
:10096000171701081717010817170108C9120108FE
:10097000171701081516010817170108171701089E
:10098000291501081717010817170108171701087B
:10099000171701081717010817170108171701087B
:1009A0006715010817170108B51401081717010882
:1009B0004B14010817170108A9130108171701089C
:1009C00081130108631301088B160108171701082A
:1009D000171701081717010817170108171701083B
:1009E000171701081717010817170108171701082B
:1009F000171701081717010817170108171701081B
:100A0000171701081717010817170108171701080A
:100A100017170108171701081717010817170108FA
:100A200017170108171701081717010817170108EA
:100A300017170108171701081717010817170108DA
:100A400017170108171701081717010817170108CA
:100A500017170108171701081717010817170108BA
:100A600017170108171701081717010817170108AA
:100A7000171701081717010817170108171701089A
:100A8000171701081717010817170108171701088A
:100A9000171701081717010817170108171701087A
:100AA000171701081717010817170108171701086A
:100AB000171701081717010817170108171701085A
:100AC000171701081717010817170108171701084A
:100AD000171701081717010817170108171701083A
:100AE000171701081717010817170108171701082A
:100AF000171701081717010817170108171701081A
:100B00001717010817170108171701081717010809
:100B100017170108171701086116010817170108B0
:100B20006112010837120108171701081717010889
:100B300017170108171701081717010817170108D9
:100B400017170108171701081717010817170108C9
:100B5000171701081717010817170108DB110108FB
:100B600017170108A3110108171701080711010839
:100B7000ED100108E70F010817170108CD0F010854
:100B800017170108A50F0108930F0108350F010879
:100B900017170108B10E01081717010817170108E8
:100BA0008F0E0108630E0108651001083D10010851
:100BB000171701081B100108171701080310010877
:100BC0001717010817170108171701081717010849
:100BD0001717010817170108171701081717010839
:100BE0001717010817170108171701081717010829
:100BF0001717010817170108D31001081717010864
:100C000017170108791001081717010817170108AD
:100C100017170108FF0D010817170108171701081A
:100C200017170108E70D0108336872689A4240F00F
:100C3000BD80AB4A284615F027FFD5E4A94B1E78A6
:100C40000A3E16F0FF063FF4CFACA74BA74F1E4459
:100C500003F101080A2314E0502B00F05186002410
:100C600021462A68501C286028461370F0F748FF78
:100C700021462846F0F744FFB0453FF4B5AC18F8DC
:100C8000013B0A2BE8D19A4A9468116804EB84046A
:100C90004FF6FF7264009442A8BF14469142A8BF69
:100CA000114624EAE47421EAE171A4B289B2D8E7DA
:100CB000904B0A681B88904CFF2BA8BFFF23511C48
:100CC00029601370A16881F3100189B22846F0F7FA
:100CD00017FF8A4B28461988F0F712FF216801F3A5
:100CE0000F0189B228460124F0F70AFF2346D3E416
:100CF0000B68DFF83C82824E591C022229601A7070
:100D00002B6806275A1C2A601F702B680A22591C60
:100D100029601A702B6801241A192A601C70B8F80F
:100D200000102846F0F7ECFEB8F802102846F0F75D
:100D3000E7FE2B681A192A601F702B6850221919B8
:100D400029601A702B680022191929601A703188DD
:100D50002846F0F7D5FE71882846F0F7D1FE2346E5
:100D60009AE4684BBBE40B685A1C0A601C700B6861
:100D70005A1C0A601C7055E40B2263492846F0F7A0
:100D80008FFE082261492846F0F78AFE01240722D7
:100D90005F492846F0F784FE23467DE4002A3FF4AD
:100DA00023AC5C4B13600124234675E45A1C32606B
:100DB00019783EE75A1C32601978C2E47B1C336014
:100DC0003B780A2B00F0EA85502B40F0C282304677
:100DD000F0F754FE4A4F38803046F0F74FFE0124BA
:100DE0007880234658E44C4B1B78DB0700F1938452
:100DF0000124F2F7A7FEF3F781F823464CE43046CE
:100E0000F0F73CFE3368ADF80C001A46591C31600F
:100E100012F8021B32608DF80E105A788DF80F20F0
:100E2000DA1C32609A788DF810201A1D3260DA7858
:100E30008DF811205A1D32601B798DF8123003A8ED
:100E40000023ADF81430F0F771FD344A344B1268CA
:100E5000801A4FF0010461F10001C3E90201234649
:100E60001AE43A467B1C33602E4B12F8021B1970B1
:100E700032607A785A70FA1C3260BA789A703046CA
:100E8000F0F7FCFD284B0124D880234604E43046CB
:100E9000F0F7F4FD244F38803046F0F7EFFD78800E
:100EA0003046F0F7EBFD0124B8802346FFF7F4BB92
:100EB000DFF8308098F80030002B3FF495AB1B4FE3
:100EC00000243046F0F7DAFD0CF016F898F8003000
:100ED000A7EC010A01349C42F3DBFFF785BB00BF9E
:100EE000A15C0208BA310020A83303082C2400209A
:100EF000F42300201C3200206431002058570020C9
:100F000028240020F8530020DC5C0308E85C030878
:100F1000F45C0308BD1B0108EF3A0020D456002002
:100F2000C0230020B8550020D83600202C520020C5
:100F3000B05500200D2B40F0EE837B1C33603C78D5
:100F4000072C00F2E883DFF8788330460C27F0F7AF
:100F500095FD07FB04F708EB0704A0803046F0F787
:100F60008DFDE0803046F0F789FD336820811A4618
:100F7000591C316012F8021BA17232605B78E37277
:100F80003046F0F763FD012448F807002346FFF7D9
:100F900083BB3046F0F772FDB74B0124188023461F
:100FA000FFF77ABB7B1C33603878060600F1678553
:100FB000B24B1B78DC073FF517AB032828BF002096
:100FC0000124F2F783FD2346FFF766BBAB4B1B788A
:100FD000D8073FF509AB0124F2F794FDF2F78EFF35
:100FE0002346FFF759BBA54B1B78DA073FF5FCAA50
:100FF000A34A1378012443F0040313702346FFF738
:101000004BBB3046F0F73AFD9E4A00EB80004300B0
:10101000012413802346FFF73FBB3046F0F72EFD37
:10102000994F38823046F0F729FD78823046F0F744
:1010300025FD0124B8822346FFF72EBB3B467A1CD0
:101040003260924A13F8021B11703360904A7B7829
:101050009370FB1C33608B4BBA789A700124234643
:10106000FFF71ABB8B4B8C4918684E22012422F0E3
:1010700002F82346FFF710BB7B1C33603B780F2B35
:1010800000F24983BA1C3260C3EBC303834A797808
:10109000D154F91C31601344BA785A703A1D326049
:1010A000FA789A707A1D32603A79DA70BA1D326035
:1010B0007A791A71FA1D3260BA795A7107F1080209
:1010C0003260FA799A71012406F016FA2346FFF786
:1010D000E3BA3046F0F7D2FC6D4FF8813046F0F7B6
:1010E000CDFC0124B8812346FFF7D6BA634B1B78A9
:1010F000D9073FF579AA6A4B4FF4C87201241A80C8
:101100002346FFF7C9BA092B40F30583DFF8B48102
:101110003B467A1CD8F80040326013F8022B22704C
:1011200033607B78A370FB1C3360BB78642BA8BF53
:1011300064233A1D63713260FB78642BA8BF64237B
:101140007A1DA37132603B79E371BB1D33607B79FB
:10115000642BA8BF6423FA1D23723260BB79E3704D
:1011600007F108033360FB7923713046F0F786FC02
:10117000726833686081D11A00290CDD591CD8F8D7
:1011800000003160521A002A1978417203DD9A1C5E
:1011900032605B78437001240CF018FD2346FFF7A2
:1011A0007BBA3C4B1868FB1C02462137991E316004
:1011B00013F8031C1170591E316013F8021C517092
:1011C000336013F8011C917003339F4202F1030254
:1011D000ECD10BF061FDFFF707BAC3F34704122C03
:1011E00000F29982BCB10CAB0DF10A0803EB440983
:1011F0004746A9F126093046F0F740FC27F8020FD0
:10120000B945F8D1274B38F8022F23F8022F47456C
:10121000F9D1112C09D8244A6300023B1344002160
:10122000223223F8021F9A42FBD1204A01231C4696
:101230001370FFF731BA7B1C1D4933600A783B7885
:10124000002A40F0E58304220A701A4A9B001380AA
:10125000F4F73AF8184B012418612346FFF71CBA3B
:10126000164F002330463B60F0F7F0FB0124386056
:101270002346FFF711BA00BF8E200020EF3A00206E
:1012800004570020D0550020184E00207C49002033
:10129000C055002060340020443803080C5300205F
:1012A000E87D0020D2370020D4370020F837002016
:1012B0004240002058570020C0230020F85300204F
:1012C0004C520020643400203B467A1CBF4C3260F4
:1012D00013F8022B227133607B7863713046F0F78C
:1012E000CDFB336820805A1C32601B78A3713046D6
:1012F000F0F7C4FB336860805A1C32601B78E371DE
:1013000001242346FFF7C8B97B1C3360B04B3A7801
:10131000DFF8F4821A700023C8F800303046F0F786
:1013200095FB3268D8F80030AA49AB4C0343501CF7
:10133000C8F80030306013780B723046F0F79EFB2F
:1013400020603046F0F79AFB60603046F0F796FB7D
:10135000A0603046F0F792FB3046F0F78FFBFFF7C6
:1013600043B99E4B1B7813F0010140F0D4817B1CE4
:1013700033603878012402F0A9F92346FFF78CB9CD
:101380003B467A1C3260964A13F8021BD1703360D8
:10139000944A7B785371FB1C3360934BBA78DA70B4
:1013A00001242346FFF778B93046F0F767FB304653
:1013B000F0F764FB3046F0F761FB3046F0F76AFB6C
:1013C00033688A4C1946581C2268306011F8020BA9
:1013D00082F82C003160597882F83610D91C3160BF
:1013E0009B7882F837303046F0F754FB3046F0F700
:1013F00051FB3046F0F74EFB30462768F0F73EFBD6
:10140000788730462768F0F739FB33687268388789
:10141000D11A01290ADD591C226831601B7882F833
:101420002E303046F0F736FB33687268D31A032B40
:1014300009DD30462768F0F721FB788630462668BC
:10144000F0F71CFBB0862068C3E67B1C3360674C5A
:10145000DFF8B8813B7888F8053030462768F0F728
:101460000DFB388430462768F0F708FB7268336854
:10147000F883D11A072900F33D83D11A032900F319
:101480002C83D21A002A05DD591C226831601B7892
:1014900082F82630F2F794FC15F064FB544B1B687D
:1014A000002B00F0E182206801240BF065F8234650
:1014B000FFF7F2B83B467A1C3260DFF8508113F830
:1014C000022B88F8022033604A4A7B781370FB1C99
:1014D0003360494CBB7823713B1D3360FB78092B8B
:1014E000A8BF09233046A370F0F7C8FA33687268C2
:1014F0002080D11A012905DD3046F0F7BFFA3368A4
:101500007268E0819A4240F0D282F2F759FC336867
:1015100072689A423FF468A85A1C32601B78E370E4
:1015200001242346FFF7B8B8344B1B78012B3FF654
:101530005BA87B1C39463360DFF8D48011F8023B8E
:1015400088F80230FB1CD21A3160012A78783360A7
:1015500040F3A0823046F0F791FA0124A8F8000089
:101560002346FFF799B8264B1B68002B3FF43CA895
:1015700012F05EF8FF283FF437A83046F0F77EFA05
:101580003F2840F29D821F4F00243C7033687268F0
:10159000B880D21A012A7FF727A81A46591C316051
:1015A00012F8021BB9700CA8326000225C7800F8B7
:1015B000242D12F00FF89DF80C30A3423FF414A82C
:1015C000204612F02BF8FFF70FB800BFF4360020CA
:1015D00010590020E8790020F0290020EF3A00207F
:1015E000C0550020283D0020D05500206034002048
:1015F000F8580020B4550020184E0020A42E0020DA
:10160000F43A0020F83A0020E45500207C490020FC
:10161000A62E00207B1C336097F80080B8F1110FD4
:1016200079D8BB1C3360B84C7B7804F8183030464E
:10163000F0F724FA40F6CA039842A8BF184640F2D1
:10164000EE23984204EB4801B8BF18460124A0F2EB
:10165000EE222346192092FBF0F24A70FFF71CB8E5
:101660003B467A1C326013F8024B3360FB1C7878DF
:101670003360B978002C00F05482012C7EF4B4AFB2
:1016800002F0E2F82346FFF707B87B1C33603B7893
:10169000002B00F0E0814FF40040012401F0BAFB80
:1016A0002346FEF7F9BF7B1C3360984938780870F1
:1016B000D21A002A7EF798AFBB1C33607B780033C8
:1016C00018BF012301244B702346FEF7E5BF072214
:1016D000B3FBF2F2C2EBC2041B1B1CD1D2B202F16B
:1016E000FF385FFA88F8002A3EF47EAFDFF82092D8
:1016F00008F101081C467B1C3360854B97F90010EC
:10170000002793F902208A4203F1080300F05B816D
:101710000137052FF5D14FF0FF342346FEF7BCBF4C
:101720007B1C33603B780E2BF5D8BA1C326078787E
:101730000328F0D87749062202FB03F28B18FC1C21
:1017400058713460B87888543A1D3260FA785A700B
:101750007A1D32603A799A70BA1D32607A79DA70FD
:10176000FA1D3260BA791A7101242346FEF794BF3C
:101770007B1C3360684B3A785A7501242346FEF788
:101780008BBF7B1C644C33603B7823723046F0F790
:1017900075F9A0833046F0F771F920833046F0F7F1
:1017A0006DF932686083531C33601278E27472689A
:1017B000D31A032B00F330813368D11A052900F3C3
:1017C000B681D21A002A7EF70FAF5A1C32601B78FE
:1017D00084F82130FEF708BF5049102B4FF000026B
:1017E00028BF10230A604A608A60CA600A74002B0E
:1017F0003EF4FAAE3268013913440132326012F815
:10180000010C01F8010F9342F7D1FEF7EDBE444BF6
:1018100007F108020137376017F8011C03F8011FB0
:10182000BA42F7D1FEF7E0BE3B46791C31603D4934
:1018300013F8020B887033607878487093423EF456
:10184000D3AEFB1C3360384BBA781A71012423469F
:10185000FEF722BF354F00233B603046F0F7F6F825
:101860003B68012403433B602346FEF715BF7B1C06
:1018700033603C780191132C3FF64DAFBB1C3360B5
:10188000787815F03BF900283FF445AF284B0278F3
:1018900003F82420FA1C326003EB8404BA786270E7
:1018A0003A1D3260FA78A2707A1D32603A79E2709D
:1018B00003F15000019902E00433984207D01A78EE
:1018C000002AF9D19C78DA789442F5D20121194B9B
:1018D00081F00101012419702346FEF7DDBE304678
:1018E000F0F7CCF8144F38603046F0F7C7F878605E
:1018F0003046F0F7C3F80124B8602346FEF7CCBEAB
:10190000BC683968FFF7C2B96C3A00201059002052
:10191000147A002004540020E87900209455002017
:10192000E7790020E0550020C0230020E455002086
:1019300060390020681B0020F02900203B467A1CFB
:101940003260834C13F8022B627033607B78237013
:10195000FB1C3360BB78A3703046F0F78FF8336818
:101960002081591C1A46316012F8021B61713260E5
:101970005B78A37101242346FEF78EBE7B1C336087
:101980003B780A2B10D03046F0F784F83046F0F759
:1019900081F83046F0F77EF8FEF726BE3046F0F7C5
:1019A0006DF86C4FFFF717BABB1C33606A4B7A783F
:1019B0001A70FA1C3260BA785A703A1D3260FA789E
:1019C0009A70FEF711BE09EBC70A30468AF802107A
:1019D000F0F754F8336829F837001A46591C31607B
:1019E00012F8021B8AF8031032605A788AF8042031
:1019F000DA1C32609A788AF806201F1D376001349D
:101A0000DB788AF80530A0457FF475AEFEF7ECBDB3
:101A1000042A7EF4E9AD18E43046F0F72FF8A084EC
:101A20003046F0F72BF833687268E084D11A032946
:101A30007FF7C3AE1A46591C316012F8021BA1771A
:101A400032605B7884F820303046F0F717F833685E
:101A500072686084B1E6414A1368012423F40043AC
:101A600013602346FEF718BE3D483E493E4A3F4BB1
:101A7000036001240B6013602346FEF70DBE00F0E7
:101A80007F00032828BF0020012401F0F9FE23462F
:101A9000FEF702BE364BB9781A88012412FB00F219
:101AA000234692FBF1F2A8F80020FEF7F5BD5A1C80
:101AB00032601B78003318BF012388F8073024E513
:101AC000C40800F0070301340133E4B2294F204673
:101AD00019467B7007F0DEFB57E53046EFF7CEFF87
:101AE000A8F80E003046EFF7C9FF33687268A8F80F
:101AF0001000C6E43046EFF7C1FFA8F80A003046F0
:101B0000EFF7BCFFA8F80C0030462768EFF7B6FFE8
:101B1000788430462768EFF7B1FF33687268B8847D
:101B2000ABE401240AF046FF2346FEF7B5BD5A1C7C
:101B300032601B78E3723046EFF788FF3368E0606D
:101B40005A1C32601B7823743368726839E600BF10
:101B5000F0330020B0550020732D002058340020B1
:101B60001435002068350020D0350020F50300082A
:101B700078550020F83A00200C4B1B78DB0700D585
:101B800070470B490B68002BFAD04FF47A7202FBB6
:101B900003F39842F4D3074B1B781BB9064B9A68A2
:101BA0001B69136000230B60704700BFEF3A0020F1
:101BB00094240020882400207424002008B50BF011
:101BC0001DFA024B024ADA60FEE700BF00ED00E0BA
:101BD0000400FA059F4B1B7803B170472DE9F043D1
:101BE0009D4D2B688BB013B90BB0BDE8F0839B4EB5
:101BF0009B4A3378044601A8D75C07F019FB736849
